:020000040800F2
:100000000000022081290C08052A0C0879C906087D
:10001000052A0C08052A0C08052A0C080000000017
:10002000000000000000000000000000052A0C088D
:10003000052A0C0800000000052A0C08554A05088E
:10004000052A0C08052A0C08052A0C08052A0C08A4
:10005000052A0C08052A0C08FD290508012A0508AF
:10006000052A0508092A05080D2A0508494004083B
:100070005D40040871400408854004089940040864
:10008000AD400408C1400408052A0C08052A0C08E4
:10009000052A0C08052A0C08052A0C08112A05084F
:1000A000052A0C08052A0C08052A0C08A14A040890
:1000B000B54A0408C94A0408DD4A04086D33040837
:1000C00061330408A133040895330408052A0C0899
:1000D000052A0C0875540408815404088D5404083A
:1000E000152A0508052A0C0800000000194B040811
:1000F000694B0408914B0408054B0408D5400408DB
:10010000052A0C0825650408F14A0408052A0C088C
:1001100099540408052A0C08052A0C08B999040802
:10012000E9400408FD400408114104082541040881
:1001300039410408052A0C08052A0C08052A0C0870
:1001400000000000000000000000000000000000AF
:100150004D4104086141040875410408A554040890
:10016000D5330408C9330408052A0C08052A0C08ED
:10017000052A0C08052A0C08052A0C0800000000B6
:10018000052A0C08052A0C08B1540408BD540408BB
:10019000052A0C08052A0C08052A0C08052A0C0853
:1001A000052A0C08052A0C08052A0C08052A0C0843
:1001B000052A0C08052A0C08052A0C08052A0C0833
:1001C000052A0C08052A0C08052A0C08052A0C0823
:1001D000052A0C08C9850408052A0C08052A0C08FC
:1001E000052A0C08052A0C08052A0C08052A0C0803
:1001F000052A0C08052A0C08052A0C08052A0C08F3
:10020000052A0C08052A0C08052A0C08052A0C08E2
:100210002D4B0408414B0408554B0408052A0C08D3
:10022000052A0C08052A0C08052A0C080000000005
:1002300029650408052A0C0800000000052A0C089E
:10024000052A0C08052A0C08052A0C08052A0C08A2
:10025000052A0C08052A0C08052A0C08052A0C0892
:10026000052A0C08052A0C08052A0C08052A0C0882
:10027000052A0C08052A0C08052A0C0800000000B5
:10028000052A0C0800000000052A0C0800000000E8
:0802900000000000052A0C0823
:08029800E8190C000100000050
:1002A00088AD01240201000002001400A8AD012461
:1002B0000202000002001400C8AD0124020B00007D
:1002C00002001400E8AD0124020300000400140041
:1002D00008AE0124020800000400140028AE012426
:1002E000010C00000001770048AE0124010D000060
:1002F0000001760068AE01240111000000017600C3
:1003000088AE0124010E010000017700A8AE01248F
:100310000113000000017600C8AE012401150000A1
:1003200000001E00E8AE0124011B000000000D00CB
:1003300008AF0124011C000000002C0028AF01249C
:100340000116000000000C0048AF01240117000056
:1003500000000C0068AF0124011D000000000E0029
:1003600088AF0124011E000000001E00A8AF012478
:100370000118000000000C00C8AF012401190000A2
:1003800000000E00E8AF0124011A000000000C007C
:1003900008B001240120000000000C0028B0012456
:1003A0000121000000000C0048B00124012A0100D6
:1003B0000001180068B0012401220000000148007B
:1003C00088B001240123000000014900A8B00124E5
:1003D0000124000000014A00C8B0012401250000EA
:1003E00000014B00E8B001240126000000014C0090
:1003F00008B101240127000000014D0028B10124AB
:100400000128000000014E0048B10124012900002C
:1004100000014F0068B10124012D000000002900F7
:1004200088B10124012E010000002900A8B1012497
:10043000012F010000007000C8B10124013100004B
:1004400000003100E8B10124013001000000520039
:1004500008B20124013201000001280028B2012461
:10046000013300000001760048B20124013401008C
:100470000001280068B201240137000000003C00A0
:0C04800088B20124013A000000002000B6
:020000040804EE
:10000000836B5A6D12F0500F5A6D1AD1196842F471
:1000100000725A650A6812F0080FCA6816D012F406
:10002000406F15D1CA68920412D45A6D22F48072BE
:100030005A655A6DD1040BD45A6D42F001025A65CB
:100040007047D20604D4DB6CDB6C18479007ECD009
:10005000704700BF704700BF836B5A6D42F040028B
:100060005A659A6D42F004029A65704702685549D4
:1000700038B5554B554D564CAA4218BF9A420CBF45
:10008000012300238A4208BF43F001033031A2421A
:1000900008BF43F0010330348A4208BF43F0010334
:1000A0003031A24208BF43F0010330348A4208BF16
:1000B00043F0010301F55C71A24208BF43F0010364
:1000C00004F55C748A4208BF43F001033031A24258
:1000D00008BF43F0010330348A4208BF43F00103F4
:1000E0003031A24208BF43F0010330348A4208BFD6
:1000F00043F001033031A24208BF43F001038A42BA
:1001000008BF43F0010313B9324B9A4208D10423CC
:1001100080F83530136823F001031360002038BDE8
:100120002D4B2E4D1168AA4218BF9A422C4C21F03B
:100130000E0105F13C050CBF012300231160A24212
:1001400008BF43F0010311682834AA4208BF43F0F6
:10015000010321F00101A24208BF43F0010314345E
:100160001160A24208BF43F001031E498A4208BF42
:1001700043F0010313B91C4B9A4217D10123856D3B
:10018000D0E91714226801F01F0122F480728B401D
:1001900022606B60C36ED0E91921516033B11A68D7
:1001A000D0E91C1422F480721A604C6001210022F4
:1001B000036D80F8351080F83420002BAED09847BE
:1001C000ACE700BF4000024010000240280002409F
:1001D00058000240B80402401C5402580854025807
:1001E0003054025880540258945402580168002236
:1001F0000B6880F842205A0410B40ED50B6823F423
:1002000080430B6090F84130292B10D090F841309A
:100210002A2B24D05DF8044B70471B04F2D50B68E1
:1002200023F400430B6090F84130292BEED12822B3
:10023000212380F841200022036390F841300C68AC
:1002400003F02803282B14BF6FF0F2036FF0420372
:1002500023405DF8044B0B6080F840207047282253
:10026000222380F841200022036390F841300C687B
:1002700003F02803282B14BF6FF0F4036FF044033E
:1002800023405DF8044B0B6080F84020704700BFAE
:100290000023202210B4174C4363C462036380F828
:1002A000412080F842304B07026811D5526A436AF8
:1002B0001A70436A028D013343624AB1438D013A99
:1002C000013B02859BB24385436C43F004034364C6
:1002D0000368102490F84120002190F841201A680A
:1002E00022F0FE021A60DC615DF8044B80F84010D9
:1002F000704700BF0000FFFF70B5574B002590F816
:100300004120044680F84250283AC3624585436C38
:10031000022A41EA0301036841642FD890F8411092
:1003200090F84120282001F0280102F02802282915
:1003300014BFF6214621282A1A680CBFC9436FF062
:10034000F6010A4045491A6084F84100A06B226B0F
:10035000616318B1112A42D0212A40D0E06B18B154
:10036000122A51D0222A4FD094F84130602B4FF0FE
:1003700000032DD0236384F8403070BD90F84120F5
:1003800090F841201A6822F0FE021A609A699207DA
:1003900000D59D629A69D60703D49A6942F001029A
:1003A0009A6194F84120602A10D0202284F84120DC
:1003B0009A6995060AD59A69D00605D51022DA61A0
:1003C000626C42F0040262642022DA610021BDE71F
:1003D000202284F8403084F84120236370BD1A68DD
:1003E00051042CD490F83530012BBDD000221C4B89
:1003F000036584F8402090F83520022A24D080221A
:100400004265BDE8704018471A68120403D51A689F
:1004100022F400421A6090F83530012BA4D000225B
:100420000F4B036584F8402090F83520022AE6D16E
:10043000FFF71CFE0028A0D0E06B036DE1E71A680F
:1004400022F480421A60CDE7FFF710FE002894D016
:10045000A06B036DD5E700BF0000FFFFDD040408BB
:100460002D08040803689A69196810B4D40528D5C2
:100470000C0606D4416C11F00B0F1FD15DF8044B34
:100480007047416C4FF4807441F0010141645105A3
:10049000DC6120D5416C4FF48064920541F0080185
:1004A0004164DC61E6D5426C4FF4007142F0020217
:1004B0004264D961416C11F00B0FDFD05DF8044B41
:1004C0001AE7540502D50906E4D4D3E79405D1D53B
:1004D0000906E8D4CEE79205E5D4CBE7F8B590F865
:1004E00040300D46C16A012B00F008810123AE06A1
:1004F000044680F8403001D5900656D4EB0619D555
:10050000D70617D5638D9BB2002B40F0F98094F885
:100510004130B1F1007FDBB240F0D580282B40F0B4
:10052000D28029462046FFF7B3FE0023184684F800
:100530004030F8BD68071AD42F0701D516074AD4F2
:10054000A807F2D59307F0D5638D9BB2002B00F07E
:10055000FA80616A236811F8010B228D9862638D1D
:10056000013A6162013B22859BB26385DDE7530757
:10057000E2D5638D9BB26BB12268636A526A1A70CE
:10058000638D606A228D013B0130013A9BB260624B
:1005900022856385638D9BB2002BC6D111F5803F08
:1005A000C3D02046FFF722FEBFE72368202118684A
:1005B000E66A94F84120D961213A092A1ED8DFE879
:1005C00012F0C70015001D001D001D001D001D00BC
:1005D000F000C700150094F84130226803F02803AA
:1005E000282B00F0C5800823D3619EE794F84120B2
:1005F0001A6822F0FC021A60222222635A68894992
:1006000042F400425A605A680A405A609A69910757
:1006100001D500229A629A69D20703D49A6942F0FE
:1006200001029A6147047BD51A6822F480421A605D
:10063000A26B1AB111684A6892B262856A070BD53B
:100640005A6A25F00405636A1A70636A01336362AB
:10065000238D002B40F08580638D9BB21BB1636CB2
:1006600043F004036364EB061AD5C70618D5638DFF
:100670009BB2002B40F0AA8094F84130282B03D184
:10068000B6F1007F00F0C98094F8413016F5803F44
:100690002268DBB202D0292B00F0AD801023D36199
:1006A000002384F84230666C6363002E40F084803F
:1006B000E36A5D4DAB423DD194F84130202384F88C
:1006C0004130266331E794F841202368292A4FF00E
:1006D0001002DA617FF429AF11F5803F3FF425AFB6
:1006E0009A69960701D500229A629A69D5073FF563
:1006F00058AF9A6942F001029A6152E70220F8BDB0
:1007000023681022DA61636C43F00403636431F000
:1007100080737FF40AAF616C2046FFF7EDFD04E7BC
:1007200001048BD51A6822F400421A60E26B002A99
:1007300080D183E72046FFF759FD2023E56284F846
:1007400041302663F1E631F080737FF4EEAE28E7A6
:1007500094F841201A6822F0FA021A6021222263DA
:100760004CE7013B2385638D013B9BB2638573E7B7
:10077000E1689369022990699368D56836D1C3F31B
:10078000C21383EA104313F006032FD1A16C013189
:10079000A164A16C02297FF4C8AE0821A364D161D1
:1007A000C3E694F8412094F841201A6822F0FE0232
:1007B0001A600022226321E7616C2046FFF79CFD4E
:1007C00094F84130282B7FF4B0AEAAE623681022BB
:1007D000DA61636C43F00403636436F080737FF482
:1007E0005FAF616C2046FFF787FD59E7136823F080
:1007F000B803136099E61023D3619369980701D574
:10080000002393629369D90703D4936943F00103EA
:1008100093612046FFF7EAFC42E729462046FFF7AE
:1008200037FD3DE700E800FE0000FFFF836B9A6B99
:100830000AB100211165DA6B0AB10021116593F844
:100840004120602A05D000221A63002283F840204C
:1008500070470022202183F841101A63002283F898
:1008600040207047016870B4CC072DD5914A1369B8
:10087000926A03F03803102B00F0E180182B00F08F
:10088000D9804368B3F5803F00F00581002B00F06C
:100890005A81B3F5A02F874B1A6800F0678222F4C3
:1008A00080321A601A6822F480221A60824B41F268
:1008B000883C804C1D6804E01A68521B624500F2B7
:1008C0003F8122689603F7D58A0768D4CD0631D5D3
:1008D000784A1369926A03F03803082B00F0C0804D
:1008E000182B00F0B880C369724C002B00F05F81B8
:1008F0002268714B42F0800222601D6804E01A6891
:10090000521B022A00F21C812268D205F7D56B4BDC
:10091000026A1D6841F20303B3EB154FC0F0448235
:100920006368202A23F0F8430CBF43F0804343EA76
:10093000826363600D0713D543695E4C002B00F0A2
:100940001881626F5C4B42F0010262671D6804E02F
:100950001A68521B022A00F2F380626F9207F7D5E1
:100960008C0613D58369534C002B00F0118122684B
:10097000514B42F4805222601D6804E01A68521BF9
:10098000022A00F2DD8022689204F7D5490700F1BF
:100990008880436A002B40F0BC80002059E0454A23
:1009A0001369926A13F038032BD1424AC368126864
:1009B000520701D5002B4BD03E4C226822F0190281
:1009C0001A433D4B22601D6804E01A68521B022A3C
:1009D00000F2B68022685607F7D5384B02691D68C9
:1009E00041F20303B3EB154F6368C0F0028123F4B7
:1009F0007C33402A0CBF43F4003343EA0233636084
:100A000064E7182B00F0F180C3682A4C002B00F03B
:100A1000DD80226822F019021A43274B22601D68EC
:100A200004E01A68521B022A00F28A8022685207E8
:100A3000F7D5D2E702F00302022A7FF422AF1D4B62
:100A40001B689B037FF540AF4368002B7FF43CAFEE
:100A5000012070BC704702F00302012A7FF443AF0B
:100A6000144B1B68DC0502D5C369802BF0D1134CF5
:100A700041F20303026A2468B3EB144FC0F0BF8055
:100A8000202A00F09E810B4C636823F0F84343EA70
:100A9000826363604EE7074A136843F48033136050
:100AA00004E70749044B0A6842F480720A601C6834
:100AB0000CE000BF00440258802C00240010005CB1
:100AC000004802581A68121B642A39D80A68D505EA
:100AD000F8D58268012A00F06E81002A00F04E816C
:100AE000052A9F4A116F00F0748121F001011167FE
:100AF000116F21F0040111671D6841F28834984993
:100B000003E01A68521BA2421AD80A6F9207F8D55E
:100B10003FE793490A6902F03802182A00F0D580AD
:100B20000A68022B8F4B22F080720A606FD018681F
:100B30000A6892017FF531AF1A68121A022AF7D9B2
:100B4000032070BC7047864C41F28835854B226883
:100B500022F480322260226822F4802222601E6801
:100B600003E01A68921BAA42EAD822689203F8D4DA
:100B7000AAE6626F7B4B22F0010262671D6803E008
:100B80001A68521B022ADBD8626F9607F8D4E7E690
:100B90002268744B22F4805222601D6803E01A68B8
:100BA000521B022ACCD822689604F8D4EEE62268BA
:100BB0006C4B22F0800222601D6803E01A68521B11
:100BC000022ABDD82268D605F8D4B3E62268654B60
:100BD00022F0010222601D6803E01A68521B022AFB
:100BE000AED822685607F8D470E694077FF40CAFAD
:100BF000DBE623F0FE4343EA0263636066E6584C9B
:100C0000E36823F07C5343EA0263E36092E61C68E6
:100C100003E01A68121B022A92D80A689501F8D4D8
:100C20008C6A514A2240846A2243C46A42EA04120E
:100C30008A62D0E90D24013A013C5202240492B2A6
:100C400004F4FE042243046B013CC4F30804224371
:100C5000C46B013C240604F0FE4422430A63CA6AC2
:100C600022F00102CA624A6B846C6FF3CF0242EA3F
:100C7000C4024A63CA6A046C22F00C022243384C54
:100C8000CA62CA6A406C22F002020243CA62CA6A9D
:100C900042F48032CA62CA6A42F40032CA62CA6A44
:100CA00042F48022CA62CA6A42F00102CA620A6839
:100CB00042F080720A601968226890013FF56DAEBB
:100CC0001A68521A022AF7D93AE7012B8A6A0D6B81
:100CD0003FF4BEAE02F00303846AA3427FF4B8AED1
:100CE000C2F30512C36A9A427FF4B2AE036BC5F336
:100CF0000802013B9A427FF4ABAE436BC5F3462238
:100D0000013B9A427FF4A4AE836BC5F30642013BDC
:100D10009A427FF49DAEC36BC5F30665013B9D42CD
:100D20007FF496AE4B6B816CC3F3CC0399423FF4D6
:100D300034AE0B480B4BC26A22F00102C2621A6841
:100D400018688242FCD0064A536B6FF3CF0343EA24
:100D5000C1035363D36A43F00103D3621DE600BFAE
:100D600000440258802C00240CFCFFFF42F4802237
:100D70001A601A6842F480321A6097E5194941F204
:100D800088350A6F22F001020A670A6F22F0040216
:100D90000A671C6804E01A68121BAA423FF6D0AE2C
:100DA0000A6F9607F7D4F4E5E36823F07C5343EA2F
:100DB0000263E360BEE50B490A6F42F001020A6775
:100DC0009AE6084A536823F0F84343F0804353609F
:100DD000B0E541F004011167116F41F001011167A5
:100DE0008AE600BF00440258334B30B4996A9C6ACB
:100DF000DD6A14F47C7F5A6BC4F3051036D0C2F35D
:100E0000CC0205F0010501F0030107EE900A05FB95
:100E100002F20129B8EEE77A06EE902AFAEEE96AC4
:100E200002D0022942D019B3DFED247A87EE876A17
:100E30001B6BC3F3080307EE903AF7EE005AF8EE87
:100E4000E77A77EEA67A77EEA57A67EE867A1A4B7E
:100E50001B6BC3F34623013307EE103AF8EEC76A63
:100E600087EEA67AFCEEC77A17EE900A30BC704780
:100E70001A6892061DD51968F7EE005A104A1B6BC6
:100E8000C1F3C101C3F30803CA4007EE903A06EE6E
:100E9000102AF8EEE77AB8EEC66A77EEA66AC6EED2
:100EA000077A36EEA57A67EE877AD0E7DFED057A26
:100EB000BCE7DFED057AB9E7004402580024744A24
:100EC0000090D00320BCBE4B0024744C836A1A07E8
:100ED00010B406D50168846B4A6822F400422243AC
:100EE0004A60DC0706D50168C46A4A6822F4003209
:100EF00022434A60990706D50168046B4A6822F4C8
:100F0000803222434A605A0706D50168446B4A681A
:100F100022F4802222434A60DC0606D50168C46BB5
:100F20008A6822F4805222438A60990606D50168B5
:100F3000046C8A6822F4005222438A605A060AD559
:100F40000168446C4A68B4F5801F22F4801242EABA
:100F500004024A600BD01B0606D50268C16C5368B8
:100F600023F400230B4353605DF8044B70474A6839
:100F7000846C22F4C00222434A60ECE70022836BB7
:100F8000A3F85E20704700BF124B41F2883C124A22
:100F900001461B68A2FB03235B0A0CFB03F33BB176
:100FA0004A6B12F0450F01D0920404D5013BF7D1F2
:100FB0004FF0004070474B6B5B0707D4486B10F055
:100FC000010014BF0123054B8B63704704231846AF
:100FD0008B63704700000024D34D6210C5002000D1
:100FE000036942681F2B70B432D9A3F12005202475
:100FF0005168AC40214229D08169087C032838D04F
:10100000087C022801D10020087448681F2BC96899
:10101000046906684D68C4F303244079164931F821
:10102000100001EB840100F4F0508C68F16821EAB3
:101030000001F1601149085D295821F00101295092
:1010400011D9A3F1200120238B40D36070BC7047DD
:10105000202411689C402142F8D08169087C032833
:10106000CED19460F2E7202101FA03F370BC9360C3
:101070007047D460EAE700BFF0770C0860790C088D
:10108000D0E907239A423CBFC1685218D01A704772
:10109000D0E9092300699A4238BF12180138D31ADF
:1010A000C01A7047D0E90902101AB0FA80F040095E
:1010B000704700BF016A034640694A1C405CD9681A
:1010C0008A4228BF00221A62704700BF436A8269C1
:1010D00010B4D154436A416B046901330A68A342D6
:1010E00028BF00235DF8044B42F0800243620A608F
:1010F000704700BF436BD86910F0100002D0102277
:1011000001201A62704700BF024B01F00101197102
:10111000704700BF00000024704700BF704700BF49
:10112000704700BF01207047034B58689B68C01A86
:10113000C0F30B00704700BF802C0024074B93F8CE
:10114000A822012A01D10020704793F8A832032B6E
:10115000F9D1034B1879C0B2704700BF802C00242E
:1011600000000024012380F849307047EFF311821A
:10117000702383F312880849D2B2D1E9BA3182F3DD
:101180001188581E8B42A0EB01008CBF0023012365
:1011900000EB0330704700BF802C002470B5D0F8FE
:1011A000D442D0F8C86200EB840EDEF8C05245B3DA
:1011B00001F00F040A4604EB840C00EB8C0CDCF805
:1011C00018306BB9DEF8C43200211B69C5F814125F
:1011D00023B105F50471D5F808029847002070BDC9
:1011E00004EBC40406EB8406F469B3FBF4F604FBD9
:1011F0001633002BE6D11A46CCF818307FF0E4F90C
:10120000ECE7032070BD00BFD0F8D42200EB8202CF
:1012100010B5D2F8C042ACB101F00F03D0F8C8024B
:10122000D2F8C42204F5037103EBC303D26800EBC8
:101230008303D4F80402D3F86832C4F80C32904720
:10124000002010BD032010BDD0F8D43200EB830085
:1012500010B5D0F8C04284B1D0F8C4325BB194F874
:101260000002FF2807D09B68214694F80122984786
:10127000FF2384F80032002010BD032010BD00BF02
:1012800030B52B4C8646237A65899D4242D9184653
:10129000083419461A4602E0954246D921780C4492
:1012A0000A44617892B20529F6D1A1788229F3D156
:1012B0009C461A461F4903E0AA4234D291F800C066
:1012C0006144624491F801C092B2BCF1050FF3D1C0
:1012D00091F802C0BCF1010FEED1164A02E0A8421B
:1012E0001DD213781A44034492F801C098B2BCF19D
:1012F000050FF4D19378812BF1D10CB11023A37198
:1013000019B10020022308714B711AB10021022388
:101310001171537143230748AEF8003030BD0022ED
:10132000002CEBD1ECE70021D7E70024C0E700BF99
:10133000000000240800002430B52B4C8646237A98
:1013400065899D4242D91846083419461A4602E07A
:10135000954246D921780C440A44617892B2052915
:10136000F6D1A1788229F3D19C461A461F4903E0A1
:10137000AA4234D291F800C06144624491F801C09D
:1013800092B2BCF1050FF3D191F802C0BCF1010F8C
:10139000EED1164A02E0A8421DD213781A44034443
:1013A00092F801C098B2BCF1050FF4D19378812B6B
:1013B000F1D10CB11023A37119B100204023487161
:1013C0000B711AB100214023517113714323074857
:1013D000AEF8003030BD0022002CEBD1ECE700214C
:1013E000D7E70024C0E700BF000000240800002465
:1013F000A2E700BF03460A2201481A80704700BFD7
:101400004C000024064B4FF0120C064AA3F11400C6
:10141000526DA1F800C0022A18BF1846704700BFDD
:101420006C00002400400058042301480B807047E2
:10143000800000242DE9F047046982B0C3681C4095
:1014400046D0814688464FF0004501F1500701F132
:101450003806B4FA84F325FA03F21B3BD243144056
:10146000C9F81020B8F1000F5FD0042B2ED8DFE8A8
:1014700003F052483D320300D8F81030D9F82CA0C0
:1014800033B19B6823B11FFA8AF108F1080098472D
:10149000D8F8283033B19B6823B11FFA8AF108F1DC
:1014A00020009847D8F8403033B19B6823B11FFA29
:1014B0008AF108F138009847D8F8583033B19B6862
:1014C00023B11FFA8AF108F150009847002CC0D1CF
:1014D00002B0BDE8F087D8F8103008F10800D9F85C
:1014E00034105B689847002CB3D1F1E7D8F8283066
:1014F00008F12000D9F838105B689847002CA8D173
:10150000E6E7D8F840303046D9F83C105B68984799
:10151000002C9ED1DCE7D8F858303846D9F8401076
:101520005B689847002C94D1D2E7042B07D8DFE8FA
:1015300003F01903140F0A00D9F83C300193019B02
:10154000002C86D1C4E7D9F82C300193019BF7E732
:10155000D9F834300193019BF2E7D9F83830019380
:10156000019BEDE7D9F840300193019BE8E700BF0C
:10157000174A10B55368906891681B1AC3F30B03A0
:10158000002BF7D0B1F5805F0AD04B1C1148C3F394
:101590000B03445C936092F8F0324BB9204610BDC7
:1015A00001230C49936092F8F0320C78002BF5D0AF
:1015B0009368516803F6FF735B1AC3F30B03802B28
:1015C000ECD9002382F8F03277F05AFD204610BDA6
:1015D000802C002410360024F8B5104D95F8A83260
:1015E000012B00D1F8BD95F8A832032BFAD10C4B92
:1015F0001B79002BF6D00F461446D5F8F46208E0AC
:1016000008F080FAD5F8F432241A07449B1B322BD9
:10161000E8D8002C21463846F2DCF8BD802C0024A6
:1016200000000024F8B590F848305D1C0344EDB28A
:1016300080F8485083F8341090F8493053B1132D96
:1016400007D9002380F84830104F97F8A832012BB3
:1016500005D1F8BD80F84830002DF5D1F8BD97F8D8
:10166000A832032BF5D1D7F8F46200F134042946EF
:10167000204608F047FAD7F8F4322D1A04449B1B91
:10168000322BE6D8002DF2D1F8BD00BF802C00240B
:10169000F8B5002390F84850A0F8483005B9F8BDD7
:1016A0000D4F97F8A832012BF9D097F8A832032BE9
:1016B000F5D1D7F8F46200F134042946204608F049
:1016C00021FAD7F8F4322D1A04449B1B322BE6D8AA
:1016D000002DF2D1F8BD00BF802C00242DE9F0418F
:1016E000012104464FF4077085F0D4FC054600281C
:1016F0006CD0D4F8D46204EB8606C6F8C002237C12
:10170000C4F8BC02002B40D0402302228121204695
:101710007EF0CCFC012140230222204621877EF06E
:10172000C5FC4FF001080823032282212046A4F8BB
:1017300078817EF0BBFC294B0027E364D6F8C432E5
:10174000C5F804721B689847D5F80402C5F81472EE
:10175000C5F8187200283ED0227CD4F8C83222BBCB
:10176000C3F88C224FF400749A7903F51E71C3F804
:101770008402012AA3F87882C3F8884223D018682B
:101780007EF012FE0020BDE8F08120464FF4007389
:10179000022281217EF08AFC01214FF40073022293
:1017A000204621877EF082FCBBE79A79402403F52E
:1017B0001E71C3F88C72012AC3F88402A3F87882E0
:1017C000C3F88842DBD1C3F89402D8E7D4F8D43206
:1017D000B03344F823000220BDE8F081010010007E
:1017E000F8B5D0F8C85240F20112044695F8943486
:1017F0002A87012B3ED00126002728683246314631
:1018000085F894647EF060FF27873A463146286861
:10181000A5F8786285F894647EF056FF4FF48173E2
:10182000A4F8787132460221286885F89464A5F8F6
:101830005C307EF049FF85F89474D4F8D4320025EA
:1018400004EB8303E564D3F8C0228AB1D3F8C43231
:101850005B689847D4F8D432B03354F8230085F04D
:101860003DFCD4F8D432B03344F82350C4F8BC5211
:101870000020F8BD00224FF481710287A5F878326C
:10188000A0F87821A5F85C10D7E700BFD0F8D432D3
:1018900000EB8303F0B5002683B0D3F8C0728DF857
:1018A0000560ADF806605FB191F800C004460D46D2
:1018B0001CF060022FD0202A05D020467EF03AFD91
:1018C000032003B0F0BDCA884878002A42D01CF03B
:1018D000800F00F08380D3F8C43239469B68984764
:1018E000EA8802234FF48071072AC4F8943228BF93
:1018F0000722D4F8C832C4E906225A629A7999823A
:1019000003F11401012A1F629E6200D11F6318684F
:101910007EF04AFD22E04B780B2BCED801A252F884
:1019200023F000BF611904085D190408BB180408FE
:10193000BB180408BB180408BB180408BB1804082B
:10194000BB180408BB180408BB180408A119040834
:1019500097190408D3F8C4329B6898470020B0E771
:1019600090F89C32032BA8D10222D0F8C832002074
:10197000C4F8942203F11401C4E906220DF106040F
:101980009862C3E908424FF480729A829A79012AD8
:10199000BDD11C63BBE790F89C32032BDED08CE7F3
:1019A00090F89C32032B88D101220221D0F8C83252
:1019B000C0F8941203F11401C0E906220DF10500EC
:1019C000C3E908024FF4807200209A829A799862E3
:1019D000012A9CD10DF10500186398E7402A4FF0C9
:1019E000030387F8000228BF402287F80122C4F8C9
:1019F0009432D4F8C832C4F85821C4F85C2103F5F5
:101A00001571C3F864229A79C3F86072012AC3F889
:101A10006862A3F8546208BFC3F8707277E700BF2A
:101A200070B5124D124A2B68A2FB03239B09013BA0
:101A3000B3F1807F01D3012070BD4FF0E0220D494A
:101A400000240F2853614FF0F003064681F823303D
:101A50004FF0070394611361EDD801464FF0FF305A
:101A600076F048FF2046C5F8846070BD0000002471
:101A7000D34D621000ED00E03749024603688B4207
:101A800033D01831591AB1FA81F1490969BB334889
:101A9000834240D01830834240D01830834236D041
:101AA000183083423DD01830834240D018308342F2
:101AB0002CD000F55670834237D029498B4233D061
:101AC00018318B4236D018318B4236D018318B42C8
:101AD00036D018318B4236D018318B4236D018317F
:101AE0008B4236D023F0FF0013E0DBB21D491E48C5
:101AF000103B10B41D4CA4FB03435DF8044B01EBF9
:101B0000131393F82810C2E91601704716211848DC
:101B1000D1659065704710211348F9E716211248E6
:101B2000F6E706211248F3E706211248F0E71021F4
:101B30000F48EDE710210F48EAE716210D48E7E7C7
:101B400000210D48E4E706210B48E1E710210A488F
:101B5000DEE716210848DBE71000024040000240A3
:101B600028040240F0770C0800000240ABAAAAAAA1
:101B7000040002400004024004040240F0B50C4698
:101B8000114602688646936913F0100C72D04FF02C
:101B9000000C102338486546D36193699E065FD4D4
:101BA00045B903685B1AA3423DD893699F06F8D5EF
:101BB0002023D3614CF0040C01209369D90552D540
:101BC0004FF480715F054CF0010CD16104D54FF4E6
:101BD00080614CF0080CD1619D0504D54FF4007371
:101BE0004CF0020CD3619369990701D500239362ED
:101BF0009369DB0703D4936943F00103936153684E
:101C000020241E4901200B4000215360DEF844309F
:101C10008EF8401043EA0C03CEF844308EF8414071
:101C20008EF84210F0BD57689EF842309669DBB2DC
:101C3000360408D57E0406D4202B04D0536843F420
:101C400080435360016893699F06A6D403685B1ABA
:101C5000192BF8D993694FF0200C01259E069FD5CA
:101C6000002DA5D0A6E75E05B1D49C05B6D400280A
:101C7000B9D1F0BD6046A0E7802C002400E800FE4A
:101C80002DE9F04707689A46089EBB6931EA0303CD
:101C90000CBF01230023934220D180460C461546F9
:101CA000DFF85C90324651464046FFF767FF20BBA5
:101CB000D9F80030A3EB060CD44507D9BB6934EA48
:101CC00003030CBF01230023AB420AD0BB6934EAF3
:101CD00003030CBF01230023AB42E3D00020BDE887
:101CE000F087D8F84430202288F840001343C8F821
:101CF000443088F8412088F842000120BDE8F08790
:101D0000802C00240C4A136903F03803102B0DD0EB
:101D1000182B09D063B913689B060BD513680748C5
:101D2000C3F3C103D8407047FFF75EB8044870475B
:101D30000448704701487047004402580090D0039F
:101D400040787D0100093D00184A136903F038030B
:101D5000102B10B524D0182B09D01BBB13689B0681
:101D600022D513681248C3F3C103D84001E0FFF73E
:101D70003BF80E490F4A8B698969C3F303230E4C64
:101D800001F00F0113440A4493F8301092F83030F8
:101D900001F01F0203F01F03D0402060D84010BDA7
:101DA0000648E6E70648E4E70148E2E7004402584F
:101DB0000090D003F0770C080000002440787D01EB
:101DC00000093D00474A70B4946A956AD66A15F4D2
:101DD0007C3FC5F30533D16B5BD0C1F3CC01C6F3B7
:101DE000001604F0030407EE903A06FB01F1012C03
:101DF000B8EEE77A06EE901AFAEEE96A03D0022C02
:101E00006AD0002C4AD0DFED387A87EE876A936B70
:101E1000C3F3080307EE903AF7EE005AF8EEE77ABC
:101E200077EEA67A77EEA57A67EE867A2D4AB7EE38
:101E3000006A936BC3F3462307EE103AB8EEC77AF5
:101E400070BC37EE067AC7EE876AFCEEE66AC0ED34
:101E5000006A936BC3F3064307EE103AB8EEC77AF5
:101E600037EE067AC7EE876AFCEEE66AC0ED016AD5
:101E7000936BC3F3066306EE903AF8EEE66A76EEED
:101E8000866A87EEA67AFCEEC77A17EE903A8360F0
:101E9000704770BCC0E900338360704713689B06CD
:101EA0001DD51468F7EE005A936B1049C4F3C102B4
:101EB000C3F30803D14007EE903A06EE101AF8EE8D
:101EC000E77AB8EEC66A77EEA66AC6EE077A36EE0D
:101ED000A57A67EE877AA9E7DFED057A95E7DFED6A
:101EE000057A92E7004402580024744A0090D00317
:101EF00020BCBE4B0024744C474A70B4946A956A67
:101F0000D66A15F07C7FC5F30553516C5BD0C1F3E5
:101F1000CC01C6F3002604F0030407EE903A06FB5A
:101F200001F1012CB8EEE77A06EE901AFAEEE96AB2
:101F300003D0022C6AD0002C4AD0DFED387A87EE2D
:101F4000876A136CC3F3080307EE903AF7EE005A62
:101F5000F8EEE77A77EEA67A77EEA57A67EE867ADC
:101F60002D4AB7EE006A136CC3F3462307EE103A0E
:101F7000B8EEC77A70BC37EE067AC7EE876AFCEE19
:101F8000E66AC0ED006A136CC3F3064307EE103A2D
:101F9000B8EEC77A37EE067AC7EE876AFCEEE66AD5
:101FA000C0ED016A136CC3F3066306EE903AF8EED7
:101FB000E66A76EE866A87EEA67AFCEEC77A17EEB8
:101FC000903A8360704770BCC0E90033836070470B
:101FD00013689B061DD51468F7EE005A136C104960
:101FE000C4F3C102C3F30803D14007EE903A06EEF2
:101FF000101AF8EEE77AB8EEC66A77EEA66AC6EE71
:10200000077A36EEA57A67EE877AA9E7DFED057ADB
:1020100095E7DFED057A92E7004402580024744A00
:102020000090D00320BCBE4B0024744C026983682E
:1020300070B5044605681343C069626986B02968B3
:102040001343AC4A03430A40616A1343E2682B60BE
:102050006B6823F440531343A2696B60A64B9D4207
:1020600000F06681236AAE681A43A44B33401A43DA
:10207000AA60EB6A23F00F030B43EB62A04B9D4277
:1020800028D0A04B9D421AD09F4B9D4217D09F4B0A
:102090009D4214D09E4B9D4211D09E4B9D4219D023
:1020A0009D4B9D420BD09D4B9D4208D001200023AB
:1020B0004FF001126367A266A36706B070BD984B2C
:1020C0005B6D03F00703052BF0D8DFE803F09F7F7B
:1020D0008A925F79924B5B6D03F03803282BE5D829
:1020E00001A252F823F000BF95220408AD20040895
:1020F000AD200408AD200408AD200408AD2004087C
:10210000AD200408AD200408CD210408AD2004084A
:10211000AD200408AD200408AD200408AD2004085B
:10212000AD200408AD200408E3210408AD20040814
:10213000AD200408AD200408AD200408AD2004083B
:10214000AD200408AD200408F3210408AD200408E4
:10215000AD200408AD200408AD200408AD2004081B
:10216000AD200408AD2004088D210408AD2004082A
:10217000AD200408AD200408AD200408AD200408FB
:10218000AD200408AD200408C1210408B0F5004FBB
:10219000644853D0644B626803EB4103B3F84030AA
:1021A000B0FBF3F000EB52004FF6EF73B0FBF2F030
:1021B000A0F110029A423FF679AFE860002076E77E
:1021C000B0F5004F3AD04FF40040E3E7B0F5004FD0
:1021D0002DD003A8FFF7F6FD04980028EED0616A21
:1021E000D8E7B0F5004F71D06846FFF785FE01983B
:1021F000F3E7B0F5004F5ED0494B1A68920639D527
:102200001B684A48C3F3C103D840C3E7B0F5004F89
:1022100032D0FFF799FD424A434BD269C2F3021212
:10222000134493F8303003F01F03D840D5E703A8D8
:10223000FFF7C8FD04980028C0D0616A3A4B626875
:1022400003EB41034FF6EF71B3F84030B0FBF3F00E
:10225000530803EB4003B3FBF2F3A3F110028A42ED
:102260003FF624AF23F00F02C3F3420392B21343AD
:10227000EB60A3E72D488DE7FFF766FD284A2A4B60
:10228000D269C2F30212134493F8303003F01F03F3
:10229000D840D0E7B0F5004F1DD0FFF755FD204ADC
:1022A000214BD269C2F30222134493F8303003F079
:1022B0001F03D84091E71A4B1A68900640F1A58099
:1022C0001B681A48C3F3C103D840B7E76846FFF755
:1022D00013FE0198AFE7FFF737FD114A124BD269A1
:1022E000C2F30222134493F8303003F01F03D840A6
:1022F000A1E700BFF369FFCF000C0058FFF4FF1106
:10230000001001400044004000480040004C0040E4
:10231000005000400014014000780040007C004064
:102320000044025800093D00F0770C080090D003EB
:10233000A868374B03401343364AAB60EB6A23F07F
:102340000F030B43EB62936D03F00703052B3FF67E
:10235000ADAEDFE803F0413C3303524F2D4B1A681A
:1023600095064CD42C482D4B656803EB410305EBD7
:102370004501B3F84020B0FBF2F399423FF696AE28
:10238000B3EB053F3FF692AE0023194680F0DEFA2C
:102390002A460902030241EA1061680818184FF042
:1023A000000341F1000180F0D1FA1D4BA0F540720D
:1023B0009A423FF67BAE1B4BD860FFE66846FFF7BC
:1023C0009BFD019800283FF4F9AE616ACBE703A8B2
:1023D000FFF7F8FC0498F5E7FFF7B6FC0D4A0F4B42
:1023E000126AC2F30212134493F8303003F01F0351
:1023F000D840E7E74FF40040B5E70B48B3E71B6868
:102400000548C3F3C103D840ADE7034816E700BF52
:10241000FFF4FF11004402580090D003F0770C083D
:10242000FFFC0F00000C005800093D00474A70B443
:10243000946A956AD66A15F47C7FC5F30513516BCF
:102440005BD0C1F3CC0106F0010604F0030407EEF3
:10245000903A06FB01F1012CB8EEE77A06EE901AED
:10246000FAEEE96A4ED0022C6DD0002C4DD0DFED93
:10247000387A87EE876A136BC3F3080307EE903A46
:10248000F7EE005AF8EEE77A77EEA67A77EEA57ABD
:1024900067EE867A2D4AB7EE006A136BC3F34623C4
:1024A00007EE103AB8EEC77A70BC37EE067AC7EE80
:1024B000876AFCEEE66AC0ED006A136BC3F306435D
:1024C00007EE103AB8EEC77A37EE067AC7EE876A9B
:1024D000FCEEE66AC0ED016A136BC3F3066306EE19
:1024E000903AF8EEE66A76EE866A87EEA67AFCEE19
:1024F000C77A17EE903A8360704770BCC0E900332A
:1025000083607047DFED137AB3E713689B06AED59F
:102510001468F7EE005A136B0F49C4F3C102C3F3FA
:102520000803D14007EE903A06EE101AF8EEE77A6B
:10253000B8EEC66A77EEA66AC6EE077A36EEA57AD8
:1025400067EE877AA6E7DFED057A92E70044025846
:102550000024744C0024744A0090D00320BCBE4B6D
:10256000344A136830B423F08063334C1360256819
:1025700003E023685B1B022B54D813681B01F8D4BB
:10258000936A056823F47C3343EA053393628368D6
:10259000C568013B013D5B022D049BB205F4FE05BD
:1025A0002B434568013DC5F308052B430569013DF3
:1025B0002D0605F0FE452B439363D36A456923F04E
:1025C000C0032B43D362D36A856923F020032B43D6
:1025D000D362D36A23F01003D362D36BC0696FF365
:1025E000CF0343EAC003D363D36A43F01003D3623B
:1025F000D36AD1B101290CBF43F4801343F4001313
:10260000D3620C4A136843F080631360216803E0CF
:1026100023685B1A022B05D813681B01F8D500202C
:1026200030BC7047032030BC704743F40023D362B2
:10263000E7E700BF00440258802C0024344A1368A6
:1026400030B423F08053334C1360256803E02368D3
:102650005B1B022B54D813689B00F8D4936A05685F
:1026600023F07C7343EA055393628368C568013B9A
:10267000013D5B022D049BB205F4FE052B4345682A
:10268000013DC5F308052B430569013D2D0605F005
:10269000FE452B431364D36A456923F440632B43FF
:1026A000D362D36A856923F400732B43D362D36A60
:1026B00023F48073D362536CC0696FF3CF0343EA92
:1026C000C0035364D36A43F48073D362D36AD1B135
:1026D00001290CBF43F4000343F08073D3620C4A1A
:1026E000136843F080531360216803E023685B1A8A
:1026F000022B05D813689B00F8D5002030BC70472A
:10270000032030BC704743F48003D362E7E700BF87
:1027100000440258802C0024F0B5354AB0F1804FB7
:10272000344DA0EB02020368A0EB050E4C69B2FA2F
:1027300082F28F68BEFA8EFE0E684FEA52124FEA9E
:102740005E1E1FD0F2B9DFF8B8C0604537D00CF577
:10275000806C604533D00CF5806C604512D0BEF1C2
:10276000000F0FD1244D254A904218BFA8422AD00D
:1027700002F58062904226D023F08003C762866211
:102780001C4314E04D6823F07003D1F80CC02B43B8
:10279000C762866223F4407343EA0C0323F080038C
:1027A0001C4312B9BEF1000F16D00B690363036816
:1027B000012243F00403036042610460F0BD23F092
:1027C00070034A681343CA6823F44073C762134313
:1027D000866223F080031C43074A084B984218BFC7
:1027E0009042E2D003F580639842DED0DFE700BF7D
:1027F000000001400004014000400140004401404D
:1028000000040040026810B452E8003F23F49073C3
:1028100042E800310029F7D1144C02F1080353E8D3
:10282000003F234002F1080C4CE800310029F4D1AC
:10283000C36E012B08D0002320225DF8044BC0F8A2
:102840008C204367C366704752E8003F23F01003B3
:1028500042E800310029EED052E8003F23F0100397
:1028600042E800310029EFD1E5E700BFFEFFFFEFAE
:10287000436BDA69F0B5970683B0044642D5586ACF
:10288000E36AC0B2002B00F09580216B9847636B20
:102890001A681D4622F480721A609A6822F00102BA
:1028A0009A609A6942F008029A61DA69D6072DD4D3
:1028B000DA69900701D502221A62DA69510701D557
:1028C00004221A62DA69120701D508221A62DA694B
:1028D000170612D5D4F8BC20212A0ED0D4E909124B
:1028E0008A4273D0A169895C0132C9B299622169B7
:1028F000B2FBF1F001FB1022A262DA69560608D49D
:1029000003B0F0BDDA691D46D607D1D501221A629F
:10291000CEE7DA6940F60F0C1E6804F1340012EAC3
:102920000C0F996836D0B24F0F4040F0BB80DFF8F3
:10293000CCC216EA0C0F40F06381D4F8A050012DF0
:102940004CD0D50202D54F0200F16781150606D59D
:1029500001F4000106F080050D4340F0438151066B
:10296000CED57206CCD553E8002F22F0400243E8C2
:10297000002141B1626B52E8003F23F0400342E87E
:1029800000310029F7D120220023C4F8BC20C4F86C
:10299000AC30B5E79506D0D506F0200501F080579C
:1029A0003D43CAD0D4F8A830002BA9D003B0BDE86D
:1029B000F0401847E3696269D054E369E268013383
:1029C000B3FBF2F102FB1133E36160E70022A4F8EC
:1029D0008A201A6822F080021A608EE7D706B0D5E6
:1029E000F506AED51022B4F890501A629A685706D0
:1029F00040F11D81D4F8B40001684A6892B2002AFF
:102A000000F05081AA4280F04D81C169A4F8922063
:102A1000B1F5807F40D053E8002F22F4807243E864
:102A2000002141B1626B52E8001F21F4807142E83D
:102A30000015002DF7D103F1080252E8002F22F013
:102A4000010203F1080545E800210029F3D103F153
:102A5000080252E8002F22F0400203F1080545E881
:102A600000210029F3D12022C4F8C020C4F8A0100E
:102A700053E8002F22F0100243E80026002EF7D181
:102A80005C490D6840B190F83530022B00F013819D
:102A9000802380F8346043650223C4F8A430B4F87E
:102AA00092302DE712F0010F0CD016F4807F09D080
:102AB0004FF0010CC3F820C0D4F8C4C04CF0010C96
:102AC000C4F8C4C012F0020F7BD112F0040F0CD076
:102AD00011F0010F09D04FF0040CC3F820C0D4F856
:102AE000C4C04CF0020CC4F8C4C012F0080F0CD0E3
:102AF00006F0200C5CEA070C07D008271F62D4F808
:102B0000C47047F00807C4F8C47017050AD57701E8
:102B100008D54FF400671F62D4F8C43043F0200397
:102B2000C4F8C430D4F8C430002B3FF4E9AE9206A8
:102B30000CD506F0200601F080510E4306D0D4F8E3
:102B4000A8301BB101909847656B0198D4F8C42058
:102B5000AB6802F0280203F04003134361D0FFF793
:102B600051FEAB685B067FF5CBAE05F1080353E879
:102B7000003F23F0400305F1080141E8003262B153
:102B8000626B02F1080353E8003F23F0400302F1B7
:102B9000080040E800310029F3D1D4F8B40000283F
:102BA0003FF4AEAE90F83520134B022A03653BD1BB
:102BB000FDF75CFA00283FF4A3AED4F8B400036D2F
:102BC000F4E611F0010F90D04FF0020C12F0040F58
:102BD000C3F820C0D4F8C4C04CF0040CC4F8C4C07E
:102BE00083D078E7D4F8AC30002B7FF4DFAE87E6F3
:102BF00001000010802C00247D0F04082001000437
:102C000012F0010F3FF471AF16F4807F7FF450AFE4
:102C100012F0020F7FF469AF57E74FF480121A6287
:102C20006EE6C4F8C4306BE680224265BEE6B4F8B6
:102C30009220B4F8921092B289B2AA423FF460AEE8
:102C400000293FF45DAE53E8002F22F4907243E870
:102C5000002141B1626B52E8001F21F4907142E8FB
:102C600000100028F7D1954803F1080252E8002F20
:102C7000024003F1080545E800210029F4D1202293
:102C8000C4F8A810C4F8C020C4F8A01053E8002F5E
:102C900022F0100243E800210029F7D10223C4F8F2
:102CA000A4302DE6AA427FF42BAEC369B3F5807F32
:102CB0007FF426AEF2E70368814A824E824FB34228
:102CC00018BF934206F118060CBF01220022B3423E
:102CD00008BF42F001021836B34208BF42F00102B9
:102CE0001836B34208BF42F001021836B34208BF9B
:102CF00042F0010206F55676B34208BF42F00102E7
:102D00001836B34208BF42F001021836B34208BF7A
:102D100042F001021836B34208BF42F001021836F1
:102D2000B34208BF42F001021836B34208BF42F076
:102D300001021836B34208BF42F00102A6F59266BE
:102D4000BB4218BFB34207F592670CBF01260026AD
:102D5000BB4208BF42F0010256EA020779D0D3F81D
:102D600000C02CF01E0CC3F800C0D3F814C02CF027
:102D7000800CC3F814C0D0F860C076BBD0F860C037
:102D8000DCF8006026F48076CCF800601A6822F047
:102D900001021A6003E00A68521B052A24D81A6847
:102DA000D607F8D4D0E9165101F01F012FB33F2305
:102DB0008B40AB60C36ED0E91921516033B11A6802
:102DC000016F22F480721A60436F4B60012200236E
:102DD00080F8352080F834305EE6DCF8002022F4FC
:102DE0008072CCF80020D1E7202103220023416526
:102DF00080F8343080F835204EE6344A344EB34201
:102E000018BF934206F114060CBF01220022B34200
:102E100008BF42F001021436B34208BF42F001027B
:102E20001436B34208BF42F001021436B34208BF61
:102E300042F00102012606FA01F1696025498B4240
:102E400008BF42F00102002AB4D1234A9342B1D014
:102E5000BCE71E4EDFF878C0634518BFB3420CF1E3
:102E6000140C0CBF01260026634508BF46F001067E
:102E70000CF1140C634508BF46F001060CF1140C6C
:102E8000634508BF46F001060CF1140C634508BF0A
:102E900046F00106D3F800C02CF00E0CC3F800C0B9
:102EA000DFF830C0634508BF46F00106002E7FF40E
:102EB00065AF094EB3423FF461AF67E7FEFFFFEF36
:102EC00040000240580002402800024008540258C6
:102ED0001C54025880540258945402584B4B10B45E
:102EE0001B684B4CA4FB03435B0A03FB02F25AB181
:102EF0008446531E4748DCF83420013B024201D08F
:102F0000920406D55C1CF6D14FF000405DF8044BEE
:102F10007047DCF834305C0741D4DCF83430D80733
:102F200009D43D4BCCF83830DCF81030DBB2994294
:102F300005D00120EAE70123CCF83830F9E7DCF8C6
:102F40001430364818400028E0D0002B2CDB5A0003
:102F50002DD49C002DD4D9002DD41A012ED45C017F
:102F60002FD4D90130D41A0231D45C0232D4990260
:102F70003CD4DA0237D45C0332D499032DD4DA037B
:102F800040D41C043BD4590436D49A0431D413F0F1
:102F9000080F0CBF4FF480304FF40000B6E7042355
:102FA0001846CCF83830B1E74FF00070AEE740205B
:102FB000ACE78020AAE74FF48070A7E74FF40070D9
:102FC000A4E74FF48060A1E74FF400609EE74FF460
:102FD00080509BE74FF4005098E74FF4802095E72E
:102FE0004FF4003092E74FF400408FE74FF48040F9
:102FF0008CE74FF4800089E74FF4001086E74FF428
:10300000801083E74FF4002080E700BF0000002419
:10301000D34D621045002000C500200008E0FFFDF0
:1030200082B00023019302E00369002B09DB019BBE
:1030300001330193019BB3F1706FF5D9032002B006
:1030400070478901002341F020010193016103E0F1
:10305000036913F0200307D0019B01330193019B07
:10306000B3F1706FF4D9E9E7184602B0704700BFBA
:1030700082B00023019302E00369002B09DB019B6E
:1030800001330193019BB3F1706FF5D9032002B0B6
:103090007047002210230192036103E0036913F0DB
:1030A000100307D0019B01330193019BB3F1706FB3
:1030B000F4D9EBE7184602B0704700BF82B0002396
:1030C000019302E00369002B09DB019B01330193AB
:1030D000019BB3F1706FF5D9032002B07047002354
:1030E0000193036943F00103036103E0036913F0F3
:1030F000010307D0019B01330193019BB3F1706F72
:10310000F4D9E9E71846E8E72DE9F84305680746EA
:103110000C46C5F31009B9F1000F39D18A4B4FF6AF
:10312000FF72B3F88030934256D0002B54D0874AB8
:1031300002EA432808F10068454534BF4FF0010812
:103140004FF00208824B9D4206D903F500339D42A1
:1031500000F2CF804FF001097E4E96F80C33012B20
:1031600012D00123B8F1010F86F80C334FF00003A1
:10317000C6F8103336D0022075F068FB002800F046
:103180009980002386F80C334FF0FF30BDE8F883B8
:10319000704E96F80C33012B4CD0012386F80C337B
:1031A00005F17843B3F5801F48D3A5F10163B3F56A
:1031B000801F3FD200230220C6F8103375F046FB73
:1031C000002870D1644A4FF00208D2F80C3143EA6B
:1031D0000803C2F80C313FE0B5F1016F67D3052059
:1031E00012F068F9404675F031FB0028C9D140461D
:1031F000DFF86481D8F80C3023F4E663C8F80C30AB
:10320000D8F80C3043EA092343F0A403C8F80C3083
:1032100075F01CFBD8F80C20504B1340C8F80C304C
:103220000028AED105F178430122B3F5801F86F85E
:103230000C2303D36FF00100BDE8F88300230120C5
:10324000C6F8103375F002FB68BB434A4FF0010823
:10325000D36843F00203D360BFF36F8FBFF34F8F88
:1032600004F1200254F8043B944245F8043BF9D1A0
:10327000BFF36F8FBFF34F8F404675F0E7FAB8F199
:10328000010F354A30D0D2F80C3123F00203C2F8D6
:103290000C31002386F80C330028CBD13B68203357
:1032A0003B60BDE8F883002386F80C33C2E74FF09B
:1032B000010847E7DFF8A0800220D8F80C3123F49A
:1032C000E663C8F80C31D8F80C3143EA092343F01F
:1032D000A403C8F80C3175F0B9FAD8F80C211F4BCB
:1032E0001340C8F80C319BE7D36823F00203D36086
:1032F000CFE703F500339D4211D903F500339D421A
:1033000010D903F500339D4206D903F500339D42E1
:103310000BD84FF005091FE74FF004091CE74FF0E9
:10332000020919E74FF0030916E703F500339D4240
:1033300006D9B5F1016FBFF452AF4FF007090BE7A3
:103340004FF0060908E700BF00E8F11F00FE1F006C
:10335000FFFF0108802C002400200052FBF8FFFF33
:103360000148FDF77FB800BF982F0024084810B42B
:10337000D0F81833D0F84C4399691A682CB1234619
:1033800000F546705DF8044B18475DF8044B704734
:10339000802C00240148FDF765B800BFF02F002401
:1033A000084810B4D0F87033D0F8A44399691A686B
:1033B0002CB1234600F55C705DF8044B18475DF8AE
:1033C000044B7047802C00240148FDF74BB800BF28
:1033D00048300024084810B4D0F8C833D0F8FC4373
:1033E00099691A682CB1234600F572705DF8044B98
:1033F00018475DF8044B7047802C00242DE9F04FEE
:10340000DFF85C9300EB400583B0430009EB8505D2
:103410000093D5F888300193002B00F05E81804640
:10342000B5F88E0074F09EFD95F88C000FF09AFBB5
:10343000044695F88D000FF095FB08F1010307464F
:10344000DBB2002C00F06E8140F60C12A1882372D2
:10345000E2802268002800F05981037240F60C23B4
:10346000C38091613B68BA889A6111212046092680
:103470000FF034FB112138460FF030FB6525002C8E
:1034800000F02E812268A38811690B4200F0288188
:103490001B04936111F030FB05468B4611F02CFBA9
:1034A000401B61EB0B01052871F10001F6D314B14B
:1034B0002368A2889A6111F01FFB05468B4611F024
:1034C0001BFB401B61EB0B01052871F10001F6D3DA
:1034D000013ED3D11CB1A38822681B04936111F073
:1034E0000BFB05460E4611F007FB401B61EB060186
:1034F000052871F10001F6D31FB1BB883A681B049F
:10350000936111F0F9FA05460E4611F0F5FA401BE9
:1035100061EB0601052871F10001F6D314B12368AF
:10352000A2889A6111F0E8FA05460E4611F0E4FA15
:10353000401B61EB0601052871F10001F6D317B1BC
:103540003B68BA889A61009B20463E21434409EBC0
:10355000830393F8934022460FF0E2FA224638465E
:103560003E210FF0DDFA784C5823019A03FB084303
:10357000C3F81823754B9A4200F0C380FEF7E4FBB2
:10358000734BDA69C2F30212724B134493F8303072
:1035900003F01F03D840009B434409EB830393F8D7
:1035A0009030022B00F0B980032B00F0B180012B8A
:1035B00014BF4FF4C8714FF4487174F061FD0346B5
:1035C0005822002102FB0842C2F82013C2F81C3323
:1035D000C2E9CA11C2E9CD110121C2F8241392F83F
:1035E000591301F0FF00002900F0A480582123F0B6
:1035F000706224264FF4004701FB08415648D1F879
:10360000183381F859631D6825F001051D601A61A2
:103610009A6822F400429A609F605A6822F400621D
:103620005A605A681043D1F8302358601202D868A3
:1036300020F40040D860DA6000221A60186840F078
:10364000010018602020C1F85C2381F85903C1F8FB
:10365000482381F85A2391F859032028C5B217D17D
:1036600091F85803012813D081F85963186820F0A5
:1036700001001860186820F48050186018681860FD
:10368000186840F00100186081F8595381F85823F8
:10369000009B02210126314F434409EB830999F82D
:1036A0009250284675F026F905F01F036A0999F82B
:1036B000915006FA03F30221284647F8223075F0AC
:1036C00019F9582303FB084405F01F036D0906FA96
:1036D00003F347F8253084F8146303B0BDE8F08F96
:1036E000013D2AD011F008FA83468A4611F004FA07
:1036F000B0EB0B0061EB0A01052871F10001F5D375
:10370000BDE6FEF721FB124B1A6A3BE79161ACE67E
:10371000C82174F0B5FC034652E7642174F0B0FC94
:1037200003464DE700283FF4A0AE037240F60C2399
:10373000C38097E682F8580358E7002C3FF4AAAEFE
:10374000A3882268A4E600BF802C0024001C005837
:1037500000440258F0770C080080000200E100E00D
:10376000000000242DE9F04F441C85B017469DF859
:103770003C202DD05824DFF8A8831E46054600FBC8
:1037800004F408EB040393F81493B9F1000F1FD06D
:1037900044444900FF2F04F54674039100D0EEB96C
:1037A000002A40F0C680582303FB058393F8592371
:1037B000202A04D1B6B94FF40072C3F85C23B8F8DC
:1037C0001C34284601339BB2A8F81C34FFF716FEC0
:1037D0004FF00009484605B0BDE8F08F93F8593323
:1037E000202BECD14FF0580A0AFB058A9AF858337F
:1037F000012BE4D00122D8F800B019234FF4004186
:103800008AF858232046CDF800B0FEF739FA002890
:10381000D5D10E9BDAF81813CAF83C332123BA4AE3
:103820008AF859334023CAF84C038AF85A33CAF845
:103830005C032046AAF842634B681340039A134383
:10384000B24A1A434A60594674F0D2FF0246002831
:1038500040F0FB80DAF81833802120469F620A236B
:10386000CDF800B0FEF70CFA002840F0EE80BAF870
:1038700042339BB2FF2B40F21681DAF81813FF2374
:10388000A348AAF840334B68A24A03400398034375
:103890001A434A605826DDF80CA05F46039506FBE4
:1038A000058605E0B6F842339BB2002B00F010818C
:1038B0003946204674F09CFF002840F0F280D6F88C
:1038C0003C13D6F8185311F8012BB6F84033AA620E
:1038D000C6F83C13013BB6F842139BB20139A6F877
:1038E000403389B2A6F84213B6F8421389B2002BCE
:1038F000D8D10029D6D002460A238021204600973D
:10390000FEF7BEF9FF22002840F0CB80B6F8423324
:103910009BB2934240F2A080D6F81813A6F8402339
:103920004B687B4A13407B4A43EA0A031A434A60C6
:10393000B8E74FF0580A0AFB058A9AF85933202B4A
:103940007FF43DAF9AF85833012B3FF438AF012292
:10395000D8F8007019234FF400418AF85823204604
:103960000097FEF78DF900287FF429AF0E9BCAF867
:103970004C03CAF83C3321238AF8593310238AF8C0
:103980005A33CAF85C03AAF84263BAF842339BB2CE
:10399000FF2B00F2C780BAF842339BB2AAF840333B
:1039A000002B40F0F180DAF8181357484B685A4A58
:1039B0000340039803431A434A605826AA4606FB6D
:1039C0000586B6F8423339469BB2002B00F0D4800E
:1039D000204674F00DFF002878D1D6F83C13D6F8B5
:1039E000185311F8012BB6F84033AA62C6F83C13FD
:1039F000013BB6F842139BB20139A6F8403389B2B5
:103A0000A6F84213B6F8421389B2002BD9D1002987
:103A1000D7D002460A23802120460097FEF730F9CE
:103A2000FF22002852D1B6F842339BB2934225D9E7
:103A3000D6F81813A6F840234B68354A1340039A6A
:103A40001343344A1A434A60BBE75823002203FB5E
:103A5000058383F85823B2E6B6F84233D6F8182324
:103A60009BB22B485168A6F84033DBB201404AEACA
:103A700003430B4343F00073536013E7B6F842333C
:103A8000D6F818139BB2039A2148A6F84033DBB24C
:103A900042EA03434A680240134343F000734B6019
:103AA0008FE7039D8BE6BAF84233DAF818139BB21E
:103AB000039A1748AAF84033DBB242EA03434A6844
:103AC0000240134343F000734B60E3E6554676E64D
:103AD00039462046039D74F05DFE00287FF46FAEEA
:103AE000D6F8183320210D4CD9615A6822405A600B
:103AF0005823002286F8591303FB058386F85A03DE
:103B000083F8582366E600BF009800FC00200101FE
:103B1000009C00FC0000FF010020000200E800FE05
:103B2000802C0024FF234FF47F00FE224FF080768C
:103B3000AAF84033039BDDF838E01E4358231EF8F3
:103B400001AB03FB0583DFF850C0D3F81813C1F8AD
:103B500028A0A3F84023B3F84223C3F83CE3013A7A
:103B600092B2A3F842234B6803EA0C0333430343A6
:103B700043F400534B6020E72046554674F00AFE9C
:103B800000287FF41CAEABE7013B4FF000769AB201
:103B9000501CC0B20004CDE7009800FC2DE9F04FA6
:103BA000441C85B099469DF83C3000F0968058251D
:103BB000C64C064600FB05F504EB050B9BF814A369
:103BC000BAF1000F00F089802544FF2A90464FEAA1
:103BD000410705F5467540F08680002B00F0838094
:103BE0009BF85933202B6FD19BF85833012B6BD0A6
:103BF0000122D4F8008019234FF400418BF8582398
:103C00002846CDF80080FEF73BF800285CD10E9BDB
:103C1000CBF84C03CBF83C3322238BF859331023D9
:103C20008BF85A33CBF85C03ABF84293BBF84233C2
:103C30009BB2FF2B00F21781BBF84233DBF818135D
:103C40009BB2A3484A68ABF84033DBB2024047EA74
:103C5000034313439F4A1A434A604FF0580909FB34
:103C60000649B9F842339BB2002B00F08A81D9F89B
:103C700018339A69520700F1378142460A212846D3
:103C8000FDF77CFF002840F0FB80D9F818339A69D3
:103C9000910640F100819A699A6912F0100200F0D1
:103CA000F880102220218C4DDA610422C9F85C23AF
:103CB000D9615A682A405A6089F8591389F858031B
:103CC00089F85A0322689B69B4F81C3430460133E2
:103CD0009BB2A4F81C34FFF791FB4FF0000A50464A
:103CE00005B0BDE8F08F4FF0580B0BFB064B9BF86F
:103CF0005933202BE8D10E9B002B00F0AC80B9F19A
:103D0000000F00F0A8809BF85833012BDCD023680B
:103D100001224FF4004128468BF858230393009367
:103D20001923FDF7ADFF0028CED12223DBF81813AD
:103D30000E9A8BF859334023CBF83C238BF85A3337
:103D4000CBF85C03ABF84293DFF884914A68CBF878
:103D50004C03284602EA09023A4342F490324A6090
:103D6000039974F045FD0246002840F03681402357
:103D700028461946DBF81833C3F82880039B0093C4
:103D80000A23FDF77DFF002840F02781BBF842336E
:103D90009BB2FF2B40F22881DBF81813FF234F4A18
:103DA000ABF840334B6803EA09033B431A434A60CC
:103DB0004FF05808B946039F08FB064805E0B8F8DD
:103DC00042339BB2002B00F021810A230022042100
:103DD00028460097FDF754FF00287FF475AFD8F808
:103DE0001833596AD8F83C331970B8F84213D8F828
:103DF0003C330139013389B2C8F83C33B8F8403359
:103E0000A8F84213013BB8F842139BB289B2A8F854
:103E100040330029D3D0002BD1D102460A23802180
:103E200028460097FDF72CFFFF2200287FF44CAFB7
:103E3000B8F842339BB2934240F2BD80D8F81813D1
:103E4000A8F840234B68264A1340264A43EA090350
:103E50001A434A60B3E758234FF4007203FB06434A
:103E6000C3F85C2330E7DBF81813FF231848ABF8DE
:103E700040334B68194A03403B431A434A60ECE61F
:103E8000582303FB0643D3F818339A6922689B69C9
:103E90001AE7C9F85C232268A2EB08020A2A7FF617
:103EA000E8AE9A6912F004027FF4E3AE582101FBF8
:103EB0000641D1F85C0381F85823202240F020000D
:103EC000C1F85C0381F859239B69FDE6802C00242E
:103ED000009800FC0024000200E800FE0024FF011E
:103EE000009C00FC0000FF015A6AD9F83C331A70AC
:103EF000B9F84233D9F83C23013B01329BB2C9F8EF
:103F00003C23A9F84233B9F84033B9F84223013BC6
:103F100092B29BB2A9F84033002A3FF4A2AE002B24
:103F20007FF49FAE0A23002280212846CDF800802E
:103F3000FDF7A6FE00287FF4C7AEB9F842339BB266
:103F4000FF2B0CD9D9F81813FF233B48A9F84033AD
:103F50004B683A4A03403B431A434A6081E6B9F84A
:103F60004233D9F818139BB233484A68A9F8403352
:103F7000DBB2024047EA0343134343F000734B6054
:103F80006FE64146284674F005FC00287FF49CAE9D
:103F9000D9F8183320212A4DD9615A682A405A602D
:103FA00089F8591389F85A035822002302FB064462
:103FB00084F8583393E6B8F84233D8F818239BB204
:103FC0001D485168A8F84033DBB2014049EA034379
:103FD0000B4343F000735360F1E65823002203FBC8
:103FE000064383F858236FE6BBF84233DBF8181317
:103FF0009BB24A68ABF84033DBB202EA090247EAF7
:10400000034313430F4A1A434A60D1E603992846F3
:1040100074F0C0FB034600287FF456AED8F818238E
:104020002020074DD06151682940516088F859031C
:1040300088F85A33B8E700BF009C00FC0000FF017D
:1040400000E800FE002400020348D0F8B8300BB1AD
:10405000AC301847704700BF000000240348D0F878
:10406000D8300BB1CC301847704700BF0000002497
:104070000348D0F8F8300BB1EC301847704700BF58
:10408000000000240348D0F8183113B100F5867001
:1040900018477047000000240348D0F8383113B1A6
:1040A00000F5967018477047000000240348D0F8C8
:1040B000583113B100F5A67018477047000000246E
:1040C0000348D0F8783113B100F5B670184770473F
:1040D000000000240348D0F8983113B100F5C670F1
:1040E00018477047000000240348D0F8B83113B1D6
:1040F00000F5D67018477047000000240348D0F838
:10410000D83113B100F5E67018477047000000245D
:104110000348D0F8F83113B100F5F670184770472E
:10412000000000240348D0F8183213B100F50370E2
:1041300018477047000000240348D0F8383213B104
:1041400000F50B7018477047000000240348D0F8B2
:10415000583213B100F5137018477047000000245F
:104160000348D0F8783213B100F51B701847704738
:10417000000000240348D0F8983213B100F52370F2
:10418000184770470000002410B41C46436884465A
:104190006FF30F0323434360036843F0010303609D
:1041A000036843F400730360002C3AD040F2E93016
:1041B000DCF814309B0748D5002A49D012F8013B9F
:1041C00040F2E9308CF82030DCF81430DB0720D4E2
:1041D0000138F9D1214B9C450CD0A3F578439C457F
:1041E00038D003F580639C4536D003F578439C4571
:1041F0000BD103201A4A00EB400002EBC002B2F8D8
:10420000C03201339BB2A2F8C03200205DF8044BEB
:1042100070479CF83000C0B209B101F8010B013CB5
:10422000C4D1DCF814301B07FBD5DCF818300120B2
:104230005DF8044B43F01003CCF81830DCF8003084
:1042400023F00103CCF8003070470138B0D1C1E74A
:10425000FF23B5E70120CDE70220CBE70030014086
:10426000000000242DE9F84300242C4E804603680A
:1042700056F83450AB4209D001340E2CF8D1284AFC
:104280000021052009F088F9002019E0254B03EBF7
:104290008409D9F82074AFB198F8051000204B1CA0
:1042A00001EB410203EB430307EBC202DB00C2F860
:1042B0000C80C2E90400F854182303FB0170083095
:1042C000BDE8F8830721682009F0EEF90146C9F836
:1042D0002004F0B13946682282F0E0FFD9F82014BA
:1042E00006EBC4043B4689600C600962896309657A
:1042F00056F83320954205D001330E2BF8D14F608C
:104300000F46C9E7084F4C2202FB03774F600F4668
:10431000C2E7064A052009F03FF9B5E748780C08DE
:10432000B8220D08802C0024D8300024E0220D088B
:10433000F0B54468A37913F002025FD002224FF077
:10434000080C036864795B689B48204493F83C4000
:10435000012C90F8C80050D0012483F83C40142868
:1043600048D8DFE810F015004700470047008400F8
:104370004700470047003B01470047004700BB009C
:10438000470047004700F2004700470047004D0044
:1043900018688A4C056A8A4E25F00205B04242EA46
:1043A0000502056A25F0010505624768856904EA8A
:1043B000050444F0600407D0824DA84204D005F5FE
:1043C0007055A84240F04D8122F0080247F4407732
:1043D0004CEA020222F004024760846141630262F7
:1043E000826942F008028261826922F004028261DD
:1043F00082698261002283F83C20F0BD9446A0E7E8
:1044000018686F4E046AB04224F4001444EA025261
:10441000046A24F4801404626B4C4568476D04EA16
:10442000070444F4C0440ED006F58066B0420AD0BA
:10443000664F06F58046B04218BFB84203D006F575
:104440008066B04201D145F4802545604465C16570
:104450000262426D42F400624265426D22F4806263
:104460004265426D4265002283F83C20C5E718682A
:10447000574C056A524E25F02005B04245EA021518
:10448000026A22F0100202624768826904EA0204AA
:1044900044F4C04400F0DE804A4A904200F0DA80E2
:1044A0004A4E4C4A904218BFB04203D002F5806297
:1044B000904201D147F4406747608461816305629F
:1044C000826942F400628261826922F480628261C0
:1044D00082698261002283F83C208EE71868384E9A
:1044E000046AB04224F4005444EA0232046A24F418
:1044F00080540462364C4568C76904EA070444F4F2
:10450000C0440ED006F58066B0420AD02F4F06F5A3
:104510008046B04218BFB84203D006F58066B0426C
:1045200001D145F480454560C46101640262C269FD
:1045300042F40062C261C26922F48062C261C2694F
:10454000C261002283F83C2057E718681C4E046AB9
:10455000B04224F4003444EA0242046A24F4803471
:1045600004621D4C4568476D04EA070444F060048A
:104570000ED006F58066B0420AD0144F06F580468C
:10458000B04218BFB84203D006F58066B04201D1F0
:1045900045F480354560446581650262426D42F0B4
:1045A00008024265426D22F004024265426D426596
:1045B000002283F83C2020E7F0770C088CFFFEFFF8
:1045C0000000014000040140FF8FFFFE0040014059
:1045D000FF8CFFFE004401408FFFFEFF1868264C51
:1045E000056A264E25F4007EB0424EEA0225026A94
:1045F00022F4807202624768C26904EA020444F04D
:10460000600420D01E4A90421DD01E4E1E4A904289
:1046100018BFB04203D002F58062904201D147F446
:1046200040574760C461C1630562C26942F0080235
:10463000C261C26922F00402C261C269C261002281
:1046400083F83C20D9E625F4006E4EEA0C2E2EF4B9
:104650008065E4E725F0800545EA0C1525F0400566
:1046600028E705F58065A8423FF4AEAE05F5806504
:10467000A8427FF4B1AEA7E68CFFFEFF0000014028
:104680000004014000400140004401404268537969
:10469000032B0FD8DFE803F00B0805021068403049
:1046A000704710683C3070471068383070471068A9
:1046B0003430704700207047D0E90002064B517932
:1046C00092790B44406893F8C810530701D57CF0E9
:1046D000B9B87CF033B900BFF0770C084268C36802
:1046E00012695B68C2F30322F0B53B4D05EB820211
:1046F0009668EFF31182102484F312884468374FD0
:1047000094F805C0D0F80CE035F81CC025680CF40E
:10471000F05CEC6824EA0C0417F806C0EC60DEF8E4
:10472000105053F80C401F2D24F0010443F80C40A6
:1047300042D9203D2024DEF804C0AC40CCF80C4027
:10474000D2B282F3118817F806C042F2107203EB5E
:104750000C0EDEF80040E40702D500BF013AF8D1A4
:1047600053F80C2012F0010223D1DEF80440456911
:104770006FF30F0421434468CEF8041061790329D4
:1047800005D8DFE801F02326022022683C32CEF86B
:104790000C500121CEF8082053F80C2042F01002F2
:1047A00043F80C2053F80C200A4343F80C20017402
:1047B000F0BD00230374F0BD2024DEF804C0AC403B
:1047C000CCF80840BCE722684032E0E72268343287
:1047D000DDE722683832DAE7F0770C0860790C08F8
:1047E00003681A7E012A2ED0002293F83010012986
:1047F00009D093F8481001290ED093F860100129D0
:104800001BD02ABB7047022142F4806283F830102B
:1048100093F84810012904D1022142F4006283F880
:10482000481093F86010012907D01B6800211B680D
:104830005962D9680A43DA607047022142F4805213
:1048400083F86010F1E702214FF400721976CCE78B
:104850004FF40072E9E700BF08B5204B98420ED034
:1048600003F5806398420AD01D4A03F580439842BD
:1048700018BF904203D003F5806398421BD1FDF727
:1048800063FA1849184BCA69C969C2F30222C1F315
:1048900002211A4492F8302002F01F02D040114A3F
:1048A0001269C2F3C03241EAC202134493F8CC3019
:1048B00003FB00F008BDFDF747FA0A490A4BCA6935
:1048C000C969C2F3021CC1F3021103EB0C0292F896
:1048D000302002F01F02D040E1E700BF000001409D
:1048E0000040014000440258F0770C0870B50E46B5
:1048F00005EE102AD0E90031013E1A680868B6B208
:104900005C681568FFF7A8FF07EE900AB8EE455AF5
:104910009FED5D7AF8EE677A87EE850A30EE070A3A
:1049200080F012FB23680138AB4280B268D0C4E942
:10493000005000238022E660A360A261C4E9043332
:1049400094F83D3003F0FF02002B78D00223211DA4
:10495000284684F83D30FDF7DFFE4C4A0123B5F1CF
:10496000804FA5EB020284F84830B2FA82F284F854
:104970003E3084F83F304FEA521284F8403084F8D9
:10498000413084F8423084F8433084F8443084F86D
:10499000453084F8463084F8473084F83D3034D0D0
:1049A0009ABB3B4B9D420CD003F580639D4208D0DF
:1049B00003F580639D4245D003F578439D4241D085
:1049C00070BD94F83C30012BFAD00222314B01210A
:1049D00084F83D20A8680340AB6084F83D1084F85B
:1049E0003D206B68A96823F0700321F0800101224B
:1049F0006B600023A96084F83D2084F83C3070BDD2
:104A0000636883423AD0606093E794F83C30012BAE
:104A1000D6D002211F4B002084F83D10A9680B401E
:104A20000121AB6084F83D10022384F83D306B68AF
:104A3000A9680AB90028D6D023F47003D3E784F814
:104A40003C2083E794F83C30012BB9D00221114B74
:104A5000114884F83D10A968281A0B40B0FA80F07C
:104A60000121AB600023400984F83D1084F83C30FC
:104A70000A4B9D42D8D00028D6D170BDE368B3421E
:104A80007FF457AF70BD00BF0AD7233C0000014040
:104A9000000400408800CEFF00040140000C0040EC
:104AA000024B0348D3F82014FCF7C4BC802C00242C
:104AB00000000140034B4FF08040D3F82414FCF772
:104AC000B9BC00BF802C0024024B0348D3F8281443
:104AD000FCF7B0BC802C002400040040024B0348CB
:104AE000D3F82C14FCF7A6BC802C0024000800404E
:104AF000024B0348D3F83014FCF79CBC802C0024F4
:104B0000000C0040024B0348D3F83C14FCF792BC65
:104B1000802C002400040140024B0348D3F84C14BD
:104B2000FCF788BC802C002400180040024B03488E
:104B3000D3F85814FCF77EBC802C002400400140C0
:104B4000024B0348D3F85C14FCF774BC802C00249F
:104B500000440140024B0348D3F86014FCF76ABCE0
:104B6000802C00240048014010B5064C0648D4F8BB
:104B70003C14FCF75FFCD4F850140448BDE8104026
:104B8000FCF758BC802C002400040140001C0040AD
:104B900010B5064C0648D4F83C14FCF74BFCD4F88E
:104BA00054140448BDE81040FCF744BC802C002499
:104BB0000004014000200040BFF34F8F0549064B21
:104BC000CA6802F4E0621343CB60BFF34F8F00BFAB
:104BD000FDE700BF00ED00E00400FA050021012020
:104BE00008B50EF091FA72B6FFF7E6FF2DE9F04333
:104BF000BFB0BFF35F8FA14C0023626A22F4803202
:104C00006262C4F894309DF843109DF844C00906D0
:104C10009DF842200F9841EA0C7141EAC2419DF88B
:104C2000452041EA82419DF8462041EA42419DF8F3
:104C3000472041EA02419DF8412041EA02219DF8C6
:104C4000402041EA4201C4F898300133D4F8A02052
:104C5000112B22F00102C4F8A020C4F89C00C4F873
:104C6000A010F0D10523C4F89430636A43F4803374
:104C70006362BFF34F8FBFF36F8F8148814A8249D0
:104C8000121A82F0EDF9814B5A6D012A00F0DF8093
:104C9000D4F8881000227E4B012041F47001C4F842
:104CA000881018601A61196841F08001196019684C
:104CB00001431960196841F480311960196841F4A1
:104CC000805119609A61DA611A629A62DA621A6333
:104CD0005A639A63DA631A645A64196821F480216A
:104CE00019601A664FF000636A49C1F80801A360B1
:104CF0007CF03CFF684AD36813F0040FD36840F09F
:104D00009480664B0021644A0591D96A21F0010123
:104D1000D962DB6A03F001030593936943F44043CE
:104D20009361936903F440430593059B93699E0443
:104D3000FCD54C2200210EA8594C82F0AFFA594AFA
:104D400042F20303A4F110011268B3EB124F4FF0CB
:104D500000024FF00C0308BF0C460892E268A370F3
:104D6000002A4FD04D4BD96A21F00101D962DB6A8C
:104D7000494903F0010308938B6923F4404313432B
:104D80008B618B6903F440430893089B424A936903
:104D90009D04FCD53E4B4FF4403543480321D3F8E6
:104DA000E02042F08002C3F8E0200122D3F8E03096
:104DB00003F080030793079B85610D9BCDE90013EA
:104DC00000237CF081FD022301204FF48031A28872
:104DD000CDE917330C231993A379CDE90E01E079BE
:104DE000217A1C900EA81D91CDE91A2304220023DC
:104DF000CDE91E23FBF736FD032800F06082002872
:104E000058D0FEE7244A254B916941F44041916115
:104E1000926902F440420892DA6A42F00102DA62D0
:104E2000DB6A03F001030893AFE723F007031F4C8D
:104E300043F00203D360216805E023685B1AB3F5F1
:104E40007A7F3FF65EAF53689F04F6D559E7104A64
:104E5000002017495865D2F8F43043F00203C2F835
:104E6000F430D2F8F43003F002030E930E9B0B687B
:104E700083F308884B689847FEE700BF00ED00E029
:104E80000000000018390000F4A00D080040005890
:104E900000440258008000510048025800040058A5
:104EA0001C0300240010005C001C0258802C00240D
:104EB0000098F01F754B1A6812F00E0F0BD11A688C
:104EC00022F00F0242F002021A601B6803F00F0387
:104ED000022B40F0F6816E4A936903F070033F2B7A
:104EE00005D8936923F0700343F040039361684A47
:104EF000D36903F070033F2B05D8D36923F0700307
:104F000043F04003D361624AD36903F4E063B3F52D
:104F1000806F05D2D36923F4E06343F48063D361E7
:104F20005B4A136A03F070033F2B05D8136A23F022
:104F3000700343F040031362554B9A69140705D47C
:104F40009A6922F00F0242F008029A61504A93696E
:104F500023F4706393611368980130D5136941F2AB
:104F600088314C4C23F0070343F00303136120689E
:104F700004E023681B1A8B4200F2AC81136903F032
:104F80003803182BF5D1936903F00F03082B05D9CB
:104F9000936923F00F0343F0080393613B4A1368BE
:104FA00003F00F03022B0BD9136823F00F0343F018
:104FB00002031360136803F00F03022B00D0FEE717
:104FC000334A936903F07003402B05D9936923F0AA
:104FD000700343F0400393612D4AD36903F07003DB
:104FE000402B05D9D36923F0700343F04003D3610C
:104FF000274AD36903F4E063B3F5806F05D9D36919
:1050000023F4E06343F48063D361214A136A03F01D
:105010007003402B00F256811D4EFCF773FE1E4DAF
:10502000B269B369C2F303221C4B134493F83030C6
:1050300003F01F0320FA03F3D5F884002B60FCF77C
:10504000EFFC002840F08D811023159017900EA8DA
:105050000E93FBF707FC002840F030813368104ABC
:1050600043F080033360D6F8F43043F00203C6F80F
:10507000F430D6F8F43003F002030493049B136A6F
:1050800043F001031362074B216810E00020005237
:1050900000440258802C002400000024F0770C0803
:1050A0000004005880380100013B00F008812268AC
:1050B0009142F9D0226823689B1A0A2BFBD9002160
:1050C0004FF48020A74C4FF4401300260027309364
:1050D0004FF00208CDE90E010EA87BF01BFDD4F8BD
:1050E000EC30A14941F2030243F002030EA8C4F8D8
:1050F000EC30D4F8EC3003F002030393039BD4F8B4
:10510000943043F00203C4F89430D4F8943023F080
:105110000203C4F894300B689449B2EB134F944BDC
:10512000944A28BF0A465A601A6822F47C5242F414
:1051300000521A601A6842F060021A6003220023CB
:10514000CDE92C67CDE90E237BF0E4FC4FF4E0427F
:1051500000230EA8CDE9266700270326CDE90E23FC
:105160003A977BF0D7FC182200230EA82F9734978C
:10517000CDE90E237BF0CEFC4FF4803200230EA845
:105180001797CDE90E2305224FF4FA73CDE91023CA
:10519000042314934FF48033CDE915772293CDE99E
:1051A00012867BF0B7FCD4F8E03042464FF48071B1
:1051B00043F001037048C4F8E030D4F8E03003F065
:1051C00001030993099B3B46CDE900677CF07CFB1A
:1051D00023694246694823F0FE7343F088732361D4
:1051E000D4F8E03043F00403C4F8E030D4F8E03001
:1051F00003F0040306933B4606994FF40071CDE992
:1052000000677CF061FB236923F07E4343F0FC439D
:105210002361FCF777FD2860BFF35F8F584C3E4653
:10522000584D4FF00108636A23F480336362C4F879
:10523000947028E0002A4CD02F686B7A103515F84E
:10524000061C1B0643EA017343EA420315F8052CCA
:1052500043EA824315F8042C43EA424315F8032C31
:10526000C4F89860013643EA0243D4F8A020032E24
:1052700043F0010322F00102C4F8A020C4F89C709E
:10528000C4F8A03027D06B682A7A002BD2D02F68C0
:10529000002AD2D127F01F02A3EB0209B9F1200F97
:1052A00038BF4FF02009484681F062FE421E08FADE
:1052B00002F1894508BF0246D2B2BEE7FEE7FFF71A
:1052C0008DFC7CE6136A23F0700343F04003136205
:1052D000A2E6FEE773E60523C4F89430636A43F45C
:1052E00080336362BFF34F8FBFF36F8FBFF34F8F76
:1052F000BFF36F8F0022C4F85022BFF34F8FBFF36C
:105300006F8F636943F400336361BFF34F8FBFF363
:105310006F8FC4F88420BFF34F8FD4F8805043F6CA
:10532000E0761749C5F34E34C5F3C905640104EAB4
:1053300006002B4640EA8372013BC1F86022F9D295
:10534000203C14F1200FF2D1BFF34F8F4B6943F48F
:1053500080334B61BFF34F8FBFF36F8F3FB0BDE81A
:10536000F0832CE6004402580010005C7FBB220052
:10537000008400407FBB2230000002580008025821
:1053800000ED00E02C0300242DE9F843374E984649
:1053900006EB8003D3F8DC40002C65D004F1D20387
:1053A000FC360546B4F8D202A36104F5E9736660E1
:1053B0001746E3614FF48073261DE160C4E90433AE
:1053C0002368C4F8CC30A36300284AD194F8D100F4
:1053D0000DF0C8FB18F0080F94F8D09034D1BA073C
:1053E00023D4FB0711D4052194F8D60273F082FA76
:1053F00094F8D63201221E4903F01F005B09824057
:1054000041F823203046BDE8F883013548460DF0C9
:10541000A9FBEDB218B140F206630572C38094F89F
:10542000D42202210DF07CFBDDE76B1CDBB218B14E
:10543000037240F20653C38094F8D52202210DF086
:105440006FFBFB07CFD5E0E70135EDB218B140F2B5
:1054500006730572C38094F8D52202210DF060FB1B
:10546000C1E772F07FFDB1E72646CBE7F0770C0885
:1054700000E100E00148FDF7FBB900BF6003002434
:105480000148FDF7F5B900BF380600240148FDF7D3
:10549000EFB900BF100900240148FDF7E9B900BFCA
:1054A000E80B00240148FDF7E3B900BFC00E00245B
:1054B0000148FDF7DDB900BF981100240148FDF750
:1054C000D7B900BF70140024F8B52422456B00231F
:1054D0008168C0F8BC2004462A6800F13407C66D14
:1054E00022F001022A602B606B60AB6090F806E04E
:1054F000C0F8C43080F8B830C0F8BC30C364C0F81D
:10550000C0304365C0F8A030C0F8A4304FEA8E2305
:10551000816303F48053C3634FEA0E3303F40053F3
:1055200003644FEA0E2303F4806343644379D8078E
:1055300003F0020253D4002A6FD1A264574B03F147
:10554000200C53F8042F22B11068D4F8C8108842F8
:105550006FD09C45F5D11EF0080FD4F8BC3077D041
:10556000002B00F097802423C4F8BC302B6823F074
:1055700001032B60002E40F089803846FCF756FD71
:10558000012812D06B68384623F490436B60AB68F7
:1055900023F02203AB60AB6843F00803AB602B68D9
:1055A00043F001032B607BF0EDF86279D1070DD554
:1055B000D4F8C830196841F480711960996841F0D5
:1055C00001019960196841F020011960930705D520
:1055D000D4F8C820136843F080031360F8BD042397
:1055E000A36482B10C231EF0010FA364A6D04FF474
:1055F000803346F00206636646F001064FF400333E
:10560000E66523669AE71EF0010F97D046F0020682
:105610004FF48033E665636690E708231EF0010FC0
:10562000A3648BD046F001064FF40033E665236691
:1056300084E792F8D732002B8DD04FF4004346F028
:1056400008061EF0080FE366E665D4F8BC3087D183
:10565000CBB12423C4F8BC302B6823F001032B60AA
:105660006EB93846FCF7E2FC01289ED06B683846DC
:1056700023F490436B60AB6823F02A038EE738462F
:10568000FBF724FCEDE784F8B830E2E73846FBF797
:105690001DFC72E784F8B83065E700BFC8780C08D5
:1056A000816011E741710FE781710DE72DE9F84342
:1056B000434D3C20434C05F59872B5F83631C4F89B
:1056C0008028A4F88C38B5F83A21B5F83E31A4F812
:1056D0008E28A4F884380DF045FA074642200DF0D4
:1056E00041FA064638200DF03DFA81461FB10D23E0
:1056F000FB8000233B721EB10D23F3800023337225
:10570000B9F1000F05D00D23A9F80630002389F860
:105710000830B5F842313920A4F88638B5F846315A
:10572000A4F88838B5F84A31A4F88A380DF01AFA86
:1057300080463A200DF016FA05463B200DF012FA8D
:105740000446B8F1000F05D00D23A8F80630002359
:1057500088F808301DB10D23EB8000232B721CB19B
:105760000D23E3800023237248460DF0ABF901219D
:1057700048460DF0B3F940460DF0A4F928460DF067
:10578000A1F920460DF09EF9404601210DF0A6F941
:10579000284601210DF0A2F9012120460DF09EF9C5
:1057A00038460DF08FF930460DF08CF9384601215E
:1057B0000DF094F930460121BDE8F8430DF08EB9A3
:1057C000F0770C08802C002438B5134D41F20D13EE
:1057D000124941F28832D5F8D408D5F8904800042F
:1057E000A060E068014020460B430D21E360FDF717
:1057F00075FB38B1D5F8C428034600201343C5F81B
:10580000C43838BD606900F4F050A0F50060B0FA0B
:1058100080F0400938BD00BF802C0024C0E0FEFFAE
:105820002DE9F04FA64D7C2200219BB005F50963C0
:10583000184681F033FD4FF400310346D5F8804817
:105840004FF48030226819610221C5F8940859612B
:1058500095F8C038C5F89028002B00F08880042205
:10586000984B85F8C028DA6C1B68D6030DD5180153
:1058700000F1D98001224FF0006385F8C028C5F8F7
:10588000C43801201BB0BDE8F08F9C01F2D50AABF3
:1058900018460193FCF7CAFD0B990029EAD0D5F808
:1058A00090480A0A884B6668A3FB0232874B884FF0
:1058B00033401009B94243EA12136360236843F08E
:1058C0000303236040F2F6804300824AB1FBF3F306
:1058D000B2FBF3F2296802322B685B1A9A42FBD8BA
:1058E00000237D4A0493A3607C4BE16817680B405A
:1058F00043F48053E3607A4BA3FB073741F28833CC
:105900007F0A03FB07F73B46002B00F0C880626B61
:10591000013B1106F8D5734B704AA3634FF4D5735E
:10592000A360E3681A4041F208131343E3604FB1E8
:105930003B46626B12F0450F02D0920440F1DA80D0
:10594000013BF6D10023C5F8CC38A360634BE26875
:10595000134043F48053E3603B46002B00F09F80EC
:10596000626B013B1106F8D55E4BA363E1E05E4B31
:105970009A425FD05D4B9A4200F00D8195F88C08F9
:105980000DF0F0F8834695F88E080DF0EBF882469E
:1059900095F884080DF0E6F8814695F886080DF034
:1059A000E1F8804695F888080DF0DCF8074695F890
:1059B0008A080DF0D7F895F88D2806460E2158462E
:1059C0000DF0AEF8504695F88F280E210DF0A8F88E
:1059D000484695F885280E210DF0A2F8404695F826
:1059E00087280E210DF09CF895F8892838460E215D
:1059F0000DF096F80E2195F88B2830460DF090F8B2
:105A00000221B4F9040072F075FFB4F90430002BE0
:105A1000FFF625AF03F01F0001225B0934498240E5
:105A200041F823201BE70AAB18460193FCF7CAF99B
:105A30000C9932E7234BD3F8D42022F48032C3F8F8
:105A4000D420D3F8D4200243C3F8D420D3F8D420F0
:105A500002400392039ADA6F0243DA67DA6F22F4A4
:105A60008032DA678AE72A684FEA134EA2EB09020E
:105A70007346824213D8002B40F03281C4F808E00C
:105A8000E36803EA0A030B43E3603B46626B12F0F0
:105A9000450F02D0920440F1F180013BF6D14FF066
:105AA0000040012385F8C038D5F8C4380343C5F851
:105AB000C438E6E6074AB2FBF1F229680BE700BFFB
:105AC000802C002400440258598B4F01002CC0FF49
:105AD000FF340C001021010000000024C0E0FEFF94
:105AE000D34D6210C500200000700052002402480F
:105AF00000E100E0636B5B0700F16F83636BDE071F
:105B000069D4636B580601D54023A3630123704A0F
:105B100037212046C5F8CC380023A360E3681A403B
:105B200041F23713134341F28832E360FDF7D6F9AF
:105B300070BB049A4FF6FE739A4200F23982DFF886
:105B400090A1DFF89881634E002241F2371337218C
:105B50002046A260E26802EA0A02134341F2883258
:105B6000E360FDF7BBF900289BD1C4F8088041F23F
:105B70002913E26802EA0A021343E36047B13B4695
:105B8000626B12F0450F01D0920427D5013BF7D18B
:105B90004FF0805085E7504BD3F8DC2022F40072A0
:105BA000C3F8DC20D3F8DC2042F40072C3F8DC2018
:105BB000D3F8DC2002F400720292029AD3F8842017
:105BC00042F40072C3F88420D3F8842022F40072D7
:105BD000C3F88420D2E60123A36397E7636B5B07D6
:105BE00058D4A6636269049B002A03F1010304935D
:105BF000049B03DB4FF6FE718B42A5D904994FF647
:105C0000FE73994200F21782500040F1D4814FF0A8
:105C10000108D5F80090C5F8C8882368990700F0F6
:105C2000C4810023DFF8A8A02046A36041F202331C
:105C3000E26802EA0A021343E360FBF7A5F90028D1
:105C40007FF42FAF636941F20311C5F8FC38A369F3
:105C5000C5F80039E369C5F80439236AC5F808397D
:105C6000A060E36803EA0A030B43E360002F3FF4FC
:105C700016AFDFF860C041F2873006E7636B5B0761
:105C800022D4636BDE071CD42369DBB2032B06D05E
:105C9000012006E704234FF08050A36301E7C4F816
:105CA00038C0636913F4604F3FF4DDAE590400F16E
:105CB0009D8213F4004F0CBF4FF480304FF480509E
:105CC000EFE60123A363E3E704231846A363E8E6B2
:105CD000C0E0FEFFC500200000440258000010C1D3
:105CE0004FEA0E49C5F8D4E8D44A2046C4F80890D3
:105CF000E3681A4041F209331343E360FBF744F9C8
:105D000000287FF4CEAE6269C5F8EC28A369C5F817
:105D1000F038E769C5F8F478216AC5F8F818D4F8BE
:105D200018C04FEA1C5CC5F8D0C84FEA927C8DF8C9
:105D300028C0C2F3836C8DF829C0C2F3016C8DF8C2
:105D40002AC0C2F3074C8DF82BC0C2F3072CD2B285
:105D50008DF82CC08DF82D201A0DADF82E20C3F330
:105D600003428DF83020C3F3C0328DF83120C3F3E5
:105D700080328DF83220C3F340328DF83320C3F3E4
:105D800000328DF834208DF83500B8F1000F00F0A6
:105D90001F811B0403F47C1343EA17430E934FF453
:105DA0000073C5F8DC380E9B01339B02C5F8D83868
:105DB000C5F8E038C7F380334FF4007A20468DF8F9
:105DC0004130C7F3C61307F07F07C5F8E4A88DF884
:105DD0004230CB0F8DF8437001278DF84430C1F36A
:105DE00041738DF84530C1F382638DF84630C1F3BD
:105DF00083538DF84730C1F340538DF8483000236A
:105E00008DF84930C1F300438DF84A30C1F3C033F7
:105E10008DF84B30C1F380338DF84C30C1F34033F3
:105E20008DF84D30C1F300338DF84E30C1F381232E
:105E30008DF84F30C1F30123C1F346018DF8503086
:105E400041F207138DF8511007218DF85270C4F8F4
:105E50000890DFF8E891E26802EA0902134341F290
:105E60008832E360FDF73AF800287FF41AAEC4F8F0
:105E700008A041F2101BE36841F28832102120464D
:105E800003EA090343EA0B03E360FDF727F8002860
:105E900040F0948095F8C038032B3FF4F2AC2F68A3
:105EA00063699A017ED44FF0400A41F28832102192
:105EB0002046C4F808A0E36803EA090343EA0B0399
:105EC000E360FDF70BF8002843D1D5F8D43837212B
:105ED00020461B04A36041F23713E26802EA09027C
:105EE000134341F28832E360FCF7F8FF88BB4FF0C0
:105EF000FF330D216362C4F828A0E36A23F0FF0397
:105F000043F06303E36241F20D13A0602046E268B0
:105F100002EA0902134341F28832E360FCF7DEFF34
:105F2000B8B9019E04E02B68DB1B013300F08A80C6
:105F3000636B13F4957F636B40F087801B04F2D58D
:105F400006F12002D4F8803046F8043BB242F9D181
:105F5000E9E7D5F8C438C5F8C438394B0122A36342
:105F6000D5F8C43818434FF40073C5F8C408204668
:105F700085F8C028A36041F21013E1682F4A0A4057
:105F80001021134341F28832E360FCF7A7FF002899
:105F90003FF477AC2A4A0123A263C5F8C40885F808
:105FA000C0386EE44FF40060D7E74FF0806078E5CA
:105FB000049A9A423FD84FF000082AE6204BA36388
:105FC000D5F8C4380343C5F8C43885F8C07858E418
:105FD00040F6FC7202EA830343EA97730E93C7F319
:105FE000C2638DF83C30C7F302638DF83D30C7F3D0
:105FF00042538DF83E30C7F382438DF83F30C7F3EC
:10600000C2338DF8403001230E9A9DF840001A44A7
:1060100000F00700023082409DF8300000F00F00D1
:10602000C5F8D8288340C5F8DC385B0A02FB03F3C7
:10603000C5F8E038BEE64FF0807032E5C0E0FEFF04
:10604000FF0FE01F4FF0004087E7180700F1C880FE
:10605000636B990700F1C880636B9A0608D5C1E0AD
:10606000D4F880202B6846F8042BDB1B0133E9D0E1
:10607000636BDB04F4D40A9B5E4AA263C3F3811210
:106080008DF81420C3F340128DF815201A0A22F05F
:10609000FF0242EA1362DDE90B1392B209BAADF8CE
:1060A0001620DAB206918DF81C20C3F307229DF862
:1060B0003B108DF81D20C3F303521B0C8DF81E20DE
:1060C0000D9A23F0FF03D0B203432046ADF82030F1
:1060D000C2F385238DF82230C2F301238DF82330DB
:1060E000C2F3031302F00F028DF824304FF4007353
:1060F0008DF825208DF826101021A3603E4AE36814
:106100001A4041F21013134341F28832E360FCF766
:10611000E5FE00287FF43EAF9DF82430B8F1010F72
:106120009DF82520DBB2D2B205D1134314BF4FF442
:1061300000784FF48078D5F89C08C5F8E88872F0AC
:106140002BFA00287FF49DAB2C6803E02B681B1B07
:10615000013330D072F0FEF90428F7D10023012179
:10616000D5F8D828C5F8C438C5F8BC3885F8C018A3
:10617000002A3FF486AB4FF4804072F00DFA0028FD
:106180007FF47FABD5F8C838F3B1012B7FF479AB3E
:1061900002201A4C85F80C09A4F124030FCB84E8E3
:1061A0000F00A4F1140310340FCB84E80F0000207B
:1061B0001BB0BDE8F08F4FF000420123C5F8C428A2
:1061C00085F8C038FFF75DBBD5F8CC38002BE0D0A0
:1061D000012B7FF456AB1846DBE70423A36395E459
:1061E0000820BAE62020B8E60220B6E64FF40050B8
:1061F00057E400BF3A0F0018C0E0FEFF90350024BE
:10620000C74BD3F81019D3F8142970B58C0F93F835
:106210000C59100EC2F3072C83F83849C1F383647C
:106220000001012D83F83949C1F3016483F83A492B
:10623000C1F3074483F83B49C1F30724C9B283F88B
:106240003C49C2F3035483F83D19A3F83E09C2F355
:10625000C030B3F83E1989B241EA0401C2F30344E5
:10626000A3F83E19C2F3403183F84049C2F38034A9
:1062700083F841094FF0000083F8424983F843193D
:10628000C2F3003183F84419D3F8181983F845098B
:1062900040F2EF80022D00F0C3802A204FEA4C0C20
:1062A00083F85149C1F3C01201F07F010CF07E0C5C
:1062B00083F852C94FF0010C93F852491443D3F8B4
:1062C0001C2983F85249D40F83F85319910D83F890
:1062D0005449C2F3417401F00C01C2F3815583F8B3
:1062E0005549C2F3826483F8564983F8571993F8E5
:1062F0005719D3F82049294383F85719C2F340515D
:1063000083F85819002183F85919C2F3004183F822
:106310005A19C2F3C03183F85B19C2F3803183F894
:106320005C19C2F3403183F85D19C2F3003183F880
:106330005E19C2F3812183F85F19C2F30121C2F310
:10634000460283F86019C4F3074183F86129220EDD
:10635000090283F862C983F86429C4F30722A3F809
:1063600066192406B3F8661989B21143A3F86619B1
:10637000D3F82419C3F868490C0ED3F8682942EA07
:106380000442C3F868290A0AD3F8684902F47F4234
:106390002243C1F30724C9B2C3F86829D3F8685966
:1063A000D3F828292C43C3F8684983F86C19110ED7
:1063B00083F86D19110C0906C3F870191102D3F88E
:1063C00070490A4601F47F01214392B2D3F82C4967
:1063D000C3F87019D3F870190A43C3F87029C4F3CD
:1063E0000352D3F8701941EA1461C3F8701993F895
:1063F00074191143C4F3072283F87419210A01F4B4
:106400007061A3F87619B3F8761989B21143C4F311
:106410004602A3F8761983F8782983F879C970BD04
:106420001204C1F3072C0D0E02F47C12C3F84829A4
:10643000C1F30742D3F8484944EA0524C3F8484960
:10644000D3F8484922434FF40074C3F84829D3F8DD
:106450004829C3F88849013240F10004A40244EA03
:1064600092549202C3F88449C1F38034C3F880295E
:1064700014E74FEA8C2CC1F3C26594000CF440621F
:10648000C1F3072C04F47F74C3F84829D3F84829D2
:106490001443CA0BC3F8484902F00602D3F848492E
:1064A00044EA9174C3F84849C1F3026483F84C5933
:1064B000012583F84D49C1F3425483F84E49C1F395
:1064C000824483F84F49C1F3C03483F8502993F8CC
:1064D0005029224383F85029D3F8484993F850298A
:1064E00093F84069023205FA02F2B540D617A2FBD2
:1064F000052EC3F8885905FB06EE04FB0EEE0134A9
:10650000A2FB0424A644520AC1F3803442EACE52CC
:10651000C3F880294FEA5E22C3F88429BEE600BF93
:10652000802C002471F072BE71F070BE10B51C207A
:106530000CF018FB044611210CF0D0FA20460CF0A8
:10654000C7FAC8200EF006FB2046BDE810400CF04C
:10655000B9BA00BF1C48D0F80038D0F8082830B5C8
:106560009B184FF01A040C8001D1184830BD174A0F
:106570000024D0F8040802F1100511464FEA137EFA
:10658000B3F1204FCC7001F102010EF1370C38BF8E
:106590000EF1300C8D424FEA031381F800C0EDD1AB
:1065A0000B4D0024010FB0F1204FD47402F1020210
:1065B00001F1370338BF01F1300395424FEA001073
:1065C0001374EFD1014830BD00E0F11F44170024DF
:1065D0004C170024122301480B80704758000024F8
:1065E00000207047212808B524D0222816D0202862
:1065F00012D189B1072A0FD1154A0868154BB1F895
:1066000004C012688979D861A3F820C083F82210E9
:1066100012B1014600209047002008BD0029FBD0A0
:10662000022AF9D10A4A5368002BF5D009889068EC
:106630009847F1E70029EFD0072AEDD1054B00205C
:10664000DA690A601A8C8A8093F822308B7108BD4F
:10665000204600244417002400207047034B93F881
:106660003000003818BF0120704700BF20460024CA
:10667000034B93F83000032894BF0020012070479B
:10668000204600240048704754460024164B002042
:1066900030B493F82A4014B1DD698D4205D0013041
:1066A00010330828F5D130BC7047104BB2B1D96F08
:1066B00001EB40218A4201D1022C08D093F81C2220
:1066C00012B9012283F81C22012283F8652003EB12
:1066D0000013012283F88E2030BC704703EB0013B7
:1066E00083F88E20DFE700BF844600242046002484
:1066F00030B40023194C04F1640084F8083103E03D
:1067000001331030082B1BD0C5698D42F8D190F8A9
:106710002AC0BCF1030FF3D1A2B1E16F01EB432119
:106720008A4208D094F81C2212B9012284F81C2253
:10673000012284F8652004EB0314012384F88E30D1
:1067400030BC7047D4F8042104EB03130421013258
:1067500083F88E10C4F80421F2E700BF204600241D
:10676000C0B1836823B10F4B072283F866207047BE
:106770000C4A042192F8640082F87830032882F8E9
:106780006610C2E91C3314BF4FF480738023C2E942
:106790001A337047034B012283F81C2283F86520CB
:1067A000704700BF20460024244910B5CC8C91F8D6
:1067B00024C0644531D963462431E646624603E08D
:1067C000944238D991F800E07144724491F801E0A4
:1067D00092B2BEF1050FF3D191F802E0BEF1810F44
:1067E000EED1174A03E0A3421BD292F800C06244E4
:1067F000634492F801C09BB2BCF1050FF3D192F84B
:1068000002C0BCF1010FEED119B1002402230C71BA
:106810004B7100210223117153712023038008481A
:1068200010BD0029F9D0022300224B7120230A71E8
:106830000380034810BD0021D3E700BF44170024A4
:1068400068170024244910B5CC8C91F824C0644505
:1068500031D963462431E646624603E0944238D992
:1068600091F800E07144724491F801E092B2BEF1F7
:10687000050FF3D191F802E0BEF1810FEED1174A76
:1068800003E0A3421BD292F800C06244634492F832
:1068900001C09BB2BCF1050FF3D192F802C0BCF16C
:1068A000010FEED119B1002440234C710B7100216E
:1068B00040235171137120230380084810BD002923
:1068C000F9D0402300220B7120234A710380034832
:1068D00010BD0021D3E700BF44170024681700242F
:1068E000244910B5CC8C91F824C0644531D9634655
:1068F0002431E646624603E0944238D991F800E03C
:106900007144724491F801E092B2BEF1050FF3D1E7
:1069100091F802E0BEF1810FEED1174A03E0A342E5
:106920001BD292F800C06244634492F801C09BB24B
:10693000BCF1050FF3D192F802C0BCF1010FEED10A
:1069400019B1002440234C710B7100214023517177
:10695000137120230380084810BD0029F9D040237B
:1069600000220B7120234A710380034810BD0021CF
:10697000D3E700BF441700246817002403460A2207
:1069800001481A80704700BF8817002438B5D0F836
:10699000D432B03350F823507DB195F81C32044600
:1069A00023B9D5F818320BB16B7A8BB1812120460F
:1069B00079F084FC6B7A022B00D038BD204681210F
:1069C00079F07CFC20460121BDE8384079F076BCA6
:1069D000012179F073FC20468121BDE8384079F02F
:1069E0006DBC00BFD0F8D42200EB82022DE9F0414B
:1069F000D2F8C0420646002C4ED0B4F8643204F1FE
:106A00001007D4F870520846D2F8C422394603FB66
:106A100005F5D2F81080B5F5007FD4F86C2228BFB8
:106A20004FF40075B5FBF3F39BB2C04700281BDBA6
:106A30002B463A468121304679F0C6FDB4F86422EF
:106A4000B5FBF2F2D4E99B1311449B1AD4F8382217
:106A5000521BC4E99B13C4F8382213B10020BDE8CF
:106A6000F08103232372F9E7D6F8D432B03356F815
:106A700023208AB192F861320424112003F14801E5
:106A80000133DBB202F8314002EBC101A34288803E
:106A900008BF002382F861324FF0FF30DFE700BF0C
:106AA00038B5084BD3F88C3253B1DB6914460D4628
:106AB00098474FF40073026800202A60238038BD95
:106AC0001B68FFDE2046002408B5064BD3F88C3245
:106AD00023B11B699847013840B208BD4FF0FF3021
:106AE00008BD00BF204600240020704700207047EA
:106AF00008B520B9044871F007FA044808BD0448F5
:106B000071F002FA014808BDFC220D08B0480024CB
:106B100020230D08024808B571F0F6F9014808BDB8
:106B200044230D08B0480024024808B571F0ECF980
:106B3000014808BD4C230D08B0480024024808B5A0
:106B400071F0E2F9014808BD58230D08B04800244F
:106B500008B520B9044871F0D7F9044808BD0448C5
:106B600071F0D2F9014808BD68230D08B04800242F
:106B700088230D08024808B571F0C6F9014808BD20
:106B8000A8230D08B0480024024808B571F0BCF9EC
:106B9000014808BDB4230D08B0480024D0F8D43211
:106BA000B03370B550F823402CB30026124B054685
:106BB00084F83C12C4F8303204F50C7226720D23AE
:106BC000812104F5047479F0FFFCD5F8C8321F2246
:106BD0000121C3F88C62A3F8781203F51E711868BE
:106BE000C3E9A1429A79012A08BFC3F89442BDE8DB
:106BF000704079F0D9BB70BD55534253D0F8D422C0
:106C000000EB82022DE9F041D2F8C0420646002C8A
:106C100067D0B4F8643204F11007D4F87052084613
:106C2000D2F8C422394603FB05F5D2F81480B5F535
:106C3000007FD4F86C2228BF4FF40075B5FBF3F346
:106C40009BB2C047002834DBD4F83802B4F8642281
:106C5000401BB5FBF2F5D4E99B13C4F83802294474
:106C60005B1BC4E99B13FBB1D6F8C80202FB03F31C
:106C700001220021B3F5007FC0F88472A0F87822C9
:106C8000827928BF4FF40073C0F88C1200F51E7192
:106C9000012AC0F8883208BFC0F89472006879F001
:106CA00083FB0020BDE8F08119463046FFF776FFF0
:106CB000F7E7D6F8D432B03356F823208AB192F8E9
:106CC00061320424032003F148010133DBB202F8EE
:106CD000314002EBC101A342888008BF002382F843
:106CE00061324FF0FF30DDE7D0F8D43200EB8303A0
:106CF0002DE9F043D3F8C04283B0002C00F0B780F8
:106D00001646127805460F465A2A5FD85A2A00F2CC
:106D10009B80DFE812F04601990099005A01990022
:106D2000990099009900990099009900990099009B
:106D3000990099009900990099008E019900990095
:106D400099009900990099009900AC01CD01990032
:106D500099003D019900990099009900100299004D
:106D6000360299009900FA0099005E029900990094
:106D700099009900E1019900990099009900990002
:106D8000990099009900990099009900990099003B
:106D9000990099009900990099009900990099002B
:106DA000990099009900990099009900990099001B
:106DB000990099009900990099009900990099000B
:106DC00099009900990099009900F001A82A53D0E0
:106DD000AA2A00F064829E2A36D1D3F8C43208462B
:106DE00004F5197204F51A715B689847014600288A
:106DF00040F0098394F86232022B00F00483D6F845
:106E00000A301ABAE2601BB104F1100080F046FAB1
:106E1000D4F868320022013B190E61F30702190C05
:106E200061F30F22190A61F31742B4F8641263F395
:106E30001F624BBA6383002362612383D6F80A3052
:106E40001BBAE360002014E094F861220526202597
:106E50000221531C4832DBB204F8326004EBC2005A
:106E6000042B858008BF0023617284F861324FF0E3
:106E7000FF3003B0BDE8F08394F80880B8F1000F4C
:106E80007DD194F91C22002A80F2058394F86222B5
:106E9000022A00F08083D3F8C43208469B689847E2
:106EA000002840F0DE82D6F80230D5F8D4121BBAA2
:106EB000B031C4F86C32D6F8062055F8211012BA59
:106EC000C4F870220029D2D01344D1F8680283425A
:106ED00000F24783B4F8643202FB03F3D4F81822BB
:106EE0009A424AD091F861320524202003F14802E9
:106EF0000133DBB201F8324001EBC202042B908077
:106F000008BF002381F86132B1E794F80880B8F136
:106F1000000F34D194F91C22002A80F2BC8294F82C
:106F20006222022A00F03783D3F8C43238469B68C5
:106F30009847002840F09582D6F80220D5F8D41260
:106F400012BAB031C4F86C22B6F8073055F82110E7
:106F50005BBA9BB2C4F87032002988D01A44D1F8C9
:106F60006862B24200F27383B4F8642202FB03F356
:106F7000D4F818229A4240F0E182022323724FF49F
:106F8000007339462846E36003B0BDE8F04329E5C5
:106F9000337900229B1AE26018BF012384F8623221
:106FA00050E7D4F81822002A40F0398294F862128F
:106FB000022900F04683D3F8C43238469B689847CC
:106FC000002840F0D382E0603CE7D4F81832002B70
:106FD00000F025827021002294F8603221740C2187
:106FE000C4F81520E17594F86112C4F81120994293
:106FF000C4F81920C4F81D2084F8212011D004EB16
:10700000C30191F84012A17404EBC3010133B1F83C
:107010004412DBB2A183042B14BF84F8603284F8DD
:1070200060221223E36032799A4298BF1346E360EC
:1070300008E7D4F81822002A00F0F1817278D2070C
:1070400040F1B181B378002B00F0CF81802B40F06C
:10705000E0810821CC4A04F1180304F11000E1603A
:1070600012F8011D03F8011D8342F9D1EAE6D3F8B5
:10707000C4323846DB689847002840F07481327982
:10708000042A134628BF0423E360002A3FF4DAAE43
:10709000013BBD4A04F1100099B201F111030A4409
:1070A000234412F8011903F8011D8342F9D1C9E6FE
:1070B00094F862223379012A03F0030300F06A8115
:1070C000012B00F06C81022B00F06A81032B00F091
:1070D00066810023E360B5E6737813F0020340F0A5
:1070E0009881D4E99B210A44D4F868128A4200F2BC
:1070F000E581E360A6E6D3F8C4323846DB689847FA
:10710000002840F03881337A082B194628BF08211F
:10711000E160002B3FF496AE9C4A01F1100304F1AC
:1071200010000A4454FA83F312F8011D03F8011DFC
:107130009842F9D186E6D3F8C4320DF102023846FE
:1071400001A95B689847002840F06F8194F862328B
:10715000022B00F06A81BDF802200821206152BA9A
:10716000019BA061013B62830C22E174E375190E5F
:10717000E2601A0C1B0A217562750222A375227641
:1071800077E6D3F8C43204F51972384604F51A715B
:107190005B689847002840F0368194F86232022BF1
:1071A00000F03181D4F868320822A082013BE2600D
:1071B000190E1A0C61F30700190A62F30F20B4F8D4
:1071C000642261F3174052BA63F31F60E2822061C8
:1071D00038E694F80890B9F1000F40F00081D4F837
:1071E0001822002A00F08A8194F91C22002AC0F299
:1071F0001582D3F8C43238469B68984780460028E9
:1072000040F0F181D5F8D432384605EB8303D3F84A
:10721000C432DB6898470146002840F08281D6F8E6
:107220000220D5F8D40212BAB030C4F86C22B6F8F5
:10723000073055F820005BBA9BB2C4F870320028C2
:107240003FF415AE1A44D0F86862B24200F2C6812B
:10725000B4F8642202FB03F3D4F81822934240F0FE
:10726000EC80B3F5007F4FF0010004F1100428BF5B
:107270004FF4007304F8080C1A46D5F8C832C3F866
:1072800088229A79C3F88C1203F51E718242C3F8E2
:107290008442A3F8780262D1C3F894425FE0227A74
:1072A000002A40F09C80D4F81812002900F0838155
:1072B00094F91C120029C0F22181D3F8C432384657
:1072C0009B689847D5F8D432002840F05A8105EBE6
:1072D00083033846D3F8C432DB689847002840F06F
:1072E000F280D6F80230D5F8D4121BBAB031C4F807
:1072F0006C32D6F8062055F8211012BAC4F8702264
:1073000000293FF4B4AD1344D1F86802834200F27F
:107310002881B4F8643202FB03F3D4F818229342B4
:107320007FF4E0ADB3F5007F4FF0010104F11000F0
:1073300028BF4FF40073217200241A46D5F8C832D2
:10734000C3F888229A79A3F8781203F51E71012AEE
:10735000C3F88402C3F88C4208BFC3F894021868CB
:1073600079F022F86EE50A4A92F8623063F07F0302
:1073700082F8623083E6064A92F8673063F07F0352
:1073800082F86730BFE600BFA4170024A8170024C6
:1073900044170024022B3CD0012B7FF497AE00232E
:1073A00084F8623295E6D3F8C43207EBC70132792C
:1073B000D86900EB810003790533934228BF134657
:1073C000E360002B3FF43EAD03F11002034422447E
:1073D00013F8011D834202F8011DF9D132E5394647
:1073E000284603B0BDE8F04308E406219A4A04F1B8
:1073F000160304F11000E16012F8011D03F8011DED
:107400008342F9D11EE53A220221284678F080FC19
:107410002DE524220521284678F07AFC27E5202254
:107420000521284678F074FC21E528463A220221FD
:1074300078F06EFC4FF0FF301BE590F861320525C7
:10744000202403F148020133DBB200F8325000EB94
:10745000C202042B948014BF80F8613280F861125C
:1074600005E5D5F8D432B03355F82320002A3FF48F
:10747000FEAC92F8613202243A2003F14801013354
:10748000DBB202F8314002EBC101042B888075D0D9
:1074900082F86132EBE494F861320520202103F197
:1074A00048020133DBB204F8320004EBC202042BC1
:1074B00091807FF4DAAC84F86182D8E4212205213E
:1074C00078F026FCD3E4D5F8D432B03355F8232035
:1074D0008AB192F861320225272003F14801013375
:1074E000DBB202F8315002EBC101042B888008BFE7
:1074F000002382F8613205232372B8E494F86132E4
:107500000525202003F148010133DBB204F8315096
:1075100004EBC101042B88807FF4A7AC84F86122BE
:10752000A5E4D5F8D432B03355F82320002A3FF42F
:107530009EAC92F86132022427209EE791F86132D6
:107540000525202403F148020133DBB201F8325053
:1075500001EBC202042B94807FF4D4AC81F8610269
:1075600085E491F8613205242120BFE43A2202210A
:10757000284678F0CDFB0523237278E482F86182F7
:1075800075E4B03355F82320002AB4D092F8613264
:1075900002253A20A1E794F8613203F14801013352
:1075A000DBB204F8312004EBC1013A22042B8A80BB
:1075B0007FF45BAC7FE794F861320525202003F16E
:1075C00048020133DBB204F8325004EBC202042B50
:1075D00090807FF44AAC84F8611248E490F86132FC
:1075E000052521242DE7D5F8D432B03355F82320D2
:1075F000002A3FF43CAC92F8613202243A2003F1B5
:1076000048010133DBB202F8314002EBC101042B27
:1076100088807FF43DAF82F8619228E494F861326B
:107620000520202103F148020133DBB204F83200C7
:1076300004EBC202042B91807FF417AC84F86192B2
:1076400015E43A2278F064FB052323720FE491F8E5
:1076500061320525212475E79A170024D0F8D43229
:10766000B03350F82330CBB110B51A7A022A07D0C4
:10767000033A012A02D80021FFF790FA002010BD3A
:1076800003F21F2293F81D120446FFF72DFB00287A
:10769000F4DA01212046FFF781FAEFE70020704776
:1076A000D0F8D432B03370B550F8235025B12B7ACE
:1076B000044683B1012B01D0002070BD05F21F22CA
:1076C00095F81D12FFF710FB0028F5DA012120467E
:1076D000FFF764FAF0E7D5E98523C5F83832D0F82A
:1076E000C832C5F83422D3F88C321F2B04D12F4B6B
:1076F000D5F810229A421AD095F861324FF0050C55
:107700002021204603F148020133DBB205F832C0E4
:1077100005EBC202042B91804FF0020208BF002348
:107720006A7285F86132FFF731F9002070BD95F873
:107730001D120129E0D895F81E32013B0F2BDBD832
:1077400005F21F22FFF7D0FA00282B7A22DB013B3B
:10775000022BB1D9EE681EB3D4F8D432B03354F84A
:1077600023100029A8D02046D1F83842D1F8183289
:1077700005F11002A41BB342C1F838424FF00004D7
:1077800028BF334681F83C4204240C72812178F0F2
:107790001BFF91E7052B99D02046FFF7F7F88BE701
:1077A00031462046FFF7FAF986E700BF55534243BA
:1077B0002DE9F8431B4F06460D683C68C4F5805818
:1077C000454517D82A46254417483146C5F30B05C9
:1077D00020447FF045FC154B3D601B6803F6FF73AA
:1077E0005B1BC3F30B03802B16D971F049FC0020FF
:1077F000BDE8F883DFF830900146424609EB04000B
:10780000A4F580547FF02CFC06EB08012544484683
:107810002A467FF025FCDEE7054B012203201A7083
:10782000BDE8F883842C002410360024882C002422
:10783000702F00245A4B00215A4A1B685A48A2FB59
:10784000032330B5DB0C594C83B0013BC4F8A013C3
:10785000C4F8981342F20F7194F8CD23C4F8900342
:10786000C4F89C13C4F89433002A00F093800225D6
:107870004F494D4884F8CD53FAF74EFF01234D4A46
:107880000621372084F8D83384F8CE3384F8CF33F8
:1078900084F8D03384F8D13384F8D23384F8D333E6
:1078A00084F8D43384F8D53384F8D63384F8D733C6
:1078B00084F8CD33D2F8E83043F02003C2F8E83042
:1078C000D2F8E83003F020030193019B71F012F825
:1078D000394B4FF400025A6094F8CD33012B3BD161
:1078E000D4F89023354B3648B2F1804F18BF9A42F6
:1078F00084F8CD53D1680CBF0123002341F001016E
:10790000824208BF43F0010300F58060D1608242EB
:1079100008BF43F0010300F580602A49824208BF96
:1079200043F0010300F57840824208BF43F00103B1
:107930008A4208BF43F0010313B9234B9A4207D18F
:107940009168224B0B40062B06D0B3F5803F03D045
:10795000136843F0010313601D4AD2F8D432B033E8
:1079600052F8233043B11B4800211B4AC3F80802D8
:10797000C3F81012C3F8042200251849184A194BFD
:107980000D606560156025601D7071F079FB2846FB
:1079900003B030BD02F0FF0084F8CC0367E700BFFE
:1079A0000000002483DE1B43001400402046002416
:1079B000B44900240044025800E100E00000014006
:1079C0000004004000180040004001400700010092
:1079D0008C2C0024F4540024FC490024842C002422
:1079E000882C0024702F0024F8B51F4FD7F84027AB
:1079F000B7F84417D7F88C3291614BB39B6998471D
:107A000030B30026D7F88C3213B11B69984790B970
:107A1000B6F57A7F24D00DF06FF8013604460D4696
:107A20000DF06AF8001B61EB0501B0F57A7F71F18A
:107A30000001F5D3E6E7B6F57A7F4FF0FF3018BFC7
:107A40000020B7F84437D7F840271B049361F8BDEE
:107A5000064B03F16C02DB6EC7F88C229847D0E727
:107A60004FF0FF30EDE700BF20460024441700240C
:107A70002DE9F84F344E90469A46B6F85027D6F87E
:107A80004C471304A361BAF1000F50D0C8EBC853A0
:107A9000C24406F5FC6901EB432B41F28937D6F865
:107AA0008C225AB100235468494640461A46A047E2
:107AB000A8B9D6F88C320BB11B699847013F3AD070
:107AC0000DF01AF804460D460DF016F8001B61EB98
:107AD0000501B0F57A7F71F10001F5D3DFE741F2DE
:107AE0008937D6F88C3213B11B69984780B9013FAA
:107AF00021D00DF001F804460D460CF0FDFF001BEF
:107B000061EB0501B0F57A7F71F10001F5D3E8E78B
:107B10000BEB482008F101084FF4007249467FF052
:107B20009FFAD045B9D1D6F84C47B6F85027002077
:107B3000A261BDE8F88FD6F84C374FF0FF30B6F8A9
:107B400050279A61BDE8F88F204600242DE9F84FB0
:107B5000364E90469A46B6F85027D6F84C4713044E
:107B6000A361BAF1000F54D0C8EBC853C24406F564
:107B7000FC6901EB432B4FF400720BEB48214846A4
:107B80007FF06EFAD6F88C220AB341F289370023CF
:107B9000D468494640461A46A047D6F88C32B8B158
:107BA0000BB11B699847013F37D00CF0A5FF044685
:107BB0000D460CF0A1FF001B61EB0501B0F57A7FCB
:107BC00071F10001F5D3D6F88C22002ADFD1002311
:107BD00041F2893713B11B69984790B9013F1CD016
:107BE0000CF08AFF04460D460CF086FF001B61EB8B
:107BF0000501B0F57A7F71F10001F5D3D6F88C322A
:107C0000E8E708F10108D045B5D1D6F84C47B6F8F9
:107C100050270020A261BDE8F88FD6F84C374FF00E
:107C2000FF30B6F850279A61BDE8F88F204600244F
:107C300010B50F4CE36D23B119689A880B691A428D
:107C40000AD0FDF7EDFD38B994F824300133DBB2EA
:107C5000072B84F8243003D9002384F8303010BD7A
:107C6000044A0123126884F83030226210BD00BF3C
:107C700020460024742F002410B50B4CE36D23B173
:107C800019689A880B691A420AD0FDF7C9FD38B9FC
:107C9000064B0122A0841B6884F83020236210BDAB
:107CA000002384F8303010BD20460024742F0024B7
:107CB00070B5164D0021164E6B6C2C681B04F162DA
:107CC000144A0D21A3602046E3681A4041F20D13C7
:107CD000134341F28832E360FBF700F950B16B6B5C
:107CE00003436B630C4A09230020126886F8303086
:107CF000326270BD636903F4F053B3F5006FF1D1E4
:107D00000423022086F8303070BD00BF10350024F7
:107D100020460024C0E0FEFF742F002470B50C4DF7
:107D200004460E4695F83030042B0AD0082B06D1B5
:107D3000AB6A83420AD0FFF7BBFF022801D00120C3
:107D400070BD0823C5E90A4685F83030022070BDB1
:107D50002046002470B5804C94F830506B1E082BE0
:107D60001BD8DFE803F06C60701A4705321A240054
:107D70007A4B5B6A002B60D1794B0722A5691B689F
:107D800084F830202362002D57D0E3690120D4E924
:107D90000321A84794F830506B1EDBB2022B46D962
:107DA000042D18BF082D0CBF0120002070BDFDF769
:107DB0000BFD002840F0C480694A236A1268FA3338
:107DC0009342EDD2FFF734FFC6E7FDF7FDFC002834
:107DD000F2D0E36A0022012B84F8242040F2B48020
:107DE000A26A013B08210132E36284F83010A262EA
:107DF000012070BD594B1E6A002E65D1FDF7E4FCD1
:107E0000002868D00423A56984F8246084F8303001
:107E1000002DEDD0E3693046E2682169A84794F867
:107E200030506B1EB9E770F095FB04285FD04C4BC7
:107E3000226A1B689B1AC82B77D8002070BD0223CA
:107E400084F8303088E7FEF7DBF90028EFD1454BA6
:107E50000421E06293F82C2084F83010D88D196B3F
:107E600084F83A20090E1A6B2087120C84F83B1014
:107E7000196B186B84F83C20090A84F83E0093F8CB
:107E8000340093F8352084F83D10120984F83F003F
:107E900093F8350084F84420996B00F00F00DD8FD3
:107EA000DA8F2164D98FC2F30B1384F8450043EABB
:107EB000152301F00F0203F00F0384F8482003F5A7
:107EC000FA63A4F8463047E7254A236A1268643308
:107ED0009342BFF465AFFFF7ABFEA569002D3FF4F9
:107EE0003BAF0022E36921691046A84734E7FEF75B
:107EF00087F900289BD11C4B1B78002BA3F10203B0
:107F0000B3FA83F308BF01255B0984F8265084F88F
:107F10002730FEF775F900287FF454AF114B032288
:107F20009B6C84F83020636316E7FFF781FE94F8BA
:107F30003000042818BF08280CBF0120002070BDA5
:107F4000042384F8303053E7FAD1FFF7B1FE94F8F8
:107F500030506B1E21E700BF2046002490350024DE
:107F6000742F0024B83500248C3500242DE9F0410D
:107F7000584C0D460646904694F830101F4604298A
:107F80000CD008297DD1A36AB34207D0FFF790FE39
:107F9000022876D194F830100429F2D101234E4AF8
:107FA000C4F8188023755362EB06E761C4E90356F1
:107FB00060D1BFF34F8F494A05F500712B46C2F8D7
:107FC000683220338B42FAD1BFF34F8FBFF36F8FEC
:107FD000002D79D0DFF8108198F83030012B49D18D
:107FE000731CD8F8501000228B42C8F834204BD8AC
:107FF0000323D8F80070C8F81C50182188F83030D6
:108000004FF40073FA623846C8F82030D8F8383098
:10801000334A012B4FF0FF337B624FF4007318BFDC
:108020007602BB62FB6A23F0FF0343F09003FB621E
:10803000FB6843F04003FB609023BD6501253D656F
:10804000C8F82C30BE60FB681A4041F21813134385
:1080500041F28832FB60FAF741FF50B3214B002216
:10806000BB63D8F834300343C8F8343088F8305054
:10807000C8F82C2094F82530022B0CD8013384F852
:1080800025300120BDE8F081D8F8343043F000738A
:10809000C8F83430EEE7002684F82560FFF7C8FD05
:1080A000A56925B1E369324621690120A84703206B
:1080B000E8E7FB6B062284F8250043F48D7384F80F
:1080C0003020FB63BDE8F081074A536B43F0006347
:1080D0005363CFE7204600249035002400ED00E0F4
:1080E000C0E0FEFFFF0FE01F103500242DE9F84F20
:1080F0005C4F0C468046164697F830101D46042902
:1081000008D0082902D00020BDE8F88FFFF7D0FD85
:108110000228F8D114F01F016AD10122524B5348B2
:108120009A6002624FF40072C7F8E0495A60002C6E
:1081300000F08A80DFF844B19BF83030012B57D132
:1081400008F10100DBF85030CBF83410984200F20F
:1081500081800323DBF800A04FF001098BF8303059
:108160005046DBF83830CAF82C101121012B4FF0A3
:10817000FF33CBE90942CAF824304FF4007314BF2F
:108180004FEA48224246CAF82830DAF82C3023F069
:10819000FF0343F09203CAF82C30DAF80C3043F0B6
:1081A0004003CAF80C308123CAF85840CAF85090EE
:1081B000CBF82C30CAF808202D4ADAF80C301A40D7
:1081C00041F21113134341F28832CAF80C30FAF726
:1081D00085FE034618B3274ACAF83820DBF8342056
:1081E00013430022CBF834308BF83090CBF82C209E
:1081F00097F82530022B03D8013387F8253082E722
:10820000002587F82550FFF713FDBC69002C3FF4CB
:108210007AAFFB692A4639692846A04773E70522E9
:1082200087F82530DAF83C30484687F8302043F4A8
:108230009573114ABE61CAF83C301368FD613B6218
:10824000C7E90348BDE8F88F0C4A536B43F000635D
:108250005363CDE7DBF8343043F00073CBF83430B0
:10826000C6E700BF204600240050002490350024BB
:10827000C0E0FEFFFF0FE01F742F00241035002424
:108280002DE9F04104464FF41D707EF01FFF0546B6
:1082900000285BD0D4F8D47204EB8707C7F8C0027B
:1082A000237CC4F8BC02002B45D0402302220121CC
:1082B000204677F0FBFE012240234FF001082046C4
:1082C000A4F8782181210222002677F0EFFEA4F89D
:1082D0003880D7F8C43230462E81A5F8606285F820
:1082E00062621B689847D4F8C84294F894342768AF
:1082F000434508D03846FAF7BBFE41463846FAF700
:108300008FFE84F8946405F504751F220023384617
:1083100004F51E71C4F88C320123C4E9A152A2797C
:10832000A4F878329A4208BFC4F8945278F03CF826
:108330000020BDE8F0814FF40073022201212046A5
:1083400077F0B4FE01224FF40073B6E7D4F8D432CC
:108350000220B03344F82350EBE700BFF0B5002310
:1083600083B0ADF80630D0F8D43200EB8303D3F8F5
:10837000C0524DB10A78044612F0600036D0202871
:1083800005D0204677F0D6FF032003B0F0BD487833
:10839000FE2849D0FF28F4D14B88002BF1D1CE889C
:1083A000002EEED11006ECD44FF4807381212B8186
:1083B00005F50475D4F8C842204679F02BFA20461A
:1083C000012179F027FA1F22012304F51E7120688C
:1083D000C4F88452A4F87832C4E9A226A2799A4259
:1083E00008BFC4F8945277F0DFFF46E04B780B2BC0
:1083F000C7D801A252F823F07F840408EF84040850
:108400008383040883830408838304088383040824
:108410008383040883830408838304088383040814
:10842000B78404086F8404084E88002EA9D1CF8831
:10843000012FA6D11206A4D5D3F8C4329B69984760
:10844000022328604FF48071C4F89432D4F8C83203
:10845000C4E906779A79998203F11401012A5F62CF
:108460001D629E6241D0186877F09EFF05E094F887
:108470009C32032B85D18B786B60002085E794F8C4
:108480009C32032B7FF47DAF0222D4F8C832002047
:10849000C4F8942203F11401C4E906220DF1060484
:1084A0009862C3E908424FF480729A829A79012A4D
:1084B000D9D11C63D7E794F89C32032B7FF461AFCA
:1084C000D4F8C8320122022104350020C4F89412E5
:1084D0004FF48071C4E90622C3E908529A7999825F
:1084E00003F11401012A9862BDD11D63BBE794F822
:1084F0009C32032BC1D14B88002BBED1D4F8C8626B
:108500008F8896F89434012B0AD0012339063068FD
:1085100086F8943410D4FAF7ABFD002386F894342F
:108520006B7A022B0DD03A06A7D5012BA5D00121DD
:108530002046FEF733FBA0E707F00F01FAF770FDC6
:10854000EBE72046812177F0B9FE0121204677F044
:10855000B5FE92E7F8B5D0F8C852012604460022CD
:1085600095F89434A5F87862B34227D0314628684C
:1085700085F89464002778F0A7F840F20113A4F876
:10858000787132463146286885F894642B8778F0F4
:108590009BF885F89474D4F8D4320025B03325873D
:1085A00054F8230040B17EF099FDD4F8D432B033B2
:1085B00044F82350C4F8BC520020F8BD40F2011327
:1085C000A0F878212B87E6E72DE9F04FDFF8B4B368
:1085D0008BB0DBF8ECA9DAF8143013F0010902D003
:1085E0000BB0BDE8F08FDAF81420DAF818301A4230
:1085F000F6D0DAF808280AF50061DAF81430C2F388
:108600000D220291CBF8C02EDAF8182013409D07F6
:1086100005D5DAF8143003F00203CAF81430DAF89A
:108620001430DAF818201340DC061BD5DAF81830BD
:1086300023F01003CAF81830DAF8203003F4F012EF
:1086400003F00F05B2F5802F00F04985B2F5402FF9
:1086500000F02583CDF804A0019A936943F010033C
:10866000936101E0CDF804A0019A53699269134027
:10867000180300F19C82019A5369926913405F03C9
:1086800000F1D281019B5A699B691A4200F1EA808C
:10869000019A5369926913401B0509D5029B9B6897
:1086A000DF0700F16485019A536903F400635361A5
:1086B00001994B698A6913401E0116D54B6903F075
:1086C00000634B619BF8B83E002B00F0C282DBF8E0
:1086D000CC3E93F89C22042A04D093F89C22D2B278
:1086E00083F89D22042283F89C22019A536992699F
:1086F0001340DD0400F14881019A536992691340E7
:108700009C0400F1D780019A5369926913401907BC
:1087100000F1C38001994B698A6913401A067DD420
:108720004B698A691340DB0228D59BF8F089B8F1C0
:10873000010F1ED9924D0AF51267012604E0013699
:1087400020372435464514D095F83C303A68012B43
:10875000F5D1002AF3DA66F07F0085F83B30C0B22D
:1087600070F0D4FBEBE7019A536992691340DA0287
:1087700004D5019A536903F480135361019A536934
:10878000926913409F0231D59BF8F079012F28D9C7
:108790000AF532627A4B012103E0B94203F1240366
:1087A0001FD093F87C020131146820320128F4D1E3
:1087B000002CF2DADBF8C05E85EA1445EE07ECD453
:1087C00083F87B02DAF8180040F08000CAF818003D
:1087D000DAF814000506E0D4029A536843F40073F3
:1087E0005360019A536903F400135361019A53696A
:1087F000926913405C0000F1BD8001994B698A6960
:10880000134058077FF5ECAE4C68610700F1BF8458
:10881000DBF8EC395A6814435C60E1E6DAF81830AA
:108820009BF8F08923F08003B8F1010FCAF81830E3
:1088300099D9534D01262F4603E00136243746458A
:1088400007D097F87B32012BF7D1F0B270F05EFBC6
:10885000F3E7019B5A699B691340DB028ED59BF8B5
:10886000F08968E7029A536823F0010353609BF88C
:10887000B83E012B00F00182DBF8CC3E93F89C223D
:10888000042A04D193F89D22D2B283F89C22019A43
:10889000536903F000435361FAE6DBF8CC0E90F81D
:1088A0009C32032B00F0ED81019A536903F0080319
:1088B00053612FE7019AD2F800396FF30A03C2F827
:1088C000003902F50063D2F8042842F480725A603D
:1088D0009B68980700F1F78113F0060F0CBF002387
:1088E0000F238BF8F339F9F72FFA9BF8F369022E6F
:1088F00000F06F844FF410530199003EDBF8CC5E1A
:10890000CA6818BF012622F47052CA60CA681343AD
:10891000CB600123002185F89C32D5F8B83269601C
:10892000C5F8A41285F8A012C5F894121BB15B68B3
:108930000BB12846984700224024012740231146C6
:10894000284677F0B3FB2346002280212846C5F84D
:108950006041A5F8647177F0A9FBDBF8CC3EDBF849
:10896000EC29AF842C621E745369019203F4005306
:108970005361C8E6019A536903F0804353613CE7B1
:108980000C50002420460024029A102101985368BC
:1089900023F001035360FAF743FB9BF8F009E0B1C1
:1089A0000AF510634FF67F31996009F101091A68E1
:1089B0002033814522F4001243F8202CC3F8E8113B
:1089C000D3F8E02122F40012C3F8E021D3F8E0212B
:1089D00042F00062C3F8E021E6D1029AD36943F085
:1089E0000113D3619BF8FB39002B00F03B81029A05
:1089F000D2F8843043F00B03C2F88430536C43F058
:108A00000B035364DAF80038019C23F4FE63B44A84
:108A10002046CAF800389BF8F21977F0C9FB636961
:108A200003F48053636167E6019AD2F81878D2F8AC
:108A30001C381F40BFB2002F3FF424AE0AF510616E
:108A40004FF00008CDF80CA01346A64D44468A46C8
:108A5000CDF8109008E07F0804F1010405F1240529
:108A60000AF1200A00F03181FE07F4D5D3F810286E
:108A700004F00F01D3F834684FEA4419CE40F601F0
:108A8000F6B2164303F5106202EB441292681640E8
:108A9000E2B2F007019221D50120029ADBF8CC8ED8
:108AA000526B00FA01F122EA010202994A639BF833
:108AB000F219CAF80800814200F078832B6A059306
:108AC000002C40F0FA82D8F89432022B00F0E883B0
:108AD00098F8A03213B1002388F8A032320702D5EB
:108AE0000823CAF80830F30602D51023CAF8083064
:108AF000700602D54023CAF80830B10700F1108192
:108B00003206DBF8EC39A6D5D5E909068642A2D8AB
:108B1000811BEA6903F5106E8A42CE4428BF0A46DB
:108B2000DEF81810033289B2B1EB920F31D39BF803
:108B3000F28903F5805C019442460CEB043C9846B4
:108B40001346B04240F29083811BEA69914228BFEC
:108B500011462A6A01F103094FEA990973B98CB2E7
:108B60000334A4080AD002EB840452F8040BA24296
:108B7000CCF80000F9D12A6AD5E909060A440E4466
:108B80002A62DEF81820AE6292B29145D9D9019CD2
:108B90004346B0423FF65FAF04F00F02012191401F
:108BA000D3F8342822EA0102C3F8342853E70198A5
:108BB000D0F81838D0F81C2813405FEA13483FF467
:108BC0005AAD484B0AF53066CDF80CA000279A46FE
:108BD000CDF8149008E05FEA580807F1010706F1A4
:108BE00020060AF1240A74D018F00109F3D0FBB270
:108BF00000F530627D01019302EB47139C68D0F8C9
:108C000014180C40E1076FD4210700F19580E506A8
:108C100001D51023B360A0070FD5039B5B6919062C
:108C200004D5029A536843F4806353609AF857322C
:108C3000012B00F01C830223B360A20601D5202380
:108C4000B360A30402D54FF40053B360DBF8EC0922
:108C5000C1E701238BF8B83E4B6DC3F38303CBF818
:108C6000BC3E42E5029942F22B034A6913434B6131
:108C70000B6943F00B030B61C4E600238BF8B83E8D
:108C800005E6D0F8B832002B3FF40EAEDB69002BBE
:108C90003FF40AAE9847DBF8EC39019304E605EBA4
:108CA000C5020AF58051C3F30A130BEB8202D2F816
:108CB000540C03440868CBF8880E0968C2F8543C89
:108CC000CBF88C1EC6E402230BE6DDE903A9019371
:108CD000D8E4DDF80CA0DDF814900190CBE400BFDF
:108CE000A85400240C5000240121B1609BF8F21913
:108CF000D0F840E00129D3F808C000F0A582B649B9
:108D00008E4500F09B83DBF8503C3B4300F04984E8
:108D1000DAF860220199DBF8CC0E77F07BFC73E780
:108D200021460398FAF77CF9EB7D012B00F0918343
:108D30000223CAF80830E3E6DBF8EC290823B36025
:108D400002F53063126C2B4410460492A34A9968D2
:108D5000904204D90A0402D54FF400429A60DBF82D
:108D6000CC5E01219BF8883E05F2AA2085F8AA3244
:108D70009BF889EE079085F8ABE2BBF88A2EA5F840
:108D8000AC22BBF88CCE0692A5F8AEC2BBF88E2EF4
:108D9000C5F8941203F01F01A5F8B0220129C5F807
:108DA000982200F0A582022900F00783002940F0F4
:108DB000DE8203F06003202B00F0E983402B00F0FB
:108DC000E683A3B9BEF1090F11D8DFE81EF0E80071
:108DD000C1001000D80010007D00640010003E00AB
:108DE0002300D5F8B4325B69002B40F0C2852846D9
:108DF00077F0A0FA794B049A9A427FF608AF9BF875
:108E0000F21901297FF403AF754ADBF8EC0977F01A
:108E1000CFF9FCE69DF81890B9F1010F8BF8D09EC0
:108E2000E5D895F89C32DAB2022B069200F0038561
:108E3000032A00F0D784284677F07CFAD5F8B832B8
:108E4000494628465B689847D4E7012ACFD195F870
:108E50009C120229CBB200F2A684002BC7D0D5F811
:108E6000C832002128464FF0020C40F8081FC5F810
:108E700094C2C5E90622C3E9092118624FF4807241
:108E800003F114019A829A79012A08BF18631868BD
:108E900077F08AFAAEE7069B00221B0AADF826207F
:108EA000013B062BA3D801A252F823F08D900408B1
:108EB0007190040847900408EF8D0408EF8D0408B2
:108EC000E58F04089F90040852EA0C0C8FD1069B92
:108ED0007F2B8CD895F89C32032B88D00698D5F838
:108EE000C8325FFA80F985F89E9293F89424012A9B
:108EF00012D01A684FF0000C83F81190D2F80018C5
:108F000021F4FE61C2F80018D2F8001841EA0011FD
:108F1000C2F8001883F894C40422002003F114015D
:108F2000C5F894224FF48072A8619A829A79986267
:108F3000012AC3E9080008BF1863186877F034FAFB
:108F4000B9F1000F40F07284012385F89C3251E79B
:108F500095F89C32013B022B3FF649AF069B012B53
:108F60007FF448AF0020D5F8C832C5F8A402A86144
:108F70000422C5F894229862C3E908007EE7069BA4
:108F8000012B00F06F84069B022B7FF430AF4FEA79
:108F90001C2CD5F8C832002085F8A0C2E7E795F868
:108FA0009C32013B022B3FF622AF022A7FF41FAF17
:108FB000D5F8A4322846002B18BF4FF0030940F81B
:108FC0000C9FD5F8C832C5F89422C5E90622C3E93A
:108FD000080200229A6251E70A31544F0A30544F76
:108FE000A85400242B7C002B7FF401AFD5F8B832B5
:108FF0000DF126005B6B98470346B5F8B0020028D8
:1090000000F03884BDF82620002A3FF4F0AE8242FA
:109010004FF0020128BF0246D5F8C802C5F89412E5
:1090200000F11401C5E90622C0E90832002282627B
:109030004FF4807282828279012A08BF036300683C
:1090400077F0B2F9D6E69DF8180005283FF6CFAEC6
:1090500001A353F820F000BFAB9904089D990408C0
:109060008F99040881990408E38D0408679904081E
:109070002A7CD5F8B832002A40F072849B6A0DF140
:1090800026009847022203464270B6E7D5F8B4326C
:109090000DF12601287C1B6898470346ADE72B7C21
:1090A000002B7FF4A4AED5F8B8320DF126001B6B6F
:1090B00098470722034642709FE798F89C32032B9B
:1090C0007FF40CADD8F8B8325B69002B3FF406ADE5
:1090D000002240460199C8F8D4229847FEE447F69A
:1090E000F07213423FF4B6AA05EBC502C3F388142D
:1090F0004FEA131CC3F301130BEB8202EE00D2F80C
:109100004C7C002C00F000830AF5805E002239467A
:109110000132DEF80000944241F8040BF8D107EB6D
:109120008404002B00F0BC810AF5805223441068AF
:10913000002220FA02F1083204F8011B9C42F8D107
:1091400073190BEB8303D3F84C7CDBF8EC390193F8
:109150007319CCF30A0C0BEB83036744D3F8542C3C
:10916000C3F84C7C6244C3F8542CFFF775BADBF8A3
:10917000CC3E93F89C22042A04D093F89C22D2B2CD
:1091800083F89D22042283F89C22FFF78CBADBF837
:10919000CC0E0122D0F8B83280F89C22002B3FF48C
:1091A00037AB5B6801799847FFF732BBD5E9070217
:1091B00002442A62002C80D1DBF80C0ADBF8102A6A
:1091C0000590002A7FF47FAC1846B74A76F0F0FF8E
:1091D00079E4B64BB64A0344934240F25281B54B10
:1091E000B54A0344934240F25781B44BB44A034416
:1091F000934240F23582B34BB34A03449342C0F0EA
:109200006B82B24BB24A0344934240F29182B14B1B
:10921000B14A03449342C0F08F82B04BB04A03443A
:109220009342FFF467ABAF4BAF4A03449342C0F0A5
:10923000D582AE4BAE4A034493422CBF4FF4C05389
:109240004FF4E053FFF758BB1CF0080F00F01D81EE
:10925000A84A96457FF6D8AC1CF4004F3FF4D4AC36
:109260004FF400429A60CFE4019C434694E400230B
:109270008AF85732DBF8CC0ED0F8D432AE3350F83F
:109280002330002B3FF4D7AC90F89C22032A7FF4C4
:10929000D2AC5B6A002B3FF4CEAC01999847CAE48C
:1092A000D8E90732934200F2278100F0988198F8BC
:1092B0009C32032B00F0C8818021404676F0FEFFEF
:1092C00005230020C8F89432D8F8C8329A7903F5FB
:1092D0001571C3F86802012AA3F85402C3E9980083
:1092E00008BFC3F87002186877F05EF8FFF7F0BBAC
:1092F00003F060025B0602D5402A7FF478AD95F852
:109300009C32013B022B3FF672AD5FFA8CFCBCF144
:10931000030F3FF66CADD5F8B8329B68002B3FF4D5
:1093200069AD4FF0000907992846C5F8D4929847CF
:10933000B5F8B022002A7FF45DAD00287FF45AAD65
:109340000422D5F8C832C5F81890C5F894224FF415
:10935000807203F11401C3F828909A829A79012A45
:10936000C3E908997FF493ADC3F830908FE51B06ED
:10937000D5F8C85200F12D81002385F8553205F546
:10938000157301224FF000099A7083F8009095F848
:10939000941491423FF42EAD286885F894245A78AD
:1093A0001978069076F050FF069805F29C42A9794C
:1093B00076F0FEFE85F894941CE503F06003202B04
:1093C00000F07C81402B00F07981002B7FF40FAD01
:1093D000BEF1010F5FFA8CF100F04681BEF1030F80
:1093E00000F07E81BEF1000F7FF401AD95F89C3254
:1093F000022BDAB200F0A481032A7FF4F8AC01F06A
:109400000F0314221CF0800F02FB035340F0B281C3
:10941000B3F86431002B3FF4EAAC02FB015202F5D1
:10942000AA70002940F02B8200230360D5F8C832CF
:109430000222C5F89422C5E90622C8E51CF4004FB3
:109440007FF40EAF1CF0200F3FF462AC20229A6034
:109450005EE40023EB75DBF8CC0ED0F8D432AE33EB
:1094600050F82330002B3FF463AC90F89C22032A81
:109470007FF45EAC1B6A002B3FF45AAC019998470D
:1094800056E44FF47053FFF737BA1CF0200F60D04A
:1094900020229A60FFF7B8BB4FF46053FFF72CBA55
:1094A000CDF804A054E600BFA8540024405327FF81
:1094B000FF340C00401E1BFF3F420F0000DC0BFF7F
:1094C0007F4F1200808CF9FE20D6130060B6E5FEB7
:1094D0005FE3160000D3CEFE40771B00C05BB3FEF7
:1094E000C091210000CA91FE20753800E05459FE59
:1094F000E09C41000A30544F9A1AD8F8C832C8E9A3
:1095000006225A6203F11401059A1A6200229A6235
:109510004FF480729A829A79012A01D105981863D2
:109520001868CDE9050376F03FFF069B00209A7985
:1095300003F51571C3F86802012AA3F85402C3E9C0
:10954000980008BFC3F87002059876F02DFFFFF76A
:10955000BFBAC64A964503D91CF4004F7FF480AECB
:109560001A69DAF87432C2F312029B1ACAF8683226
:10957000002F7FF4CDABDBF8502C002A00F0D28016
:10958000DBF84C2C1A44CBF84C2CFFF7C1BBD5F8B8
:10959000D43228460799AE3355F823309B68984754
:1095A00028E4016CB14B994203D91368002BFFF6F4
:1095B000AFAB00231361136943F4002313611369F4
:1095C00043F018031361136943F0C0431361FFF7BD
:1095D0009FBB4FF001036B7505F11403D1E6D8F87A
:1095E000182093423FF663AED8F898329A42BFF4FF
:1095F0005EAED8F8C83200204FF48072C8F8180068
:1096000003F114019A829A799862012AC3E9080049
:1096100008BF18631868CDE9050376F0C5FE069B00
:109620004FF0000C059803F51571C8F898C29A79A7
:10963000C3F868C2012AA3F854C2C3E998CC7FF4E6
:1096400053AEC3F870C24FE6D8F8B832DB68002BCF
:109650003FF432AE00224046C8F8D42298472BE6A9
:109660004FF45053FFF748B995F89C32022BDAB209
:109670004CD0032A7FF4BBAB069B002B7FF4BAAB24
:109680004806D5F8C89240F006810422002309F16B
:109690001401D9F80000C5F894224FF48072AB6130
:1096A000A9F8142099F80620C9F82830012AC9E938
:1096B000083308BFC9F8303076F076FED5F8B832F6
:1096C00000229B68C5F8D422002B3FF493AB079986
:1096D00028469847FFF78EBB4FF44053FFF70CB96D
:1096E00095F89C32022B5FFA83FC0FD0BCF1030F7C
:1096F0007FF47DAB480603D0069B134300F0C78080
:10970000D5F8C832002032E43C460AE54B0628462C
:109710003FF46EAB76F0D2FD2846802176F0CEFD88
:10972000FFF768BB524A012176F042FDFFF7F0BA1D
:109730004FF43053FFF7E0B84FF42053FFF7DCB895
:109740004A067FF454AB1CF0800FD5F8C8324FF0B6
:1097500002024FF0000114BF05F1140005F5AA70D4
:109760000160C5F89422C5E90622C3E909211862FF
:10977000FFF784BB9B8C002B3FF439AB01F07F01DA
:10978000481C00EB800005EB800000293FF44CAE44
:109790002422D5F8C83202FB01318A7D003A18BF75
:1097A0000122026044E6032B7FF421ABD5F8C832D6
:1097B0000221C5E90622C5F8941204355A62002236
:1097C00003F114011D629A624FF480729A829A79B1
:1097D000012A7FF45CAB1D63FFF759BB4FF40053C4
:1097E000FFF78AB8B9F1000F00F0AE80696801296F
:1097F00086D0D5F8B832C9B228465B6898479BF83E
:10980000D01ED5F8B8326960002B3FF479AF1B68E1
:109810002846984700283FF473AF284676F08AFD23
:10982000D5F8B832297928465B689847022385F82D
:109830009C32FFF7DFBAB9F1000F3FF481AD01218F
:10984000D5F8B8326960002B5AD01B682846984773
:10985000002855D0284676F06DFD069B85F89C3291
:10986000FFF7C8BAC5F8A4324AE700BF0A30544F20
:10987000A8540024D5F8C832A861FFF779BB242288
:10988000D5F8C83202FB013191F8562286E7284606
:1098900076F014FD34E701F00F0199F804308B42A3
:1098A000FFF4F3AE01EBC1031CF0800F4FEA83031A
:1098B00041D103F51573002209EB030C242303FBAC
:1098C000019383F855224FF000038CF800108CF8B8
:1098D000023099F89434012B3FF4D7AE0123D9F824
:1098E000000089F894349CF804309CF801209CF81E
:1098F000001076F083FC4FF0000389F89434C4E63E
:109900000422D5F8C8320020C5F894224FF48072A2
:10991000A86103F114019A829A799862012AC3E935
:10992000080008BF1863186876F03EFD032385F829
:109930009C32FFF75FBA1433012209EB030C242396
:1099400003FB01935A75BEE7022349462846C5F832
:10995000049085F89C32D5F8B8325B689847EFE4FC
:10996000DB6AFFF78CBBD5F8B4329B69002B3FF460
:109970003EAA0DF12601287C98470346FFF73DBB20
:10998000D5F8B4321B69002BF3D1FFF730BAD5F804
:10999000B432DB68002BECD1FFF729BAD5F8B4322A
:1099A0009B68002BE5D1FFF722BAD5F8B4325B688B
:1099B000002BDED1FFF71BBA2DE9F8434B4BD3F850
:1099C0009053EE682C69A70701D5B00736D461071C
:1099D00001D572072AD4270701D530071ED4E10626
:1099E00001D5F20612D4E70701D5F0073BD414F4F1
:1099F000025F2BD031066FD4600601D5710671D499
:109A0000A20601D5B30629D4BDE8F8836FF0100291
:109A10002A610022E96983F8AC23E4E76FF00802C9
:109A20002A610022E96983F8AC23D8E76FF00402C9
:109A30002A610022A96983F8AC23CCE76FF0020207
:109A40002A610022A96983F8AC23C0E7E305D3D5D6
:109A50003706D1D56FF480732B61CDE76FF020030B
:109A60002B61BDE8F883224B6FF001029D422A6111
:109A7000BDD1DFF88C801F4BD8F800201F68BA4298
:109A8000B5D01D4888BFC2F580571C4B98BFBF1A80
:109A90001A44D0F8D432B03350F82330002BA6D07B
:109AA000D3F81492C3F80822C3F81072B9F1000F6A
:109AB0009DD10121C762C3F814123B46812176F083
:109AC00083FDD8F800301F44B7F5805F14BF3B46D4
:109AD0004B46C8F800308AE76FF40253E2052B6169
:109AE0008AD5B7E76FF040032B6189E72046002451
:109AF000001400406C2F00248C2C0024F45400240B
:109B0000682F00242DE9F04F394B0A46394E83B0B7
:109B1000D3F8BC12D6F800A004E03368A3EB0A0324
:109B2000322B60D8D1F81432002BF6D1002A56D04F
:109B300000F1FF3B1946304F4FF070085B46DFF8ED
:109B4000C0908B46396813F8010F2C4C60540131DA
:109B5000C1F30B013960EFF3118088F31288C0B2B2
:109B6000D9F800103C6880F31188A142A1EB0401F0
:109B70008CBF0020012001EB003101292AD1CDE961
:109B800000323368A3EB0A03322B27D80AF0B4FF64
:109B900004460D460AF0B0FF001B61EB0501B0F56D
:109BA0007A7F71F10001F5D3EFF3118288F3128807
:109BB000D9F80030D2B2396882F311888B42A3EB16
:109BC00001038CBF0022012203EB0233012BD8D00A
:109BD000DDE900320BF1010B5A45B3D15B46184663
:109BE00003B0BDE8F08F0023184603B0BDE8F08F46
:109BF0008C2C0024742F00246C2F0024F454002497
:109C0000682F002402784368022A0FD00B490269AA
:109C1000D1F88002023A184010B4400AD1E99D14EC
:109C200004FB02005DF8044B08447047034AD2E984
:109C30009A2102EB410202EB532070472046002498
:109C40002DE9F04F83B002F00207844D019308B96B
:109C5000002F6AD1D5F87042002C53D14FF0FF3E4F
:109C60007F4C4FF0000CF146F046F246E36994F861
:109C70002A60984200F0A080002E3BD0012E05EB18
:109C80000C1B0AD19BF88F60F30706D416F07E0FE9
:109C900003D1F60900F09380E0460CF1010C10347A
:109CA000BCF1080FE2D1BEF1000F04DAB8F1000FE9
:109CB000C0F29780C646D5F800410EF1020605EBCA
:109CC0000E18013405EB061CC5F800410CF1640CBC
:109CD000CCF80440C8E920040024CCF8084005EB87
:109CE000061494F86E40042C1FD8DFE804F02944D1
:109CF0001A444600E6460CF1010C1034BCF1080F82
:109D0000B4D1D0E7D5E99D3606FB0434A042A5D3F3
:109D100095F81C3213B9012385F81C32012385F80C
:109D20006530002003B0BDE8F08F95F81C32002BA1
:109D300053D00123022085F8653003B0BDE8F08FD1
:109D400012F00104D5F87CC073D105EB0610019B1D
:109D50004FEAE20C90F86F80032B6CF3C71880F881
:109D60006F8064D94FF6FF70834228BF034605EB2E
:109D70000610A0F86C30002F45D1500707D505EB31
:109D8000061090F86F3043F0010380F86F30D3066F
:109D90000AD505EB061696F86F30C3F3450201327B
:109DA00062F3460386F86F30EB6F012003EB4E231E
:109DB0000B6003B0BDE8F08FC6B9E6467BE7666A84
:109DC0001034B24588BFE1460CF1010C88BFB246A1
:109DD000BCF1080F7FF44AAF65E7012385F81C3218
:109DE000A7E7B9F1000F9CDBCE4664E7D5F8004148
:109DF0000CF10206E646013405EB061CC5F80041ED
:109E0000CCF868406BE7D5F80401D5F80031013093
:109E10000133C5F8040105EB0E10C5F80031C0F898
:109E2000843005EB0613042083F86E00A5E7234673
:109E30009DE7D5F88C32002B3FF473AF5C680CEBD8
:109E40004E210023074AA04700283FF46AAF05EBE4
:109E50000616022386F86E3063E700BF2046002412
:109E6000844600248D66040870B5114D82B00E46FC
:109E700095F86430022B16D1020AC4B2D5F86802F4
:109E8000002301A910440322FFF7DAFE012808D1BC
:109E900095F86430019A022B0CBF22F8146042F846
:109EA000246002B070BDC0F3D41200F07F04E5E777
:109EB000204600242DE9F04F444E0D4683B017464E
:109EC00096F864102B6803293ED0022961D14FEA2D
:109ED00013294FF4807A5FFA83F8421E012A23D8AF
:109EE0004FF0010B9F421AD901288CBF0024012496
:109EF000D6F8E0211AB1D6F8FC1199424CD0D6F828
:109F000068020023092201A94844FFF799FE0128AD
:109F100023D0022814D020B12B689F42E8D8032018
:109F20002F6003B0BDE8F08FB8F1000F13D096F8A2
:109F30001C3213B9012386F81C32012386F86530E0
:109F4000022003B0BDE8F08F4FF0800AC3F3D419AC
:109F500003F07F08C1E7D346C4E796F864100229EE
:109F600013D00329ECD1019B53F8282022F0704232
:109F7000B2FA82F22B685209A2421FD0D8445B4445
:109F8000D0452B601DD20229EDD1019B33F818205A
:109F9000EEE74FF4807AD9E7D6F87812013A02EB6F
:109FA00041224902B2FBF1F21344B3FBFBF20BFB7B
:109FB00012320AB15B449B1A2B60AEE79F42B0D8C5
:109FC000ADE709F101094FF00008A6E7204600249B
:109FD0002DE9F04FDFF884918B4685B0174699F84C
:109FE00064C00968BCF1020FD9F8685240F0828061
:109FF000CEB24FF4807305EB1125A6EB0108904417
:10A000009844B94208F1FF38B8FBF3F84AD200F09F
:10A010000103A8446FF0404A0193BCF1030F07EB22
:10A020000604A8EB0503284614BF4FF48072802273
:10A03000641A03A9944228BF1446944228BF002EF4
:10A0400014BF012200220A32FFF7FAFD01282AD1AB
:10A0500099F864C0DBF800E0BCF1020F0EF10103D7
:10A0600024D0B44255D9039806EB0A02011F00EB35
:10A07000820201EB840142F8043F8A4203F10103AA
:10A08000F9D1DBF80030A11B19448F42CBF8001046
:10A0900002D1019B002B48D18F4205F101054FF001
:10A0A0000006BAD8012005B0BDE8F08FB44246D909
:10A0B00003986FF00042811E324401EB440100EB33
:10A0C000420222F8023F914203F10103F9D1A11BA0
:10A0D00071448F42CBF80010DED1019B002BDBD006
:10A0E00086466FF000434FF6FF72012023442EF89E
:10A0F0001320D8E701F07F06C1F3D413BCF1030F9E
:10A10000A6EB01081D4414BF4FF4807380239044D4
:10A1100076E7AEEB060E0EEB04018F42CBF8001093
:10A12000BAD1019B002BB7D003986FF040434FF09A
:10A13000FF32234440F82320DBF80010ACE7AEEBFD
:10A14000060E0EEB04018F42CBF80010A4D1019B48
:10A15000002BA1D0DDF80CE0C3E700BF20460024AF
:10A1600030B50446C06983B010B9012003B030BDDA
:10A170000D460023032201A9FFF762FD0128F5D156
:10A18000B4F92020002A19DB019B012D4FEA42116E
:10A1900003EB421203D0022D1BD1E5205854A368D3
:10A1A000D3612378032B04D100231377537793775C
:10A1B000D377636A190C53839182D6E7064A92F8E3
:10A1C0001C1209B982F81C020123022082F86530B2
:10A1D000CCE7E368E4E700BF204600242DE9F04126
:10A1E000044682B00D4694F83C30042B7ED8DFE85C
:10A1F00003F02B0369493A003D4E4FF6F777DFF83D
:10A20000F48016E0BA425BD86DF052FE01284FF0A0
:10A21000000134D1206BFFF727FE01282FD1019ACE
:10A22000D6F87C12531E22638B4228BF0B46C6F819
:10A230007C3296F8642001A9236B032A18469AB24F
:10A24000E0D14345E0D93BE06900204601F0FE0142
:10A25000FFF786FF01283FD1636B002B18BF022058
:10A2600084F83C00BFE794F82830042B02D1002387
:10A2700084F82830A36B0BB120469847012002B028
:10A28000BDE8F0811A4E0021E26AD6F8FC3106F5ED
:10A29000EC70C6F8FC219B1AD6F8782202FB03F377
:10A2A000D6F8E02102EB4322C6F8E021D6F8E421FB
:10A2B00002EB4322C6F8E421FFF752FF01280BD13D
:10A2C0000420CDE7626B04F130010020FFF780FE2F
:10A2D000012801D10320C3E70228D0D194F8283007
:10A2E000042BCCD1002384F82830C8E70220F5E7FE
:10A2F00020460024F7FFFF0F38B5044694F83430A9
:10A30000052B60D8DFE803F031251D130D0394F809
:10A310002830082B3FD02D4B0122022083F81D222C
:10A3200038BD94F82830082B30D0012038BD0021EA
:10A330002046FFF715FF012845D1042084F834009A
:10A34000DCE7D4E90B01FFF78FFD01283BD10320A7
:10A35000F4E74FF0FF31206BFFF786FD012832D183
:10A36000E36A002BF3D00220E8E7184D04F1300136
:10A370000120D5F870220232FFF79CFD012813D08E
:10A380000238C0B201281ED80520D7E700230120DB
:10A3900084F82830CAE700230122022084F82830FC
:10A3A0000A4B83F81D22BBE7E368D5F87812226BCD
:10A3B00003EB4123C5F87C22C4E90332E36A002B96
:10A3C000BCD16262BAE7002038BD00BF204600243D
:10A3D000F8B5044694F83830032B4CD8DFE803F086
:10A3E00021180B0200212046FFF7BAFE431EDBB204
:10A3F000012B41D9F8BD0120626B04F13001FFF758
:10A40000E7FD01284FF00303F0D184F83830E1E78D
:10A4100000211E48FFF7A4FE01284FF00203F4D0EC
:10A42000E4E71B4BE66893F86420D3F87812032A1C
:10A43000D3F8E051D3F8FC0114BF4FF480728022AE
:10A44000206102FB01F1871A0244A5EB412506EBCE
:10A450004126E660C3F8E051D3F8E451C3F8FC218B
:10A46000A5EB4121C3F8E411E36AC4E90C025BB92E
:10A4700060620123C9E7022094F82830062BB9D185
:10A48000002384F82830F8BD2763F2E7F84700245A
:10A49000204600244368C3F308020A44B2F5007F53
:10A4A0002DE9F041054682B00C4605D223446B608D
:10A4B000012002B0BDE8F08190F91A10481C0AD0C2
:10A4C000474A02EB011292F88F1021F0010182F845
:10A4D0008F10FF22AA7695F91B20511C16D0404EF2
:10A4E000023206EB021191F86F10C1F34501012908
:10A4F00044D9013901F03F0106EB0212FF2692F820
:10A500006F0061F3460082F86F00EE762A78022A27
:10A51000CCD0334ED6F87822B4EB422F4FEA422803
:10A520002EDCD6F880721F407A42A24228DCE21963
:10A530002869424513D32A7E12072DD5D6F8FC216F
:10A54000411C8A421ED300D100214344A4EB0808D9
:10A5500068610846DB1B08EB070429616B60002873
:10A56000A6D096F86420032A35D080B24FF6F77251
:10A5700090429DD81A4614446C6099E70021BBE7CD
:10A58000002096E796F81C220ABB012386F81C32AD
:10A5900086F865306B68D8E701A96DF089FC012861
:10A5A000EED16B68A4EB08042869984429786861A7
:10A5B0003C44A8EB0703019802291A466B60286106
:10A5C000CDD1D6F88812B3EB412FD4D370E7012256
:10A5D00086F86520B9E7034A90423FF669AFC9E7BC
:10A5E00020460024F7FFFF0F2DE9F0474FF0010848
:10A5F00082B0044694F83830032B00F2A680DFE8DE
:10A6000003F055170C020020236C84F8280003B1D6
:10A610009847022002B0BDE8F0870022236C84F83E
:10A6200028200BB120469847012002B0BDE8F087F2
:10A6300023786768022B03D0454BD3F880321F4044
:10A64000C7F34F272046FFF7DDFA414E3F1A054674
:10A65000BFB207EB050C022201A9002328461FFA0E
:10A660008CF9FFF7EDFA01284FF400724FF000016A
:10A67000D0D101987CF012FEE3694FF400712046BE
:10A680000BB16368EBB1D6F878325A1E914547D2C8
:10A690000135FFF7FFFE0028DBD196F81C3213B915
:10A6A000012386F81C3286F86580D2E72046FFF742
:10A6B00023FE012802D0022847D1032084F8380065
:10A6C00098E7019B4FF020324FF0100E4FF02E0C08
:10A6D00042F62E6AC3F80120C3F80520A3F809202A
:10A6E00083F800C0D4F824C0A3F820A083F80BE0BE
:10A6F000C3F82220C3F8262083F82A20E26BA3F8AF
:10A700001AC02CFA0EFC5A8722FA0EF2A3F814C0D3
:10A710009A8683F82BE0D6F878325A1E9145B7D343
:10A72000C3EBC3532046590201F50071FFF7B2FE97
:10A7300028B996F81C3223B1012386F8653002202F
:10A74000BCE7012386F81C32F6E7002062E700BF71
:10A7500020460024B1F904300F2B2DE9F0410D46BD
:10A7600082B00446164633D02046FFF74BFA94F9E0
:10A770001B80B8F1FF3F3CD05B4F07EB0813D3F8C9
:10A780008030984212D097F81C32002B6ED00123F3
:10A7900087F865302378022B5ED02269002A73D1B6
:10A7A00000230120336002B0BDE8F081F96F01EBB6
:10A7B0004821002966D0AB88204601331BB201EB4B
:10A7C0004311AB803160FFF71DFA28600120EAE7F2
:10A7D0004FF40071FFF75EFE002843D04FF6FF7381
:10A7E0002046AB80FFF70EFA94F91B80B8F1FF3FCB
:10A7F000C2D12378022B3DD02269002AD0D03A4F13
:10A8000097F86430032B66D093B24FF6F7718B4202
:10A8100094BF00230123002BC0D130B997F81C321C
:10A82000002B4BD0012387F865300023112201A9AA
:10A83000FFF706FA012825D10199FB6FCB1A48BF13
:10A8400003F2FF13B3F5805F4FEA63222CD24FFA75
:10A8500082F884F81B80ACE7D7F888226368B3EBF2
:10A86000422F9DD2002002B0BDE8F081012387F87D
:10A870001C328CE71C4F6368D7F88822B3EB422F59
:10A88000CBD38DE7237886E797F86430032B19D074
:10A8900093B24FF6F772934294BF00230123002B2B
:10A8A0007FF47EAF0020DEE797F81C3213B9012356
:10A8B00087F81C32012387F86530CAE7012387F83F
:10A8C0001C32AFE7094B9A4294BF00230123002BAF
:10A8D0007FF466AFE6E7054B9A4294BF002301235D
:10A8E000002B7FF45BAF98E720460024F7FFFF0FB3
:10A8F0002DE9F047044688B094F83030042B11D885
:10A90000DFE803F0501361035A00237E9A0640F1FA
:10A91000F8800023112204A9E069FFF791F90128CA
:10A9200000F0EF8008B0BDE8F087C44D03AE04F13D
:10A930001C0705F50879324639464846FFF70AFFF5
:10A94000012800F0F9800228ECD195F93A325F1C19
:10A950000AD005EB0313FF2193F88F2085F83A12F4
:10A9600022F0010283F88F2095F93B325E1C17D04C
:10A97000023305EB031292F86F20C2F34502012A5D
:10A9800040F25A81013A02F03F0205EB031393F8BB
:10A990006F1062F34601FF2283F86F1085F83B22A7
:10A9A000042306E0A6486EF087FD4FF6FF720123F0
:10A9B000228484F830309FE70020E36A207008B0DA
:10A9C000BDE8F04718479D4D95F84832002BA9D1B6
:10A9D00004F11C0705F5087803AE324639464046B7
:10A9E000FFF7B8FE012840F01581039B002B00F013
:10A9F000F0801A780AB1E52AEFD1EA6F9A1A48BFB7
:10AA000002F2FF12B2F5805F4FEA622180F04981C5
:10AA100009018C4A0A44917B04290CD0D5F8001115
:10AA20000131C5F80011516004219173D5F804215A
:10AA30000132C5F8042195F93A22501C0AD005EBE1
:10AA4000021292F88F1021F0010182F88F10FF227C
:10AA500085F83A2295F93B22511C17D0023205EBBA
:10AA6000021191F86F10C1F34501012940F2618193
:10AA7000013901F03F0105EB0212FF2085F83B028E
:10AA800092F86F0061F3460082F86F0020220021E7
:10AA900018467CF003FCD4F831100346D4F8352076
:10AAA00005A819605A6094F83B20B4F839109A72DE
:10AAB0001981627E0193DA7203F0CAF8019B0028C3
:10AAC00000F0D8809DF816009DF817209DF8191009
:10AAD00042EA4012BDF814004901A0F2BC7042EAFB
:10AAE00040229DF81A0041EA50019DF8180092B2E8
:10AAF00041EAC02188B2D9811A821A83D8820323FD
:10AB000057E720466EF0D8FC2369002B00F08780C1
:10AB1000237E03F0F70213F00403227640F09480C2
:10AB2000122A00F0AA800022E36A204684F8282036
:10AB300008B0BDE8F0471847DDF80C80B8F1000F09
:10AB400000F0BB8098F80030002B00F0B68098F839
:10AB50000BA01AF0080F7FF4EEAE0B2204F13101C6
:10AB600040467CF0DFFB00287FF4E5AE637E8AEA96
:10AB70000303DF0640F1E18095F93A325E1C0AD00A
:10AB800005EB0313FF2193F88F2085F83A1260F349
:10AB9000000283F88F2095F93B22511C3FF400AF4F
:10ABA000023205EB021393F86F30C3F34503012B18
:10ABB00040F20681013B03F03F0305EB021292F8DD
:10ABC0006F1063F34601FF2382F86F1085F83B3264
:10ABD000E6E695F820320922022B3FF4E1AE95F823
:10ABE0004832002B7FF4DCAE85F85832404685F8B9
:10ABF000543285F84822C5E99733D5F83432C5F880
:10AC00004C32D5F87C32C5F85032FFF7EDFC012804
:10AC10003FF4E3AE02287FF485AE0423C9E6237E29
:10AC20001B0780D5054B93F80022002A7FF47AAEEB
:10AC3000072283F8002276E70022A6E620460024B9
:10AC400040480024A04600240023A5682046E66A68
:10AC5000294684F82830FFF71DFC002863D194F8BA
:10AC60002830002B7FF45EAE0223C4E90B6584F824
:10AC7000283057E644F281723EE7E06A0421626AB6
:10AC8000A063204684F83C3084F828106363636234
:10AC9000C4E90B22C4E9023308B0BDE8F0476EF006
:10ACA0000BBC95F81C2212B9012285F81C22012246
:10ACB0006FF00F0185F86520ABE695F93A32591C23
:10ACC0000AD005EB0313FF2193F88F2085F83A1281
:10ACD00022F0010283F88F2095F93B325A1C16D0DE
:10ACE000023305EB031292F86F20C2F34502012AEA
:10ACF00021D9013A02F03F0205EB031393F86F10DC
:10AD000062F34601FF2283F86F1085F83B22237E11
:10AD1000DB067FF545AE2C486EF0CEFB4FF6FF729A
:10AD20000223228445E6002E3FF4FCAD2046334644
:10AD300045E600219FE60022DEE7B8F81420B8F8C7
:10AD40001A3043EA0243D5F8782263625202D8F8F7
:10AD50001C30B3FBF2F102FB1131A36009B11344C3
:10AD60005B1AE36084F819A095F93A325A1C0AD0AC
:10AD700005EB0313FF2193F88F2085F83A1222F098
:10AD8000010283F88F2095F93B22531C3FF4B7AEA4
:10AD9000023205EB021393F86F30C3F34503012B26
:10ADA00010D9013B03F03F0305EB021292F86F103C
:10ADB00063F34601FF2382F86F1085F83B329EE66D
:10ADC0000023FAE60023EFE74048002410B503789B
:10ADD000044690F818C0023B012B02D91CF0060F64
:10ADE0006ED11CF0200F44D194F91A20511C0AD0C6
:10ADF0003A4BFF2103EB021393F88F2022F001025C
:10AE000083F88F20A17694F91B305A1C16D0334951
:10AE1000023301EB031292F86F20C2F34502012ABC
:10AE20004BD9013A02F03F0201EB031393F86F1084
:10AE300062F34601FF2283F86F10E2761CF0080FE0
:10AE40000ED0264991F80032072B06D091F81C321B
:10AE5000002B3DD0012381F86530002381F80032BA
:10AE60000023E26A237084F8283042B3BDE8104022
:10AE700010471B4A0023E069D1691032884206D08E
:10AE80000133082BB0D0D16910328842F8D1134970
:10AE9000023301EB031292F86F20C2F34502012A3C
:10AEA0001AD9013A02F03F0201EB031393F86F1035
:10AEB00062F3460183F86F1096E70022B4E710BDF5
:10AEC0000121FFF74DF90128F9D194F818C088E75E
:10AED000012381F81C32BDE70022E5E7204600246B
:10AEE0008446002438B51A4C94F848322BB970B116
:10AEF00090F828201AB1184638BD002038BD014608
:10AF0000442204F508707CF0ABF8012038BD04F54C
:10AF100008750146442228467CF0C0F994F8643054
:10AF200003224FF6FF71022B2846A4F83A1218BFED
:10AF30001346D4F8841284F83822102284F8203280
:10AF4000C4F8441284F839226EF0B6FADDE700BF87
:10AF500020460024314A4FF0FF31F8B5A2F1640CCD
:10AF600000230C4603E001331032082B14D092F872
:10AF70002A000428F7D10CEB031090F88F00C607C5
:10AF8000F1D4651C106A01D08142ECD91C46013312
:10AF900001461032082BEAD1002C01DA0120F8BD5D
:10AFA0001F4DA61C05EB0613D5F88C22B3F86C10C8
:10AFB000E1B927012F44E96FD5F88C32D7F880002A
:10AFC00001EB4421DBB1DC680023164AA047B0B195
:10AFD000022809D1D5F8043105EB06160122013B00
:10AFE00086F86E20C5F804310020F8BD05EB041387
:10AFF0002701D3F8800012B193689847DAE7D5F8B3
:10B00000043105EB061603210122013B86F86E1080
:10B0100085F80821C5F80431E6E700BF844600241E
:10B0200020460024F16604082DE9F04390F828300A
:10B0300083B00446013B082B0BD8DFE803F0383C13
:10B040001F2305290A2E33000121FFF7C7F8012825
:10B0500002D003B0BDE8F08300222378216C84F88D
:10B060002820002BF5D00322E162D4E9010384F803
:10B070002820834238BF03462046A36003B0BDE8C2
:10B08000F043A3E6002103B0BDE8F043FFF7A6B804
:10B0900003B0BDE8F043FFF79BB903B0BDE8F04350
:10B0A000FFF72AB903B0BDE8F043FFF79DBA03B03C
:10B0B000BDE8F0431CE4DFF834914368D9F88062BE
:10B0C000026B19461E40D9F8780294F800C0B518F2
:10B0D0004702B5EB402F41D34FF6F778BCF1020F92
:10B0E00014D025692846002D5AD16168A368002034
:10B0F000E26A8B4284F8280038BF0B46A360002A1E
:10B10000A7D0204603B0BDE8F04310476168D9F8E6
:10B110008802B1EB402F5CD22069217E090732D52D
:10B12000D9F8FC11451CA9422AD299F81C12002911
:10B1300043D1012389F81C3289F86530226B63689A
:10B1400094F800C0D21B3B4432449B1B002697421C
:10B15000194663602263C4E90450BFD9BCF1020FF1
:10B1600037D02569002DC1D099F86430032B36D033
:10B17000ADB24FF6F7739D42B8D811446160B5E7A0
:10B18000E0D10025DEE701A96CF092FE01287FF4F2
:10B1900060AF2069019D94F800C06368226BD1E71D
:10B1A00099F8641003290ED0A9B2414594BF00213B
:10B1B00001210029B1D06168D4E7012189F8651027
:10B1C00094F800C0BEE708498D4294BF00210121D8
:10B1D000EFE7D9F88832B1EB432FCED386E7024BA5
:10B1E0009D4283D8C9E700BFF7FFFF0F2046002428
:10B1F000704700BF007970470079C0F34010704776
:10B2000000794009704700BF704700BF704700BF1A
:10B2100003685A1C02601970704700BF03685A1C0B
:10B2200002601970704700BF024B186803681B6802
:10B23000184700BF006500242DE9F0413A4E3378ED
:10B240007E2B03D000273846BDE8F08108214FF45B
:10B25000FC4341F221041AB25B00002A84EA420056
:10B260009BB2B8BF83B20139F5D1B6F80140002CCA
:10B2700037D02E4A2E4DAA42E4D2052CA2F1060266
:10B280008CBF002701271444AC4228BF47F00107B8
:10B29000002F46D141F2210EA24214D0501E04F1DB
:10B2A000FF3810F8011F082283EA012319B25B005E
:10B2B00000298EEA410C9BB2B8BF1FFA8CF3013A09
:10B2C000F4D14045EDD1218861B1A21DAA42BAD284
:10B2D000052904EB01002246B5D9A842B3D20446A1
:10B2E000DAE7144C671E41F22105BC4617F8012F1E
:10B2F00083EA0223082219B25B00002985EA410093
:10B300009BB2B8BF83B2013AF5D16445EDD16788ED
:10B31000094AFF1A231DB7FA87F79B1B7F09938001
:10B3200091E70F468FE700BF000002080700020800
:10B3300000000408010002080065002490F83C2089
:10B34000034602F0FF0012B1002283F83C20704750
:10B350004FF48053838170474FF4006383817047BB
:10B360004FF40063838170474FF40063838170471B
:10B370004FF4006383817047074B10B403F1100151
:10B38000002453F8042B824208BF43F8044C8B423C
:10B39000F7D15DF8044B70470865002470B5374C51
:10B3A000E08C238BB4F930501B1AA08CB4F91EC06A
:10B3B00000FB03F3B4F92E00E66B05EBE335C002A6
:10B3C00090FBF5F000EBE330B4F92A30A0F57A6E8B
:10B3D00060630EFB0EF50EFB0CFC2D134FEAEC2CFC
:10B3E00005FB03F30CEBE32CB4F9283005FB03F366
:10B3F000B4F920501B140EFB05F503EB6533B4F9CB
:10B400001C5002330CEB850CB4F938509B10648C43
:10B410000CFA05FC03F500430CF1020C04FB03F3EA
:10B420004CF25034A6EBAC0C2C41DB0B04FB0CF4BF
:10B43000002C1EDB6400B4FBF3F389B11C1240F650
:10B44000DE3504FB04F405FB04F40D4D241403FB6A
:10B4500005F504EB254404F6CF6403EB24130B60DD
:10B460002AB100EB8000400008300011106001207C
:10B4700070BDB4FBF3F35B00DFE700BF00650024A1
:10B4800043E3FFFF01207047012070472DE9F04F93
:10B49000734D85B00F46286CB5F844300092C3EB6D
:10B4A0002014B5F948205B00B5F950E004FB04F422
:10B4B000B5F84A80C3EBE003CDF80CE02413B5F9EE
:10B4C0005260B5F9541002FB04F4B5F94620029617
:10B4D00002FB03F3A413B5F94C2004EBE3242B6E19
:10B4E000A4F5FA300193B5F94E3080FB00EA4FEA3B
:10B4F000E37B82FB002C03FB0AF94FEA0C3CEC6572
:10B500000EFB0B99A3FB0E3B4CEA125C1203CB44DF
:10B510001B0A43EA0B639B184CEB2B2BA3FB083253
:10B520000BF5004B08FB0B2B4FEAEB734FEA6B0953
:10B5300053EA6B0B00F09280029E01FB0AFA019A1B
:10B5400086FB0008039EC2F5801C4A464FEA484825
:10B550004FEAE17948EAD0380EFB09A94004A1FB83
:10B560000E1E4118F1444FF000000CF0004E49EB64
:10B5700008094EEA5C0E41184FEACC7C09EBC6097B
:10B58000BCEB010C6EEB090E1CEB0C084EEB0E0134
:10B5900018EB0C084EEB01014FEA88104FEA8119B5
:10B5A00018EB000049EA986941EB0901890041EA7A
:10B5B0009071800010EB0C004EEB0101890041EA14
:10B5C0009071800010EB0C004EEB010177F06EF9EA
:10B5D000B5F95A304FEA613884464FEA503EB5F922
:10B5E00056204FEAE37A03FB08F94EEAC14EB5F95B
:10B5F00058000EFB0A99A3FB0E35A94403FB08F57E
:10B600000EFB0955A3FB0E3E75445B0E4FEAE07E30
:10B6100043EAC51313EB0C0341EB656500FB01F135
:10B620000EFB0C11A0FB0C0C6144C00C40EA413035
:10B630001B1845EBE1451B0A43EA056303EB0213C4
:10B640000FB11B0A3B60009B23B104EB84048034E0
:10B6500024121C60012005B0BDE8F08F0023EFE745
:10B660000065002431B10A4BD3ED207AFDEEE77A74
:10B67000C1ED007A52B1064B9FED067AD3ED217AE7
:10B6800067EE877AFDEEE77AC2ED007A0120704717
:10B69000006500240000C8422DE9F04F5F4D93463D
:10B6A00085B0B5F89630D5F888001B02B5F894E05F
:10B6B000B5F89240C21AB5F89030019167EB0707D0
:10B6C000AEFB020C1B04B5F88E100EFB07CCC009B4
:10B6D000B5F89860C90340EA4C604FEAEC1CC0180A
:10B6E000A4FB023E04FB07EE4FEA13234CF1000CCF
:10B6F00043EA0E634FEA2E2E5B18A6FB021406FBEC
:10B7000007444FEAD1514EF1000E41EA4421E415BD
:10B7100011F5FA6844F10006B8F5FA6F029676F171
:10B72000000630DA01FB04F60394A1FB014A0AEBA0
:10B73000460AA6004FEA8A09361949EA9479384C34
:10B740004AEB09094FEA560AB6084AEAC97A46EAB4
:10B750008976B0EB0A0A6CEB690C9E1B50466EEBC7
:10B76000A90E3346A045029E4FF0FF34A64126DBCA
:10B7700002FB07F7A2FB022101EB4701D20F42EACD
:10B780004102B8EB0208019C84B1D5F89C10A1FBE2
:10B79000033201FB0E225B0D43EAC22352151B1A32
:10B7A00062EB0C02DB0B43EA42432360BBF1000F68
:10B7B00001D0CBF80080012005B0BDE8F08F40F645
:10B7C000AC56039C891944F1000401FB04F4A1FB6D
:10B7D000016101EB4401F4004FEAC109341B49EA5D
:10B7E000567961EB090924184CEB090C2046B41971
:10B7F00041EB0109A41941EB09094FEA890949EA1A
:10B800009479A400A41B69EB0109610841EAC9719C
:10B81000591A6EEB690E0B46AAE700BF00650024BB
:10B8200024FAFFFF01207047104B10B4104C1B6826
:10B83000D4F8A0001B1AFA2B0BD811B1D4F8AC30F5
:10B840000B6012B1D4F8B030136001205DF8044BE6
:10B850007047D4F8A430002223F00403104684F883
:10B86000A820C4F8A4305DF8044B7047742F00245E
:10B87000006500242DE9F8430D46D0E9003113445A
:10B880008B4220D80446AE18076BCAB14FF00009AE
:10B8900000F10C0801E0AE4212D0E36A5A1C2344C6
:10B8A000E262202A15F8011B1973F4D141462046A3
:10B8B00017B9F7F729FC0746AE42C4E90B97ECD15C
:10B8C0003846BDE8F8834FF0FF37F9E72DE9F04F30
:10B8D0005422044600218BB09F487BF0DFFC9F4A36
:10B8E000611EE01C144611F8013F5D1E052D88BF46
:10B8F0000023884244F8043BF5D102F110031146BD
:10B9000051F8040B012800F019818B42F8D111463F
:10B9100051F8040B022800F007818B42F8D1114640
:10B9200051F8040B032800F0F5808B42F8D152F84F
:10B93000041B042900F0E4809342F8D105204FF065
:10B940001A094FF0000ADFF81082854DFFF714FD49
:10B95000844F0620FFF710FD98F80C407CB320467A
:10B9600098F90D6007F0FEF828B1052380F80790DC
:10B97000837100230372032107F0B0F8002302E073
:10B9800001331C2B3DD015F83320A242F8D105EB32
:10B99000C3035868F42106230122C8F8100001FBF4
:10B9A000067688F816309244D6F8F03088F81520DC
:10B9B00086F8EC209A1888F81430C6F8F02009F1BF
:10B9C000010908F10C085FFA89F9B9F1200FC3D118
:10B9D000BAF1000F12D0DFF88CA14FF0000BDFF8A6
:10B9E0009C81D14699F8EC306BB90BF1010B09F150
:10B9F000F40908F58C78BBF1030FF3D10BB0BDE867
:10BA0000F08F0020C6E7B9F806006CF0ABFAB9F881
:10BA100004006CF0A7FAD9F8F0304FF4403CF42160
:10BA2000012BC9F8283001FB0BA1D9F80020D4BFA5
:10BA3000002301234FF0030EC9F81020C9F81C3071
:10BA40000023C9F8383089F82C30C9F83030C9F8EB
:10BA5000203089F8483004930823C9E905C34FF41E
:10BA60008063C9F834304FF48073A9F824304FF460
:10BA70008053C9E90FE34B6E002B69D093689F0098
:10BA800003D59168384B0B4093609368DE0014D463
:10BA9000364B37491B689068B3FBF1F335490133E6
:10BAA000014041F0805191600493049B2BB1049BB1
:10BAB000013B0493049B002BF9D19368DD001CD457
:10BAC000F423012103FB0BA30191596E41F01001F6
:10BAD0005966996E41F001019966F423916803FB60
:10BAE0000BA301F00401586E00F01000014347D091
:10BAF0005A6E42F010025A6677E700230193ECE792
:10BB00001D4B342193F8082183F8E410013283F8A7
:10BB1000082113E71849352491F8080181F8D84025
:10BB2000013081F8080102E71349312491F8080136
:10BB300081F8CC40013081F80801F0E60E4930244C
:10BB400091F8080181F8C040013081F80801DEE673
:10BB50008B6689F8603091E7B4650024086500249D
:10BB600090790C08D0170024C0FFFF5F000000246C
:10BB7000400D0300C0FFFF6F00650024000000308F
:10BB8000596E21F4817141F0020159669368DC0716
:10BB900013D4784B9A4200F0178303F580739A42CE
:10BBA00000F01283744B9B68D90706D473498B68E5
:10BBB00023F47C1343F440338B60714B71491B6851
:10BBC000D368194043F208030B43D360916893682C
:10BBD00001F0040103F00803194300F06182D9F871
:10BBE0001000D9F81C30012B00F05583036B23F0B3
:10BBF0000F030363F42303FB0BA35A6E22F003022B
:10BC000042F001025A66019A002A7FF4EEAE019AD0
:10BC1000059299F86020012A3FF4E7AE826801217D
:10BC2000940789F86010816802D4CA0700F18882FD
:10BC3000F421554A554B01FB0BA14C6E224042F0BA
:10BC400002024A668268134043F0004383608368BF
:10BC50004F4A002BC0F2E581F4214E4B4E4C4FF47D
:10BC6000806C01FB0BA14D4803274D4D4A6E22F01D
:10BC7000030242F001024A66D9F80820D9F80C60A4
:10BC8000A24218BF9A424FF40054C9F878600CBF22
:10BC900001230023C9F89C70824208BF43F00103CE
:10BCA0001830824208BF43F001031830824208BFB7
:10BCB00043F001031830824208BF43F001031830FB
:10BCC000824208BF43F001031830824208BF43F0AC
:10BCD000010300F55670824208BF43F0010318309B
:10BCE000824208BF43F001031830824208BF43F08C
:10BCF00001031830824208BF43F00103183082422A
:10BD000008BF43F001031830824208BF43F001032B
:10BD10001830824208BF43F00103002089F8600018
:10BD2000C9F89800C9E91F00C9E928004FF400606C
:10BD3000C9E921C04FF48070C9E923404FF40030B5
:10BD40004C46C9F89400286844F8742F1BB9154B69
:10BD50009A4240F0BE84F423022103FB0BA383F834
:10BD6000A9100021136889F8A81023F001031360BB
:10BD70001FE000BF0020024000600258006302582C
:10BD80000010005C03C0F0FFFDEEFFFFC0FFFE3FB0
:10BD900000F8C32510000240280002404000024085
:10BDA000802C0024B80402402B681B1A052B00F2DB
:10BDB000BD811368DF07F7D4A44913680868A44954
:10BDC0006FF30F001940A34BB0F1005F43EA01038A
:10BDD0000BD32E2E40F21F833F3E132E05D89E48D4
:10BDE000F040C00701D59D4B0B43136020465369BB
:10BDF00023F007035361F5F73FFED9F8D02002F096
:10BE00001F013F228A408260D9F87420944B9549E3
:10BE1000954E8A4218BF9A4201F11801A2EB060022
:10BE20000CBF012300238A4208BF43F001031831ED
:10BE30008A4208BF43F0010318318A4208BF43F029
:10BE4000010318318A4208BF43F0010318318A42C6
:10BE500008BF43F0010318318A4208BF43F00103D1
:10BE600001F556718A4208BF43F0010318318A4236
:10BE700008BF43F0010318318A4208BF43F00103B1
:10BE800018318A4208BF43F0010318318A4208BFC3
:10BE900043F0010318318A4208BF43F0010318310F
:10BEA0008A4208BF43F001037049511AD1F1000CD6
:10BEB0004CEB010C6E498A4208BF43F001036D4907
:10BEC0004642A2EB010701F1140146414CEA03038B
:10BED000D7F1000EA2EB010043EA06034EEB070E7A
:10BEE00041424EEA0303414163480B4302916349D7
:10BEF000571A794279410B430391111A484248413C
:10BF00005F49571A0343794279415E4FBA4214BFE1
:10BF1000002701270B4301D1002F3BD046EA0C0636
:10BF2000029B4EEA060E039E43EA0E031E43D3B263
:10BF300030430143394300F05D831422083B01265E
:10BF4000514FB3FBF2F3514A9E401A449200D9F884
:10BF50007C30C9F8DC60802BC9E9352700F0088106
:10BF6000D9F87830D8B2013B072B10607E6000F220
:10BF70000481461E002900F06885454B454903446D
:10BF80009B0001220020B240C9E93831C9F8E820FD
:10BF900018604A60F423012100204FFA8BFE03FB56
:10BFA0000BA30A460295C3F8C80083F8A91009F14B
:10BFB0001003C9F85C40C9F8AC30374B04E00132DB
:10BFC0000C33072A00F00A81597D0029F7D093F934
:10BFD0000D107145F3D1002101989D7D06912F49E7
:10BFE000039501EB80011869D1F8E04099F86010E1
:10BFF00001293FF4FAAC4FF0010189F86010D9F83B
:10C0000010108D686F0740F10F81F42303FB0BA321
:10C010005A6E42F020025A664FF0000389F86030F1
:10C02000E3E4059B01330593059B9342FFF40FAEB8
:10C03000F422002102FB0BA2536E23F0120343F003
:10C040001003536689F86010CFE400BF0010005C55
:10C050003F8010FE002D02000F030F00002D120084
:10C0600010000240280002401C5402580854025894
:10C07000B8040240305402586C54025858540258C4
:10C080008054025894540258805802580096001662
:10C090003F96001640590258B465002490790C0868
:10C0A000D068AA4B0340D9F8440043F00303D3609F
:10C0B000136923F001031361136923F070430343F1
:10C0C0001361A34B9A4277D003F580739A4273D0E1
:10C0D000A04B9B6813F4403F14BF01230023002BA7
:10C0E00000F0EA80F5F730FED9F814300146B3F5D8
:10C0F000003F00F01E82B3F5403F00F01E82B3F512
:10C10000803F00F01682944BD9F810001A6841F273
:10C110000303B3EB124FC0F0C780904B9942836882
:10C1200000F20F8123F4807383605AE5F423202208
:10C1300003FB0BA3C3F8C820032283F8A92054E40F
:10C14000826802F00D02012A1DD05A6E002142F0D1
:10C1500010025A669A6E42F001029A66F42303FBBB
:10C160000BA35A6E42F010025A6689F860103CE444
:10C170000023C9F8783013607E600023C9E93833A2
:10C18000C9F8E83006E78268754B764D134043F0F6
:10C1900002038360032303602A688368DE077FF558
:10C1A00047AD2B689B1A022BF7D98368DF07F4D5BC
:10C1B000F42303FB0BA3C8E76B4B9B6813F4403FCE
:10C1C00014BF012300238AE7614B68499B68896893
:10C1D0000B43D8073FF5F1AC6349E8E4D9F81010F8
:10C1E0005B4B029D9942D9F8F07052D003F58073F1
:10C1F00099424ED0574882688B685E073FF5F5AB91
:10C2000099F86030012B3FF4F0AB02F01F0240F2CE
:10C2100021230124D34089F86040234040F0FF806F
:10C2200089F86030FFF7E1BB00284FEA906709DB2F
:10C23000C0F31305002D40F0E6800125BD40CE6916
:10C240002E43CE61A50901F1300604F01F0407F06A
:10C250001F0705F00C054FF01F0CA7400CFA04FC5B
:10C26000745924EA0C043C4374518D688C6805F0C1
:10C27000040504F008042C4300F082808C68E60773
:10C2800032D501990131C9B20191002189F86010BC
:10C2900095E63548AFE7026BD9F8283022F00F0257
:10C2A000013B13430363A5E4314B994242D88368B1
:10C2B00023F44073836094E42E4B9A6D02F4403271
:10C2C000B2F5803F00F08881B2F5003F00F069814F
:10C2D000002A7FF418AF1B681A017FF514AF07A876
:10C2E000F5F770FD07990EE7D1F8C040C0F31305CC
:10C2F000002824EA0504C1F8C040C2DA144CA14267
:10C3000000F01D8104F58074A14200F01881114CE9
:10C31000194EA568B668F60740F11B81F423002189
:10C3200003FB0BA35A6E42F020025A6689F8601094
:10C33000FFF75BBB114B994200F22881836823F41D
:10C34000407343F4807383604BE400BFFCBFFFFF86
:10C3500000200240006302580010005C002D3101F3
:10C36000C0FFFF7F802C00240023024000210240F8
:10C3700021BCBE00004402580060025841787D0193
:10C38000C0F30454039FC50D01F1140607FA04FC21
:10C39000072705F00405A740745924EA070444EA76
:10C3A0000C0474519F4C246804F07044B4F1805F15
:10C3B000CC6800D0CC680C6E850604F0F844B4EB71
:10C3C000806F03D10C6E24F000440C664C6E04F0B8
:10C3D000F844A54203D14C6E24F000444C668C6EA8
:10C3E00004F0F844A54203D18C6E24F000448C661E
:10C3F000CC6E04F0F844A5427FF440AFCC6E24F03C
:10C400000044CC663AE790FAA0F50126B5FA85F526
:10C4100006FA05F513E7282E7FF6E7ACE3E48B6810
:10C42000DC0733D48C68804B1C421FD18C687F4B57
:10C43000234043F001038B602C688368DB0602D045
:10C440007B4B994222D079480B68DE071ED48B685B
:10C45000DE0704D48B68034043F001038B602B6834
:10C460001B1B022BF0D90B68DB07EDD4F42303FB75
:10C470000BA35A6E42F010025A669A6E42F0010205
:10C480009A66002389F86030FFF7AFBAF420694B51
:10C4900000FB0BA0446E234043F48073436612B14B
:10C4A000634B994206D0F42303FB0BA35A6E22F48C
:10C4B00080125A66F42303FB0BA35A6E12F48052C7
:10C4C00000F0A8809A6E22F006029A66D9F85C0005
:10C4D0000024594BD9F83C20C363584B0364584B94
:10C4E000C3641C230B604B6889F8604043F0100361
:10C4F0004B60CB6823F003031343CB6090F83430D8
:10C50000012B0CD0012380F8343090F83530012B0A
:10C5100000F02C814FF4006380F834404365D9F873
:10C520001020424B91680B4043F004039360FFF7E7
:10C530005CBA1B0CB1FBF3F1E5E58108E3E5414C86
:10C54000414E3B4FA568B668BF683E43F7073FF5CD
:10C55000E5AE3E4F05F0E076B84200F08D803C4FEE
:10C56000B84200F0A7803B4FB8427FF48AAE6F021A
:10C570003FF587AE384881427FF483AEA16821F051
:10C58000E071314341F48001A1607AE6334B994276
:10C5900083682AD823F4407343F400738360FFF761
:10C5A00020BBDA6C186802F04052470701D5002A18
:10C5B00032D02B4B1B68DE0503D5B2F1805F00F053
:10C5C000D380274B1B689D037FF59DAD254BB2F1B2
:10C5D000005F08BF194696E51B689B007FF593AD89
:10C5E00007A8F5F789FC09998DE543F4407383604A
:10C5F000FFF7F7BA1C48103B10441822A828B3FBD9
:10C60000F2F300D80833194A0126194F1A449E4004
:10C6100092009CE49A6659E71B681649C3F3C1036C
:10C62000D94070E50010005C3F000080C0FFFF7F34
:10C6300000210240FEF0FFFF01000408550004083D
:10C64000590004080023024000200240000084CB6F
:10C65000000052C70000B8CF0060025881F0FA0213
:10C660000044025840787D01F0FBFDBF00820010BD
:10C67000800802400090D0032D023FF502AE9F4893
:10C6800081427FF4FEAD9E499E480968B1FBF0F1FE
:10C69000A068013120F0E0704900304340F4000010
:10C6A000A060069102E006990139069106990029D9
:10C6B000F9D1E6E5E8013FF5E4AD904881427FF429
:10C6C000E0ADA16821F0E071314341F08071A160DB
:10C6D000D7E58D4B8D48824218BF9A4200F1140075
:10C6E0000CBF01230023824208BF43F00103143032
:10C6F000824208BF43F001031430824208BF43F076
:10C7000001031430824208BF43F001031430824217
:10C7100008BF43F001031BB97D4B9A4240F09B8157
:10C72000F42102207B4B01FB0BA1134481F8A900EB
:10C730001421B3FBF1F38340106842F2A0516FF370
:10C7400010100143002089F8A80020461160C9F8A4
:10C75000D030F5F791F9D9F8D02002F01F0101226D
:10C760008A404260FFF750BB6B49CCE4036840311C
:10C770006A4A6B4DAB4218BF934205F118050CBFD6
:10C7800001220022AB4208BF42F001021835AB4241
:10C7900008BF42F001021835AB4208BF42F0010267
:10C7A0001835AB4208BF42F0010205F55675AB42A1
:10C7B00008BF42F001021835AB4208BF42F0010247
:10C7C0001835AB4208BF42F001021835AB4208BF32
:10C7D00042F001021835AB4208BF42F001021835A1
:10C7E000AB4208BF42F001021835AB4208BF42F02D
:10C7F00001021835AB4208BF42F00102142505FBC7
:10C8000007F7022580F83550464D4465464CAB424B
:10C8100018BFA342856D0CBF0124002401950AB9FD
:10C82000002C37D01D6825F00105D0E919EC1D60FA
:10C83000C56E002C40F0FF80456EC5F804C0C56E83
:10C84000002D75D0D0E91C566E60002C70D0C56DDF
:10C85000019E05F01F0C3F2505FA0CF5B5601D681B
:10C8600025F480251D6085685F60402D00F0DF8025
:10C870009960C3F80C8014B9002A00F095801968FB
:10C8800021F01E0141F016011960196841F00801FC
:10C890001960B9E01C4DDFF874C0634518BFAB42A6
:10C8A0000CF1140C0CBF01250025634508BF45F0B1
:10C8B00001050CF1140C634508BF45F001050CF1AE
:10C8C000140C634508BF45F001050CF1140C6345D9
:10C8D00008BF45F00105D3F800C02CF0010CC3F8E7
:10C8E00000C0DFF848C0634508BF45F0010515B931
:10C8F000074DAB4258D1D0F868C09DE700600258A0
:10C9000000000024400D0300085402581C54025833
:10C9100094540258F8ABFDA700093D0040000240C6
:10C920005800024028000240100002408054025883
:10C93000002A8CD14B4DDFF834C1634518BFAB42A0
:10C940000CF1140C0CBF01250025634508BF45F010
:10C9500001050CF1140C634508BF45F001050CF10D
:10C96000140C634508BF45F001050CF1140C634538
:10C9700008BF45F001050CF1140C634508BF45F0F4
:10C98000010515B9384DAB420ED1C56D019E05F0BC
:10C990001F0C012505FA0CF5756085685F60402D58
:10C9A0004FD09960C3F80C8030492E4DAB4218BF70
:10C9B0008B4205F128050CBF01210021AB4208BFC5
:10C9C00041F001011D6825F00E0545F00A051D60C6
:10C9D000274DAB4208BF41F001011435AB4208BFFF
:10C9E00041F001011435AB4208BF41F001011D685F
:10C9F00045F004051D601F4DAB4208BF41F0010129
:10CA000011B919498B420DD1016E0D68EA0303D5A6
:10CA10000D6845F480750D60C16E19B1086840F469
:10CA2000807008601A6842F001021A6077E5C3F866
:10CA30000880D9601FE7CEF804C0002D7FF402AF54
:10CA400005E7C3F80880D960AEE70B4B0B490344F8
:10CA50009B00FFF796BA4023C1F8C83081F8A9704F
:10CA6000FEF7C3BF08540258945402581C5402588D
:10CA700044540258805402583F820010400902403A
:10CA800038B51446002944D0344B0D469FED344A46
:10CA900093ED437AD3ED466AB8EEC76AB3F928211D
:10CAA000B8EEE60AD3ED447A04EE902AB3F92421D5
:10CAB000C6EE046A93ED477A05EE902AB3F9262173
:10CAC00005EE102AB3F92221B3F92031F8EEE44A39
:10CAD00006EE102AF8EEE55AF8EEE77AB8EEC55AF7
:10CAE000B8EEC77AC7EE843A07EE903AB8EEC66A57
:10CAF000E6EEA45AF8EEE77AA6EE856AA6EEA57AE7
:10CB0000E6EE867AA6EE870AA3EEA70A78F01CFA6C
:10CB100028600CB3114BF6EE005A9FED115AD3ED7D
:10CB2000446AB3F91621F8EEE66AB3F9143107EE58
:10CB3000102A9FED0C6A07EE903A86EE850AB8EE51
:10CB4000C77AF8EEE77A20EE070AA7EEA50A20EEEC
:10CB5000060A78F0F9F92060012038BD006500244C
:10CB60000000F04A0000C8420369416853EA01022C
:10CB7000F0B43B4E5DD0C56A013390ED067A6A1C75
:10CB8000876830EE077A0361012AC26280ED067A77
:10CB900042D090ED075A07EE902AD0ED096A70EE68
:10CBA000455A3468B8EEE76A611AC5EE867AB9422A
:10CBB00077EE857A30EE670AC0ED087AC0ED077A25
:10CBC000F0EE667AE5EE807AC0ED0A7AC0ED097A79
:10CBD00001D8F0BC7047012A28DD06EE905AF8EE25
:10CBE000E66A87EEA66AB5EEC06AF1EE10FA1DDBC2
:10CBF000F1EEC67AF4EE677AF1EE10FA16D6D0EDC1
:10CC0000056AF4EEE76AF1EE10FA15D5037BFBB185
:10CC10000323F0BC03707047326880ED080A521A93
:10CC2000002180ED070ABA424162D2D9DFED0D7AC8
:10CC3000E5E7316841609EE707EE903A0223F8EE9F
:10CC4000677A0370F0BCC7EE276AC0ED066A7047CA
:10CC5000316800220361C36241608261B9E700BFAD
:10CC6000742F00240000000010B5DFED4F4A844609
:10CC700000F1480E0346DA6AB1EC017AD3ED067A88
:10CC8000013277EE877A012ADA62C3ED067A71D033
:10CC900093ED075A07EE902A93ED096A77EE455A0D
:10CCA000F8EEE77AC5EEA76A76EE857AF0EE466A88
:10CCB00037EE677AC3ED087AE5EE876AC3ED0A6A54
:10CCC000C3ED077A1833C3ED036A7345D3D1374CEC
:10CCD000416822680369521A816801338A420361FC
:10CCE00047D990ED056A0022DFED2F5ADCF82C10B1
:10CCF000F0EE657ADCED0A6A012901F1FF3E11DDF3
:10CD000007EE90EAF8EEE77A86EEA77AB5EEC07AFB
:10CD1000F1EE10FA45DBF1EEC77AF4EE677AF1EE48
:10CD200010FA3ED6B4EEE76A01320CF1180CF1EEBF
:10CD300010FA26D4022AD9DDB4EEE76AF1EE10FA31
:10CD40001FD407EE903AD0ED066A90ED0C7A0223DC
:10CD5000F8EE677AD0ED125A037086EEA76AC7EE36
:10CD6000276A85EEA77A80ED066AC0ED0C6A80ED31
:10CD7000127A10BDF0EE477A83ED087AF0EE646A1D
:10CD80009EE7037B13B10323037010BD00222168CB
:10CD90000361C36241608261026343648264C3656C
:10CDA00010BDDFED017ABDE700000000742F002404
:10CDB000B0EEC06AF0EEE05AF0EE407AF4EEC65AF9
:10CDC000F1EE10FA0EDCB5EE400AF1EE10FA4AD0A0
:10CDD000F4EEC65AF0EE466AF1EE10FA4FD5B0EE18
:10CDE000655A03E0F0EE656AB0EE465A85EE267AA3
:10CDF0009FED242A9FED243A9FED244ADFED244A3B
:10CE0000DFED242ADFED243AB7EE005ADFED236A86
:10CE1000F4EEC65AF1EE10FAA7EE023AE7EE223A25
:10CE2000A7EE034AA7EE235AE7EE044AE7EE246A88
:10CE3000B1EE667A87EE050A10D4F5EEC00AF1EE7F
:10CE400010FA03D59FED167A37EE400AF5EEC07A58
:10CE5000F1EE10FA48BFB1EE400A70479FED117A2B
:10CE600037EE400AE9E7F5EEC00ADFED0F7A9FEDF5
:10CE70000F0AF1EE10FA58BFB0EE670A7047B0EE35
:10CE8000465AB3E739094E3DE3B59EBE88FA16BE51
:10CE900045FE7FBF99FB243F69A2163EA7DFA8B4D9
:10CEA000DB0F4940DB0FC93FA7DFA834DA0F494049
:10CEB000D1ED007AF7EE002AD0ED043A90ED054A64
:10CEC000E7EEA73AD0ED064A90ED075AD0ED085AA2
:10CED00090ED096AD0ED0A6A90ED0B7AC0ED043A44
:10CEE00091ED003AD1ED013AD0ED0C7AA3EE234A50
:10CEF00080ED054AD1ED003A91ED024AE3EE844A15
:10CF0000C0ED064AD1ED004A35EE245A80ED075AAD
:10CF1000D1ED014A91ED005AE4EE855AC0ED085A70
:10CF2000D1ED015AA5EEA56A80ED096AD1ED015A4D
:10CF300091ED026AE5EE866AC0ED0A6AD1ED016AFA
:10CF400037EE267A80ED0B7AD1ED026A91ED007A08
:10CF5000E6EE877AC0ED0C7A91ED027AD1ED017A96
:10CF600090ED0D3AD0ED0E3AA7EE273A90ED0F4A2C
:10CF7000D0ED104A90ED115AD0ED127AD0ED135A3F
:10CF800090ED006A80ED0D3A75EEA25A91ED023AED
:10CF9000D0ED016AE3EE033A90ED027AC0ED0E3A6D
:10CFA000D1ED023A34EE234A80ED0F4A91ED004A6A
:10CFB00074EE844AC0ED104AD1ED014A35EE245A90
:10CFC00080ED115A91ED025AC0ED135A77EE857A31
:10CFD000C0ED127AD1ED017AD1ED005A67EEA77A51
:10CFE00091ED025AE5EEA57AE5EE057AA5EEA76A7F
:10CFF00080ED006A91ED016AE6EE276AC0ED016AF4
:10D00000D1ED026AA6EEA77A80ED027A90ED037A5E
:10D0100077EE277AC0ED037A704700BF2DE9F04F15
:10D020004FF00009864600F110050646034689B018
:10D0300000F13008074648462C468B469C46B246CF
:10D04000CDF80CE000283CD10CF1040CA445FBD138
:10D05000032800F1010151D09C46AA46029398B1E1
:10D06000DCED047AAAEB0903B64601927246F3ECB2
:10D07000016A0EF1100E92ED007A5345E6EEC77A82
:10D08000CCED047AF2D1019ADCED046A0CF1100CBB
:10D0900015ED047A0AF1100AC445C6EE877ACCED84
:10D0A000007ADCD1029B0436084608F104081433E8
:10D0B00014351034103709F104099C46B246002893
:10D0C000C2D0DCED007AD646394601927246F1ECC8
:10D0D000016A0EF1100E92ED007A9942E6EEC77ADF
:10D0E000CCED007AF2D10CF1040C019A0AF1040A99
:10D0F000A445E6D1032800F10101ADD1DDF80CE033
:10D100000023594604AD76467746002004930593E4
:10D1100006930793F2EC017AE5EC017AB0B104AC26
:10D120003B46B4EC017AF3EC016AE6EEC77AB3420F
:10D1300045ED017AF5D1013004280BD0F2EC017AEB
:10D1400010371436E5EC017A0028E8D11037143690
:10D150000120DFE708AD10310EF1400E042875ED17
:10D16000017AA1F10402744641ED017A1ED07346A2
:10D17000F3EC016AB1EC017AA342E6EEC77AC2EDA4
:10D18000007AF5D15EED016A013887EEA67A82ED6C
:10D19000007A17D0AEF1140E103C114675ED017AED
:10D1A0000428A1F1040241ED017AE0D15EED016AAB
:10D1B000103CAEF1140E032087EEA67A01ED017A41
:10D1C0001146EBE709B0BDE8F08F00BF60EEA00AA2
:10D1D000E0EE000AF5EEC00AF1EE10FA07DBB1EE60
:10D1E000E00AB4EE400AF1EE10FA00D670479FED67
:10D1F000010AFBE70000000060EEA00AE0EE000A72
:10D20000E1EE010AF5EEC00AF1EE10FA07DBB1EE2D
:10D21000E00AB4EE400AF1EE10FA00D670479FED36
:10D22000010AFBE700000000DFED297AB4EEE70A0F
:10D23000F1EE10FA28DD9FED277A30EE470AB4EEC2
:10D24000E70AF1EE10FAF8DCDFED237AB4EEE70A34
:10D25000F1EE10FA2FDD30EE670A37EEC00A60EE0D
:10D26000007ADFED1E5A9FED1E6ADFED1E6AA7EE03
:10D27000A56A9FED1D7A60EE275AE7EE866AA7EE53
:10D28000A67AA5EE870A7047DFED187AB4EEE70AB2
:10D29000F1EE10FAD8D59FED0F7A30EE070AB4EE12
:10D2A000E70AF1EE10FAF8D4DFED0B7AB4EEE70AF4
:10D2B000F1EE10FACFDC9FED0E7AB4EEC70AF1EE74
:10D2C00010FACCD530EE270A37EE400AC7E700BF88
:10D2D000DB0F4940DB0FC940DB0FC93F9A7C2E367C
:10D2E000FAAF4FB93587083CA4AA2ABEDB0F49C064
:10D2F000DB0FC9BF10B5404CB4FBF2F4A14219D307
:10D30000DFED3E7AF7EE005AB0EE677AB0EE676A6C
:10D31000F0EE676A0023C0ED005AC0ED017A80ED9F
:10D32000027A80ED036AC0ED046A8361436103629F
:10D33000C36110BD07EE902ADFED315AB7EE006AE7
:10D34000DFED306AB8EE677A07EE901AB0EE405A19
:10D35000F8EE677A27EE257A67EEA67AC6EE076AB8
:10D36000C7EEA64AFDEEE47A17EE902A2032402A54
:10D370003FD8B0EE640AFFF757FFB0EE404ADFED4A
:10D38000227A34EEA70AFDEEC07A17EE902A2032F8
:10D39000402A29D8FFF748FFF8EE006A60EE266AB7
:10D3A000012B1CD0B7EE006AF6EE004A36EE406A5A
:10D3B00066EE244A35EE055AF7EE007A84EE057AD9
:10D3C00077EE275A37EEC75A84EEA57AC6EE257A4D
:10D3D00086EEA56AC5EE256AF0EE475A9AE7F7EEA3
:10D3E000004AB0EE666AE5E7DFED086A9FED030AE2
:10D3F000D6E79FED024AC2E720A107000000000027
:10D40000BD378635DB0FC940DB0FC93F0000008008
:10D41000DFED077A30EE270AFDEEC07A17EE903A7C
:10D420002033402B00D8FFE69FED020A704700BF73
:10D43000DB0FC93F000000002DE9F84F9DF82840A0
:10D440008946DDF82CB00546002C17461BF8011B59
:10D450000CBF4FF020084FF030081C1E08463ADB86
:10D4600000295CD0002C53D04FF0000A5B4600E04E
:10D4700064B313F8016B013C002EF9D1BAF1000F2F
:10D480002FD1264644B14D454146284600D2B847E3
:10D49000013CF8D10B9B18780146A0B14FF0FF3446
:10D4A0004FF0000A00E09B464D45284600D2B847A1
:10D4B0005B4613F8011B0029F5D10B9BF61A5E445D
:10D4C000BAF1000F10D13046BDE8F88FBAF1000F65
:10D4D0001BD15646E0E7634229B31C464FF0010AD0
:10D4E000C4E70028E0D10646002C04F1FF3AEADD4B
:10D4F00054464D454146284600D2B847013CF8D233
:10D50000013656443046BDE8F88F30B12646CBE7A9
:10D5100026464FF0FF34B246C6E70646D3E7264616
:10D52000002CB0D1CFE76FEA040A0E46E0E700BF57
:10D530000FB430B583B00B4C06AB53F8042BD4E9D1
:10D540004B0101936DF08AFB0546206803685B6917
:10D5500098470028F9D0284603B0BDE8304004B011
:10D56000704700BF006500240EB410B583B00446B8
:10D57000084905AB01A853F8042BCDE900346DF040
:10D580006DFB0022019B1A7003B0BDE8104003B090
:10D59000704700BF1DB204080CB4F0B53D4CADF5AA
:10D5A000277DD4F83431002B6FD094F83C31994268
:10D5B0000BD90123D4F840218340134205D10DF546
:10D5C000277DBDE8F04002B07047334B4FF47A71CD
:10D5D000324A1B68A2FB030206A8920901FB123320
:10D5E0002F49FFF7C1FF06ABAC9A064603442D490D
:10D5F00001A80193ADAB00936DF030FB019B0A21B4
:10D6000000225D1C01951970019BD4F83451591CFE
:10D6100001911A70BDB12B685B6A2BB128469847FF
:10D620000028CCD0D4F834519DF818100029C6D069
:10D630000DF119042B6828461B68984714F8011B44
:10D640000029F7D1BBE7D4F83871002FB7D03044A8
:10D6500026ABFD2206A9841C1846ADF810202246F0
:10D66000CDF81250ADF8165079F0FAFC02220346BC
:10D67000044402A93846CDE9023432F04BFA0DF5E4
:10D68000277DBDE8F04002B07047D4F83831002B58
:10D690008BD194E700650024742F0024D34D6210D1
:10D6A000C4230D0811B2040838B5184C0330D4F85F
:10D6B000442102EB9003B3F5007F18D804EB8101FD
:10D6C00004F5A47520F00300C4F8443105EB82058D
:10D6D000D1F84829C3F5007310440D4A9B00C1F8E6
:10D6E000480904210020FFF757FF284638BD0021D4
:10D6F000084A00250846FFF74FFFD4F8D0392846DE
:10D7000043F00073C4F8D03938BD00BF0065002471
:10D71000D0230D08F4230D0838B505680446EB69DD
:10D72000F3B1987800B938BDB3F90A20012007EEAB
:10D73000902AF8EEE77AC4ED057AB3F90C2007EEEB
:10D74000902AF8EEE77AF1EE677AC4ED047AB3F93D
:10D750000E3007EE903AF8EEE77AC4ED067A38BD5F
:10D7600009211420FFF7A0FF0346E861D9E700BFB5
:10D7700038B505680446EB69E3B1987800B938BD5F
:10D78000B3F90420012007EE902AF8EEE77AC4ED01
:10D79000047AB3F9062007EE902AF8EEE77AC4ED92
:10D7A000057AB3F9083007EE903AF8EEE77AC4ED5F
:10D7B000067A38BD09211420FFF776FF0346E86199
:10D7C000DBE700BF38B505680446EB69E3B198783C
:10D7D00000B938BD9A880120D2BA07EE902AF8EE37
:10D7E000E77AC4ED047ADA88D2BA07EE902AF8EE26
:10D7F000E77AC4ED057A1B89DBBA07EE903AF8EEBA
:10D80000E77AC4ED067A38BD09211420FFF74CFFF2
:10D810000346E861DBE700BF38B505680C46EB69F5
:10D820007BB1987800B938BD5B890120084ADBBA22
:10D8300082FB0312DB17C3EB221303F26D13238069
:10D8400038BD09211420FFF72FFF0346E861E8E700
:10D85000797878782DE9F04103EB4306964686B057
:10D86000034602EB4606754612F9067BA3EB070C4E
:10D8700092F80080BCF1000FA3EB0804B8BFCCF114
:10D88000000C002CB8BF6442644502DA15464FFA1A
:10D8900088F70632B242E9D1688803E00EF1060E3D
:10D8A000764518D09EF800208446BA42F6D10A1A6E
:10D8B000BEF80280002AA1EB0804B8BF5242002C37
:10D8C000B8BF64429442E9DA75460EF1060E40464E
:10D8D000C4467645E6D16879CDF808C02A78049028
:10D8E000287901920390012000910321034AFFF758
:10D8F00053FE284606B0BDE8F08100BF04240D08A1
:10D9000003685A1C02601878704700BF03681A4603
:10D91000591C016012F8021B0260587841EA00208D
:10D92000704700BF02681346511C016013F802CB18
:10D930000360D31C5178036093781B0443EA0123EE
:10D94000111D43EA0C030160D07843EA0060704780
:10D9500012B370B50446864604E0981B17D114EB49
:10D960000C0C15D01EF8013BA3F14100A2EB0E0CEC
:10D97000192811F8010BA0F1410598BF203300F1DF
:10D980002006192DE9D91B1A04D10028E7D170BD52
:10D99000604670BD184670BD104670470388002170
:10D9A0001A4A30B503F0030E90F802C0184CA3F5E4
:10D9B000FA630EEB4E0E0CF1FF3C40F2B5550CEB4A
:10D9C0008E0C04EB4C044FEA930CB4F820318479AC
:10D9D00005FB0C3390F803C022444FF47A740CF129
:10D9E000FF3C634490F804C003EB43030CEBC30C0F
:10D9F00043790089CCEB0C1C03EB8C03C3EB0313C2
:10DA000002EB8302C2FB040130BD00BF80436D38CE
:10DA100090790C08F8B516461F46404D0446394625
:10DA200030464FF47A72002374F040FF3C4B0544BB
:10DA30003C4F3D4E83FB0510E9172844C1EB6011B4
:10DA400083FB0103C8170B44C0EB631087FB003C4A
:10DA5000C317C3EBAC0386FB03764FEAE37ECEEB42
:10DA6000E61EC1EB0116A5EB860CC0EB00154FEAD4
:10DA70008E0684F806C0A1EB8501617103EB4301BA
:10DA8000A0EBC10040F2B55101FB1E332071B3F58C
:10DA9000896F37DA40F2DA218B4239DCB3F5B77F90
:10DAA0002249B4BF4FF0000E4FF0010E0EEB4E00B6
:10DAB00075464FEA4E0701EBC001B1F836011C492B
:10DAC00007EB0E0C01EBCC0C0B210CF1160C01E05A
:10DAD0003CF8020D984212DD0139F9D1774413491F
:10DAE00001EBC701B1F82001012106F5FA6E0133FF
:10DAF000A17075441B1A22812580E370F8BD0131A5
:10DB0000C9B2F2E7032540F296500627AE46D6E7A3
:10DB1000022540F229400427AE46D0E780BC92C7D8
:10DB200089888888ABAAAA2A73B06D1690790C08E8
:10DB3000B07A0C0830B5304C8DB086460D46EC46B8
:10DB40001EF0030F0FCCACE80F000FCCACE80F00B9
:10DB500094E80F008CE80F000FD1284B284A03FBF4
:10DB60000EF3B2EBB30F44D3264AB2EB331F34BFEC
:10DB700001220022C2F11D0200E01C220EF1FF333F
:10DB8000019240F26D122048002B194602FB0EF262
:10DB90001E4CB8BF0EF10201EE4602EBA10280FB63
:10DBA0000310DB17ADF1040101EB8501A3EB601558
:10DBB000C3EBE0132A441A44253284FB0230D31706
:10DBC0001044C3EBA003C3EBC303D31A5EF8040FE6
:10DBD000C218714584FB023C4FEAE2739444C3EBE4
:10DBE000AC03C3EBC303A2EB0303EFD1C01A0DB028
:10DBF00030BD1D22C2E700BF107B0C08295C8FC21C
:10DC0000285C8F020AD7A3001F85EB519324499209
:10DC10000D4B10B553E9024354EA03020AD1014601
:10DC2000002340F2011218460B80C1F802208B71CC
:10DC30000B8110BD054A1268121943F10003FFF76A
:10DC4000E9FE012010BD00BFE06E0024742F002407
:10DC500030B5144D83B00446D5F8D819D5F8DC3961
:10DC600051EA03020AD1002340F201121846238030
:10DC7000C4F80220A371238103B030BD0A4A1268A0
:10DC8000521843F10003FFF7C5FEB5F8E03920460E
:10DC90000DF106022146ADF806306AF069F8012060
:10DCA00003B030BD00650024742F002488422DE9A4
:10DCB000F04198464FF0010439D301FB04F4B0FB66
:10DCC000F4FC8C45F9D264B30025BCF1000F04FBD1
:10DCD0001C00B4FBF1F7D4BF002601266DB966B96C
:10DCE000A142354619D9C6460CF1300C0EF801CBCD
:10DCF00000238EF80030BDE8F081BCF1090F18DD7B
:10DD0000002A0CBF57233723C6466344A14205F1BE
:10DD100001050EF8013BF046EAD83C46B0FBF7FCA3
:10DD2000D3E7C64600238EF80030BDE8F081844674
:10DD3000CAE73023E8E700BF2DE9F0410446154665
:10DD400008469442B4FBF2F607D205FB1644134B87
:10DD50001B5D00F8013BBDE8F0819642B6FBF2F78F
:10DD60000CD20E4B05FB176705FB1644DA5D1B5DF5
:10DD700000F8012B00F8013BBDE8F081BA42B7FB87
:10DD8000F2F807D905FB1878044B13F8082000F8BF
:10DD9000012BE7E74046FFF7CFFFF3E740240D08EC
:10DDA000B5EEC00ADFED357A0023F1EE10FA30B59A
:10DDB000C8BF30EE270A87B0D8BF30EE670ADFED64
:10DDC000307A054603A9029320EE270ACDE90033F5
:10DDD000FDEEC07A17EE904A84EAE470A0EBE4709E
:10DDE0006BF0ECF8002C03A8B4BF2D2320238DF892
:10DDF000003073F09FFF01282AD0022834D0032876
:10DE00001ED003A9684679F051FA684673F092FF74
:10DE1000044669462846033CE4B2224679F020F9DC
:10DE2000002328462B5573F085FF2E22431C0DEB53
:10DE300004012A54E81879F0D3FA284607B030BD17
:10DE4000302303A968468DF8013079F02FFADCE71A
:10DE500043F23002302303A96846ADF801208DF863
:10DE6000033079F023FAD0E743F2300303A9684680
:10DE7000ADF8013079F01AFAC7E700BF6F12033A24
:10DE800000007A440378202B03D110F8013F202BA7
:10DE9000FBD0092BF9D02D2B63D02B2BB7EE000A2A
:10DEA00008BF01300278A2F13003D9B2092961D844
:10DEB000F2EE046ADFED4D7A07EE103A10F8012F0A
:10DEC000B8EEC77AA2F13003D9B2A7EEA67A092933
:10DED000F0EE477AF0D92E2A50D0037803F0DF0312
:10DEE000452B3BD110B442782D2A73D02B2A62D017
:10DEF000A2F130030130092B63D80024002303EB87
:10DF0000830302EB430310F8012FA2F13001303BF1
:10DF10000929F4D9B3F59A7F1A46B7EE007A28BFDB
:10DF20004FF49A72072B09D91346DFED316A083B8B
:10DF300027EE267A072BFAD802F007022AB1F2EE72
:10DF4000046A013A27EE267AFBD1002C3BD0C7EEBB
:10DF5000877A5DF8044B20EE270A704720EE270AE7
:10DF6000704742780130BFEE000AA2F13003D9B207
:10DF700009299DD92E2ADFED1D7AAED143780130D3
:10DF8000A3F13002D1B20929A8D8B2EE047AF0EE9A
:10DF9000475A06EE902A10F8013FB8EEE66AA3F160
:10DFA0003002D1B2C6EE076A092927EE257A77EE4C
:10DFB000A67AEED992E782780230A2F13003092BDB
:10DFC0009BD9B7EE007A67EE877A5DF8044B20EEB6
:10DFD000270A704782780230A2F13003092B01D85A
:10DFE00001248BE7B7EE007AB1E700BF0000000024
:10DFF00020BCBE4C0378092B01D0202B05D110F892
:10E00000013F202BFBD0092BF9D02D2B09D0017813
:10E010004FF0010CA1F13002D3B2092B0AD9002034
:10E020007047417801304FF0FF3CA1F13002D3B28C
:10E03000092BF4D8002310F8011F03EB830302EB34
:10E040004303A1F13002D1B20929F4D90CFB03F04A
:10E05000704700BFB14BB24A2DE9F04F93F8E43955
:10E0600097B002EB430393F8B13113B1012005F0EF
:10E07000C5FCAC4B4FF0000AAB4A41F221051F46EC
:10E080009E1A2C2200210DEB020079F007F9A64A16
:10E09000A64B0892CDE90976DA68D10707D5A44ADC
:10E0A0005A6002F188325A60DB68DC070DD49F4B5E
:10E0B000D3F80C21D20708D59D4AC3F8042102F1F8
:10E0C0008832C3F80421D3F80C310023012205A9BA
:10E0D00008A814937E238DF854208DF81430FDF792
:10E0E000C9FB0028C0F22D8108214FF4FC4303E056
:10E0F0005B0001399BB207D01AB2002AF8DA85EA30
:10E100004202013993B2F7D18A4AADF816308A4BF0
:10E11000934280F0628198460DF11809CDE902A77B
:10E12000B8F802204FF0000CB8F80030C2F30B0B27
:10E130001004C3F30B014FEA13338DF81DC08DF8A3
:10E140001C300BF10603ADF81A10ADF8183000F1D1
:10E1500091800622494608A8FDF78CFB0028C0F2F2
:10E160000E81BDF8164049460DF11E0011F8013B25
:10E17000082284EA032403E06400013AA4B207D031
:10E1800023B2002BF8DA85EA4303013A9CB2F7D1B7
:10E190008842EBD15A46D8F8041008A8FDF76AFB6C
:10E1A0000028C0F2EC80D8F8041001EB0B0081428B
:10E1B00015D00139013811F8013F082284EA0324FF
:10E1C00003E06400013AA4B207D023B2002BF8DACE
:10E1D00085EA4303013A9CB2F7D18142EBD1ADF815
:10E1E000164008F11408534B984599D3DDE902A76E
:10E1F00000230222494608A8ADF81830FDF73AFB83
:10E200000028C0F29E80BDF816300DF11A0041F2D0
:10E21000210119F8012B082483EA022303E05B00A3
:10E22000013C9BB207D01AB2002AF8DA81EA420216
:10E23000013C93B2F7D14845EBD102220DF1160112
:10E2400008A8ADF81630FDF715FB002879DB139808
:10E25000002840F09A801498002872DB9DF8542022
:10E26000002A40F0A88000280DBF012400240123CB
:10E27000002368E0E24667460196013706224946D8
:10E2800008A8FFB28DF81D70FDF7F4FA002855DBE1
:10E29000BDF8164049460DF11E0011F8013B082259
:10E2A00084EA032403E06400013AA4B207D023B255
:10E2B000002BF8DA85EA4303013A9CB2F7D1884291
:10E2C000EBD1D8F804105A4608A801EB0A063146EB
:10E2D000FDF7D0FA002831DB06EB0B00864215D0A3
:10E2E000711E013811F8013F082284EA032403E07B
:10E2F0006400013AA4B207D023B2002BF8DA85EA11
:10E300004303013A9CB2F7D18142EBD1032FDA44A7
:10E31000ADF81640B1D1019E63E700BF006500244F
:10E3200090790C0800000408000002080020005248
:10E3300023016745C0DF0D080CDA0D08DDE9016A2D
:10E34000039F012300240AF1010ABAF1020F02DC43
:10E35000002B7FF496AE224B224A93F8E43902EB6D
:10E36000430393F8B13133B914B1FCF765FF48B9F1
:10E37000052007F09FF8002005F040FBF4E7DDE9F9
:10E3800002A7DEE717B0BDE8F08F089B099A0344A7
:10E390009342D6D80BABC0F120022146184478F046
:10E3A0007DFF149818B90BA908A8F4F7ADFE002258
:10E3B0001490139250E70C4AD16841F00101D160EA
:10E3C000D168C9077FF54FAFD2F80C1141F00101B8
:10E3D000C2F80C11D2F80C2145E70DF1180907E736
:10E3E0000065002490790C080020005270B5458823
:10E3F0000B4604460021C5F30B0518462A4678F063
:10E400004DFF0A4A21690346914206D3084A9142C8
:10E4100006D31846BDE8704008470029F9D170BD01
:10E420002A46BDE8704078F01BBE00BFC0DF0D0873
:10E43000F3E40D0810B50446C06900B110BD092110
:10E440001420FFF731F9E06110BD00BF174B03EB5B
:10E450008000806838B300EB400003EB800292F943
:10E46000B5C0BCF1FF3F1FD092F8BD00D8B103EB9F
:10E470000C00002310B590F808E18C2092F8BC1035
:10E48000142200FB0CFC0A4C0CEB0100013A714415
:10E4900034F8100013FA80F3F6D1064AA2FB0320E9
:10E4A000C0F30F1010BD70470020704700650024B6
:10E4B00000000030CDCCCCCC30B50023B0F80EE05D
:10E4C00001250EF47F4419460EF00F0EC4814A1048
:10E4D00030F81220002A18BF002511F0010F1AD0C1
:10E4E000D2B25340082213F4004F18BF83F4C05334
:10E4F000013A4FEA4303F6D101311029E7D14EEA40
:10E500000404C48155B9C3F30333B3EB0E0018BF41
:10E510004FF0FF3030BD83EA1223E3E74FF0FF30C6
:10E5200030BD00BF036810B51A790446022A03D033
:10E5300000232360237110BD987A04F013FB002898
:10E54000F6D040F61A610022C1802021027204F048
:10E55000C5FA00232360237110BD00BF2DE9F04FE1
:10E56000BA4E85B0BA4CA64256D21D4602E00C36D1
:10E57000A64251D273798B42F9D13379834201D0CB
:10E580000028F4D1F3799342F1D13468002C43D0C0
:10E59000002326606360A360E36023616361A3617D
:10E5A000E36133792371012B96F806B0C4F808B003
:10E5B000317AE16032D0022B2ED1F07A04F0D2FA17
:10E5C00096F90970A061B07A277404F0CBFA064678
:10E5D0006061F0B1DFF8948207EB47017B0058F8E7
:10E5E000319008EBC1010193B9F1000F11D0887D82
:10E5F000E8B10E2200230D213046F2713372B5715D
:10E6000004F06CFA3368B2889A61204605B0BDE820
:10E61000F08F2046FFF786FF0024F6E7F07A04F03B
:10E62000A1FA727AB37AA06122746374EDE7B1F84B
:10E6300008A0504669F096FC01214FEA5A100AF0F2
:10E640001F0A023801FA0AF1092812D8DFE810F08F
:10E65000F6001100EE0018011001E600E000D800FD
:10E66000D0000A007B4BD3F89C0020EA0101C3F8DC
:10E670009C107B00D91908EBC101487904F072FAAB
:10E68000791CCBB20146019318B1037240F60A30EF
:10E69000C8807B000291D81908EBC000C07904F053
:10E6A00061FA02990346039020B1019A027240F682
:10E6B0000A50D8807B000291D81908EBC0008079FD
:10E6C00004F050FA0299824628B1019B037240F689
:10E6D0000A40AAF806007B00D8191BF0040308EBD7
:10E6E000C0000293807A0246084614BF4E212E21B4
:10E6F00004F016FA03987B002E2103EB070B08EBBE
:10E70000CB0B9BF80B2004F00BFA50469BF80C2027
:10E710000E2104F005FA9BF804A0BAF1000F40F0B6
:10E72000ED80D9F8002022F00102C9F800204A4A01
:10E73000914500F0C180494A914540F0AC80454A7E
:10E74000D2F8901041F48041C2F89010D2F89010A5
:10E7500021F48041C2F89010029B002B40F0988079
:10E760004FF000714FF08072D9F80C0040F000407B
:10E77000C9F80C00D9F8080020F4F070C9F80800B6
:10E78000D9F80000C00727D4D9F80800344B03405B
:10E7900034481843C9F80800D9F80C00C30005D460
:10E7A000D9F8000040F48050C9F80000D9F80C00F6
:10E7B00011432D4A02400A4342F08862C9F80C20F6
:10E7C000D9F8002022F40062C9F80020D9F85020BE
:10E7D00022F00102C9F85020BAF1000F40F09B80EE
:10E7E0007B003B4408EBC308012388F8163000E7A0
:10E7F000184BD3F8880020EA0101C3F8881038E7E5
:10E80000144BD3F88C0020EA0101C3F88C1030E7D8
:10E81000104BD86F20EA0101D9672AE70D4BD3F8D6
:10E82000940020EA0101C3F8941022E7094BD3F8C1
:10E83000800020EA0101C3F880101AE7054BD3F8E5
:10E84000980020EA0101C3F8981012E7A00200081E
:10E850008C04000800440258003001400038004099
:10E86000E0FFBF8F07000020FFFF39D8AC02002473
:10E870003E4BD3F8900020EA0101C3F89010F8E66F
:10E880003A4BD3F8840020EA0101C3F88410F0E683
:10E8900000210A4668E7364A91451BD1334AD2F82F
:10E8A000901041F40041C2F89010D2F8901021F479
:10E8B0000041C2F890104FE72C4AD2F8981041F46A
:10E8C0008051C2F89810D2F8981021F48051C2F803
:10E8D000981041E7274A914527D0274A914532D1E0
:10E8E000224AD2F8981041F48011C2F89810D2F858
:10E8F000981021F48011C2F898102DE7504604F0CA
:10E9000031F920B1019B40F60A620372C2800D21E9
:10E9100004F0E4F805E7504604F024F900283FF439
:10E920005FAF0268838893615AE7104AD2F8981063
:10E9300041F40051C2F89810D2F8981021F4005117
:10E94000C2F8981008E70D4A91457FF405AF02F52B
:10E950000C32D2F89C1041F02001C2F89C10D2F881
:10E960009C1021F02001C2F89C10F5E600440258EA
:10E97000003C0040003401400050014000140058A9
:10E98000104B70B5104CA34219D2054602E00C336F
:10E99000A34214D293F805C08C45F8D193F804C073
:10E9A0000DB1AC45F3D1D8799042F0D1186890F808
:10E9B00004E0E645EBD106689E42E8D170BD002038
:10E9C00070BD00BFA00200088C0400080379022B70
:10E9D00000D0704790F9102008311C4802EB420229
:10E9E00010B41B4C83B050F8322000946944194C89
:10E9F00011F808CCA24224D017498A4223D001F54D
:10EA000080618A4205D0154B9A420CBF03234FF018
:10EA1000FF33116803EB430321F0010100EBC30056
:10EA200011600169936851F82C1023F0E0430B4307
:10EA30009360136843F00103136003B05DF8044B67
:10EA400070470023E5E70123E3E700BFAC020024A1
:10EA50000001020300300140003800400034014052
:10EA600090F91030F0B503EB4303294E154683B0FF
:10EA700056F83360044683689A0719D501230DF1CF
:10EA800006028DF8061030460DF10701F5F77CFB04
:10EA900001230DF106020DF1070130468DF80650F5
:10EAA000F5F772FBA3689B0717D5012003B0F0BDF3
:10EAB00043691BB19A88186812048261154B164A83
:10EAC000D3F8E809154BC0005768A3FB0030800954
:10EAD0005368DB1B9842FBD2D0E70E4A4FF4FA7022
:10EAE0000E4BD2F8E8290C4900FB02F24868A3FB60
:10EAF000023292094B681B1A9A42FBD26369002BBF
:10EB0000D3D01A6801209B88936103B0F0BD00BF89
:10EB1000AC02002400650024001000E0D34D621018
:10EB200010B5037984B084468E46012B0DD0022B9C
:10EB300002D0002004B010BD8368DB0758BF01F08D
:10EB40007F0104B0BDE810408AE781680DF10F0035
:10EB50001446724601F001018DF80F40CDE9000125
:10EB60009CF811109CF91000F4F7FCFD04B010BDE6
:10EB70002DE9F0410768642682B0B6227E218046E6
:10EB80003846FFF7CDFF05F0B7FF04460D4605F008
:10EB9000B3FF001B61EB0501B0F57A7F71F1000155
:10EBA000F5D3013EEFD102213846FFF70FFF7B6915
:10EBB0001BB19A88196812048A6105F09DFF04460A
:10EBC0000D4605F099FF001B61EB0501B0F57A7F5A
:10EBD00071F10001F5D37B6913B11A689B889361C9
:10EBE0000A2605F089FF04460D4605F085FF001B47
:10EBF00061EB0501B0F57A7F71F10001F5D3013EBB
:10EC0000EFD132467C213846FFF78AFF05F074FFCA
:10EC100004460D4605F070FF001B61EB0501B0F5E1
:10EC20007A7F71F10001F5D3002259213846FFF7B0
:10EC300077FF05F061FF04460D4605F05DFF001B00
:10EC400061EB0501B0F57A7F71F10001F5D397F919
:10EC500010305E218E4A03EB43038DF8071052F803
:10EC60003340BB689A0740F1E48001230DF10702AD
:10EC700000212046F5F788FA4FF4A473854A204610
:10EC80000021F5F781FABB689B0740F1E7800A266F
:10EC900005F032FF04460D4605F02EFF001B61EB28
:10ECA0000501B0F57A7F71F10001F5D3013EEFD196
:10ECB000012259213846FFF733FF05F01DFF0446B6
:10ECC0000D4605F019FF001B61EB0501B0F57A7FD9
:10ECD00071F10001F5D38C2240213846FFF720FF67
:10ECE00005F00AFF04460D4605F006FF001B61EB28
:10ECF0000501B0F57A7F71F10001F5D303224121BE
:10ED00003846FFF70DFF05F0F7FE04460D4605F007
:10ED1000F3FE001B61EB0501B0F57A7F71F1000194
:10ED2000F5D35D4C0323D8F8382098F83500B4FBB0
:10ED3000F2F291B2594AFEF78DFD43884221B4FBAD
:10ED4000F3F4C8F840400279384642F0C002FFF7B9
:10ED5000E7FE05F0D1FE04460D4605F0CDFE001B92
:10ED600061EB0501B0F57A7F71F10001F5D308225E
:10ED700043213846FFF7D4FE05F0BEFE04460D469B
:10ED800005F0BAFE001B61EB0501B0F57A7F71F169
:10ED90000001F5D3042258213846FFF7C1FE05F0E3
:10EDA000ABFE04460D4605F0A7FE001B61EB050116
:10EDB000B0F57A7F71F10001F5D30A22532138466C
:10EDC000FFF7AEFE05F098FE04460D4605F094FEF2
:10EDD000001B61EB0501B0F57A7F71F10001F5D3FD
:10EDE00000227C213846FFF79BFE05F085FE044695
:10EDF0000D4605F081FE001B61EB0501B0F57A7F41
:10EE000071F10001F5D306227D213846FFF788FE17
:10EE100005F072FE04460D4605F06EFE001B61EB28
:10EE20000501B0F57A7F71F10001F5D302B0BDE8BC
:10EE3000F0817B691BB11A689B881B049361184B96
:10EE40001849D3F8E829184BD2004868A3FB0232CE
:10EE500092094B681B1A9A42FBD206E7104A4FF4FC
:10EE6000FA70114BD2F8E8290E4900FB02F248680B
:10EE7000A3FB023292094B681B1A9A42FBD27B69B0
:10EE8000002B3FF404AF1A689B889361FFE600BF34
:10EE9000AC020024507B0C0840420F00987C0C0808
:10EEA00000650024001000E0D34D62102DE9F04110
:10EEB000816B0623654D044607686426644A90F812
:10EEC0003500B5FBF1F189B2FEF7C4FC438800219F
:10EED00080463846B5FBF3F52564FFF777FD8022C1
:10EEE0006B213846FFF71CFE05F006FE04460D4672
:10EEF00005F002FE001B61EB0501B0F57A7F71F1B0
:10EF00000001F5D3013EEFD164260722682138467F
:10EF1000FFF706FE05F0F0FD04460D4605F0ECFD9A
:10EF2000001B61EB0501B0F57A7F71F10001F5D3AB
:10EF3000013EEFD1324664266B213846FFF7F0FDE3
:10EF400005F0DAFD04460D4605F0D6FD001B61EB29
:10EF50000501B0F57A7F71F10001F5D3013EEFD1E3
:10EF60000F2601226B213846FFF7DAFD05F0C4FDBC
:10EF700004460D4605F0C0FD001B61EB0501B0F530
:10EF80007A7F71F10001F5D3013EEFD10F261822EF
:10EF90001B213846FFF7C4FD05F0AEFD04460D46C3
:10EFA00005F0AAFD001B61EB0501B0F57A7F71F158
:10EFB0000001F5D3013EEFD10F2618221C2138465F
:10EFC000FFF7AEFD05F098FD04460D4605F094FDF3
:10EFD000001B61EB0501B0F57A7F71F10001F5D3FB
:10EFE000013EEFD10F2698F804201A213846FFF78A
:10EFF00097FD05F081FD04460D4605F07DFD001BE3
:10F0000061EB0501B0F57A7F71F10001F5D3013EA6
:10F01000EFD1642698F8052019213846FFF780FDC6
:10F0200005F06AFD04460D4605F066FD001B61EB28
:10F030000501B0F57A7F71F10001F5D3013EEFD102
:10F0400038460321BDE8F041C0E400BF40420F0054
:10F05000AC7C0C082AE700BF00680379012B09D0BB
:10F06000022B01D0002070478368F022DB0717D500
:10F07000FF21F5E4826890F910C002F00102417CA2
:10F0800060464FF0F00C10B584B00DF10F04019202
:10F09000FF228DF80FC00094F4F764FB04B010BD9C
:10F0A0007F21DDE40068CA43037941EA0211012BA4
:10F0B000CAB208D0022B01D0002070478368DB075A
:10F0C00015D5D221CCE410B584B0846890F910C075
:10F0D0008DF80F200DF10F0204F00104417C009225
:10F0E000D22260460194F4F73DFB04B010BD5221DA
:10F0F000B6E400BF00680379012B09D0022B01D0D0
:10F10000002070478368B422DB0717D5FF21A7E4EE
:10F11000826890F910C002F00102417C60464FF015
:10F12000B40C10B584B00DF10F040192FF228DF8DC
:10F130000FC00094F4F716FB04B010BD7F218FE4DC
:10F1400000680379012B09D0022B01D00020704701
:10F1500083680A46DB0715D5A52181E410B584B084
:10F16000846890F910C00DF10F0204F001048DF8CD
:10F170000F10417C60460092A5220194F4F7F2FA48
:10F1800004B010BD25216BE400680379012B09D080
:10F19000022B01D00020704783689622DB0717D529
:10F1A000FF215DE4826890F910C002F00102417C09
:10F1B00060464FF0960C10B584B00DF10F0401922B
:10F1C000FF228DF80FC00094F4F7CCFA04B010BD04
:10F1D0007F2145E400680379012B09D0022B01D07F
:10F1E0000020704783680A46DB0715D5872137E47E
:10F1F00010B584B0846890F910C00DF10F0204F0CE
:10F2000001048DF80F10417C604600928722019422
:10F21000F4F7A8FA04B010BD072121E40068C90181
:10F220000379CAB2012B05D0022B01D00020704710
:10F23000782115E410B584B0846890F910C08DF879
:10F240000F200DF10F0204F00104417C009278229E
:10F2500060460194F4F786FA04B010BD00680379A3
:10F26000012B0AD0022B01D0002070478368552261
:10F27000DB0718D5A521FFF7F3BB826890F910C012
:10F2800002F00102417C60464FF0550C10B584B08D
:10F290000DF10F040192A5228DF80FC00094F4F730
:10F2A00061FA04B010BD2521FFF7DABB00680379CD
:10F2B000012B0AD0022B01D00020704783682E2238
:10F2C000DB0718D5F421FFF7CBBB826890F910C09B
:10F2D00002F00102417C60464FF02E0C10B584B064
:10F2E0000DF10F040192F4228DF80FC00094F4F791
:10F2F00039FA04B010BD7421FFF7B2BB154B00689A
:10F300001A8F03799201012B02F13402D2B209D093
:10F31000022B01D0002070478368DB0716D5F4214B
:10F32000FFF79EBB10B584B0846890F910C08DF8CB
:10F330000F200DF10F0204F00104417C0092F42231
:10F3400060460194F4F70EFA04B010BD7421FFF783
:10F3500087BB00BF00650024006810B5037984B046
:10F36000012B0FD0022B02D0012004B010BD836806
:10F370003122DB074CBFF4217421FFF771FB012020
:10F3800004B010BD82680DF10F0490F910C002F0B6
:10F390000102417C60464FF0310C0192F42200944E
:10F3A0008DF80FC0F4F7DEF9012004B010BD00BFE6
:10F3B00000680379012B07D0022B01D00020704791
:10F3C00001225821FFF74CBB8268417C02F0010208
:10F3D00010B590F9104084B020460DF10F04019251
:10F3E000582200948DF80F30F4F7BCF904B010BD2A
:10F3F00000680379012B07D0022B01D00020704751
:10F4000001224821FFF72CBB8268417C02F00102F7
:10F4100010B590F9104084B020460DF10F04019210
:10F42000482200948DF80F30F4F79CF904B010BD19
:10F4300000680379012B07D0022B01D00020704710
:10F440001A460821FFF70CBB826890F910C002F041
:10F450000102417C60464FF0020C10B584B00DF102
:10F460000F04019208228DF80FC00094F4F77AF986
:10F4700004B010BD00680379012B07D0022B01D026
:10F480000020704701220821FFF7EABA8268417C18
:10F4900002F0010210B590F9104084B020460DF141
:10F4A0000F040192082200948DF80F30F4F75AF9F6
:10F4B00004B010BD2DE9F04105461F462948164607
:10F4C00095F9103082B003EB430350F83380AB68FA
:10F4D0009A0716D501230DF106028DF80610404655
:10F4E0000DF10701F4F750FE3B463246002140463D
:10F4F000F4F74AFEAB689B0719D5012002B0BDE8BE
:10F50000F0816B691BB19A88186812048261164BEE
:10F51000D3F8E809154BC000A3FB0030144B800959
:10F520005A685C68A4EB020C6045FAD2D2E70E4A36
:10F530004FF4FA700D4BD2F8E8290D4900FB02F2A6
:10F540004868A3FB023292094B681B1A9A42FBD20D
:10F550006B69002BD1D01A6801209B88936102B09F
:10F56000BDE8F081AC02002400650024D34D621098
:10F57000001000E030B5057983B084468E46012D39
:10F580000DD0022D02D0002003B030BD8468E40706
:10F5900058BF01F07F0103B0BDE830408AE78068C2
:10F5A00014460A46009400F001049CF811109CF9DE
:10F5B00010000194F4F7D6F803B030BD2DE9F04106
:10F5C00005461F462948164695F9103082B003EBD0
:10F5D000430350F83380AB689A0716D501230DF129
:10F5E00006028DF8061040460DF10701F4F7CCFD38
:10F5F0003B46002231464046F4F7C6FDAB689B0708
:10F6000019D5012002B0BDE8F0816B691BB19A8861
:10F61000186812048261164BD3F8E809154BC00034
:10F62000A3FB0030144B80095A685C68A4EB020C01
:10F630006045FAD2D2E70E4A4FF4FA700D4BD2F879
:10F64000E8290D4900FB02F24868A3FB0232920947
:10F650004B681B1A9A42FBD26B69002BD1D01A68F7
:10F6600001209B88936102B0BDE8F081AC020024C8
:10F6700000650024D34D6210001000E030B505791C
:10F6800083B084468E46012D0DD0022D02D000207D
:10F6900003B030BD8468E40758BF41F0800103B077
:10F6A000BDE830408AE7806814460A46009400F0BE
:10F6B00001049CF811109CF910000194F4F76EFA03
:10F6C00003B030BD2DE9F043816B85B0804C06233B
:10F6D000076880467F4A962690F83500B4FBF1F122
:10F6E00089B2FEF7B7F84388002181463846B4FB5B
:10F6F000F3F4C8F84040FFF769F980226B213846DF
:10F70000FFF70EFA05F0F8F904460D4605F0F4F996
:10F71000001B61EB0501B0F57A7F71F10001F5D3B3
:10F72000013EEFD19626032268213846FFF7F8F90B
:10F7300005F0E2F904460D4605F0DEF9001B61EB29
:10F740000501B0F57A7F71F10001F5D3013EEFD1EB
:10F7500003226B213846FFF7E3F905F0CDF90446A3
:10F760000D4605F0C9F9001B61EB05010F2871F189
:10F770000001F6D310226A213846FFF7D1F905F0CF
:10F78000BBF904460D4605F0B7F9001B61EB050116
:10F790000F2871F10001F6D300226C213846FFF7E3
:10F7A000BFF905F0A9F904460D4605F0A5F9001BBF
:10F7B00061EB05010F2871F10001F6D399F80520DE
:10F7C00019213846FFF7ACF905F096F904460D46C5
:10F7D00005F092F9001B61EB05010F2871F10001A2
:10F7E000F6D318221B213846FFF79AF905F084F961
:10F7F00004460D4605F080F9001B61EB05010F285A
:10F8000071F10001F6D318221C213846FFF788F960
:10F8100005F072F904460D4605F06EF9001B61EB28
:10F8200005010F2871F10001F6D399F804201A217F
:10F830003846FFF775F905F05FF905460C4605F007
:10F840005BF98C4208BF8542F9D003213846FFF7A7
:10F85000BDF8062302AA4321D8F80000FFF70EFFE7
:10F8600028B3BDF80810BDF80A30BDF80C20C9BA9D
:10F87000DBBA07EE901AD2BAF8EEE76A07EE102A62
:10F8800007EE903AB8EEC77AF8EEE77AC8ED076A65
:10F8900088ED097AC8ED087AFDEEE77ACDED017AB8
:10F8A0009DF90430013305D005B0BDE8F083D8EDF3
:10F8B000087AF1E7D8ED077AFDEEE77ACDED017A27
:10F8C0009DF904300133EFD1062005F0F3FD00BFB0
:10F8D00040420F00AC7C0C0870B5066882B005464B
:10F8E000F469002C3ED03379221D012B2DD0022B40
:10F8F00026D1B368304613F0010F4FF00C030CBF54
:10F900008C211946FFF75AFEA070D8B1B4F9043023
:10F9100007EE903AF8EEE77AC5ED077AB4F90630CB
:10F9200007EE903AF8EEE77AC5ED087AB4F90830B8
:10F9300007EE903AF8EEE77AC5ED097A02B070BDAD
:10F940000023A370002002B070BDB368717C03F087
:10F95000010396F91000009201930C231A46F4F764
:10F960001DF9D1E709211420FDF79EFEF061044640
:10F970002E68B8E770B5066882B00546F469002CB9
:10F980003ED03379E21C012B2DD0022B26D1B36857
:10F99000304613F0010F4FF00D0314BF0C218C21E2
:10F9A000FFF70CFEA070D8B1B4F90A3007EE903A18
:10F9B000F8EEE77AC5ED077AB4F90C3007EE903A25
:10F9C000F8EEE77AC5ED087AB4F90E3007EE903A12
:10F9D000F8EEE77AC5ED097A02B070BD0023A37096
:10F9E000002002B070BDB368717C03F0010396F98A
:10F9F000100000920C2201930D23F4F7CFF8D1E709
:10FA000009211420FDF750FEF06104462E68B8E786
:10FA1000006810B5037984B00C46012B1AD0022B74
:10FA200002D0002004B010BD836803AA13F0010FB8
:10FA30004FF0030314BF2221A221FFF7BFFD0028CE
:10FA4000EFD0BDF90D3003EB83031B12E6332380A7
:10FA500004B010BD836803AA417C03F0010390F950
:10FA600010000092222201930323F4F797F8E6E7AF
:10FA700070B5066882B00546F469002C3ED0337933
:10FA8000221D012B2DD0022B26D1B368304613F056
:10FA9000010F4FF00E0314BF3B21BB21FFF78EFD7A
:10FAA000A070D8B1A389DBBA07EE903AF8EEE77AF6
:10FAB000C5ED077AE389DBBA07EE903AF8EEE77A0C
:10FAC000C5ED087A238ADBBA07EE903AF8EEE77ABA
:10FAD000C5ED097A02B070BD0023A370002002B00A
:10FAE00070BDB368717C03F0010396F910000092B9
:10FAF0003B2201930E23F4F751F8D1E7092114209A
:10FB0000FDF7D2FD0446F061B9E700BF006810B50B
:10FB1000037984B0012B10D0022B01D000200AE021
:10FB200003AAF621FFF74AFD0028F7D0BDF80C30F4
:10FB3000094A5BBA138304B010BD826803AC417CF0
:10FB4000022302F0010290F91000CDE90042F622F2
:10FB5000F4F724F8E8E700BF00650024006810B55A
:10FB6000037984B0012B1DD0022B01D0002017E0B7
:10FB7000032303AAF621FFF721FD0028F6D09DF804
:10FB80000D309DF80CC01B020D499DF80E2043EA74
:10FB90000C431343B1F93820C2F10802D340CB63C0
:10FBA00004B010BD826803AC417C032302F0010263
:10FBB00090F91000CDE90042F622F3F7EFFFDCE701
:10FBC00000650024006810B5037984B0012B31D0A2
:10FBD000022B09D01E490020D1F8EC39D1F8F029C8
:10FBE0000B660A6404B010BD062302AAF721FFF7D2
:10FBF000E5FC0028EED09DF809309DF80C209DF81A
:10FC000008C01B019DF80BE012019DF80A1043EAA1
:10FC10000C3342EA0E329DF80DC043EA11130C4931
:10FC200042EA1C12C1F8EC39C1F8F0290A640B66EB
:10FC300004B010BD826802AC417C062302F00102D0
:10FC400090F91000CDE90042F722F3F7A7FFD0E7C3
:10FC500000650024006810B5037984B0012B1DD025
:10FC6000022B0FD09DF80D3001209DF80CC01B0217
:10FC70009DF80E10104A43EA0C430B43C2F888303B
:10FC800004B010BD836803AA13F0010F4FF0030303
:10FC900014BF00218021FFF791FCE3E7826803ACE9
:10FCA000417C032302F0010290F91000CDE90042EB
:10FCB0000022F3F773FFD5E700650024006810B554
:10FCC000037984B0012B1DD0022B0FD09DF80D308D
:10FCD00001209DF80CC01B029DF80E10104A43EA4B
:10FCE0000C430B43C2F89C3004B010BD836803AAD8
:10FCF00013F0010F4FF0030314BF00218021FFF721
:10FD00005DFCE3E7826803AC417C032302F001025F
:10FD100090F91000CDE900420022F3F73FFFD5E74C
:10FD200000650024006810B5037984B0012B28D049
:10FD3000022B01D0002022E0836803AA13F0010FF8
:10FD40004FF003030CBF83211946FFF737FC00284F
:10FD5000F0D09DF80C309DF90C109DF80D201B047F
:10FD600000299DF80EC043EA02230D4AACBF0021D2
:10FD70004FF07F4143EA0C030B43C2F8103104B04B
:10FD800010BD826803AC0323417C02F0010290F9AC
:10FD90001000CDE900421A46F3F700FFD7E700BF95
:10FDA00000650024006810B5037984B0012B28D0C9
:10FDB000022B01D0002022E0836803AA13F0010F78
:10FDC0004FF0030314BF00218021FFF7F7FB002849
:10FDD000F0D09DF80C309DF90C109DF80D201B04FF
:10FDE00000299DF80EC043EA02230D4AACBF002152
:10FDF0004FF07F4143EA0C030B43C2F80C3104B0CF
:10FE000010BD826803AC417C032302F0010290F92B
:10FE10001000CDE900420022F3F7C0FED7E700BF93
:10FE20000065002490F91030F0B503EB4303274E32
:10FE3000154683B056F83360044683689A0715D593
:10FE400001230DF106028DF8061030460DF1070171
:10FE5000F4F79AF90123002229463046F4F794F981
:10FE6000A3689B0717D5012003B0F0BD43691BB100
:10FE70009A88186812048261154B164AD3F8E8096B
:10FE8000154BC0005768A3FB003080095368DB1B8B
:10FE90009842FBD2D4E70E4A4FF4FA700E4BD2F8D8
:10FEA000E8290C4900FB02F24868A3FB02329209E0
:10FEB0004B681B1A9A42FBD26369002BD3D01A6895
:10FEC00001209B88936103B0F0BD00BFAC02002409
:10FED00000650024001000E0D34D621010B50379D6
:10FEE00082B08E46012B0DD0022B02D0002002B032
:10FEF00010BD8368DB0758BF41F0800102B0BDE848
:10FF000010408FE7816814467246009401F00104A6
:10FF1000417C90F910000194F3F740FE02B010BD4F
:10FF200070B5056884B004460E462B79012B15D0B8
:10FF3000022B02D0002004B070BDAB68E122DB07C9
:10FF40001CD528461146FEF78BFD0028F2D032461C
:10FF5000FF21206804B0BDE87040BFE7AA68697C53
:10FF600002F0010295F910000DF10F050192E12256
:10FF700000958DF80F20F3F7F5FBE6E761212846A1
:10FF8000FEF76EFDE1E700BF70B5056884B004467A
:10FF90000E462B79012B16D0022B02D0002004B084
:10FFA00070BDAB68C3222846DB074CBFE12161214D
:10FFB000FEF756FD0028F1D03246FF21206804B03C
:10FFC000BDE870408AE7AA6895F9100002F00102C6
:10FFD000697C01920DF10F020092C3228DF80F206F
:10FFE000E122F3F7BFFBE5E770B5056884B004468E
:10FFF0000E462B79012B1BD0022B02D0002004B01F
:020000040805ED
:1000000070BDAB68F0222846DB074CBFE1216121BF
:10001000FEF726FD0028F1D02246FF2152F8040BFE
:10002000FFF75CFF0028E9D02379337004B070BD7E
:10003000AA6895F9100002F00102697C01920DF1A5
:100040000F020092F0228DF80F20E122F3F78AFBD5
:10005000E0E700BFF0B5046883B0002107466426DE
:100060002046FEF7B3FC15227E212046FEF758FD00
:1000700004F042FD04460D4604F03EFD001B61EB1A
:100080000501B0F57A7F71F10001F5D3013EEFD1A2
:10009000052611227E213868FEF742FD04F02CFD72
:1000A00004460D4604F028FD001B61EB0501B0F588
:1000B0007A7F71F10001F5D3013EEFD10DF1070216
:1000C00003213868FFF70AFF9DF8073003F03C036F
:1000D000142B40F09B800C2240213868FEF720FD55
:1000E00004F00AFD04460D4604F006FD001B61EB1A
:1000F0000501B0F57A7F71F10001F5D3454C092374
:10010000B96B454A97F83500B4FBF1F189B2FDF7B8
:10011000A1FB0346422138685A88B4FBF2F43C64E0
:100120001A79FEF7FDFC04F0E7FC04460D4604F0E6
:10013000E3FC001B61EB0501B0F57A7F71F1000172
:10014000F5D3082241213868FEF7EAFC04F0D4FC1C
:1001500004460D4604F0D0FC001B61EB0501B0F530
:100160007A7F71F10001F5D3002243213868FEF750
:10017000D7FC04F0C1FC04460D4604F0BDFC001B96
:1001800061EB0501B0F57A7F71F10001F5D3102222
:1001900051213868FEF7C4FC04F0AEFC04460D465D
:1001A00004F0AAFC001B61EB0501B0F57A7F71F148
:1001B0000001F5D30A2253213868FEF7B1FC04F0A0
:1001C0009BFC04460D4604F097FC001B61EB050107
:1001D000B0F57A7F71F10001F5D38022562138689D
:1001E000FEF79EFC04F088FC04460D4604F084FCF7
:1001F000001B61EB0501B0F57A7F71F10001F5D3C9
:1002000003213868FEF7E2FB03B0F0BD062005F0DD
:1002100051F900BF40420F0014810C08F0B583B0C3
:1002200015461C4606460DF107020F46FFF756FE1F
:100230009DF8072005EA0203A34201D103B0F0BDF7
:1002400022EA050239463046224303B0BDE8F040B9
:10025000FEF766BC10B582B00821044600686A4605
:10026000FFF73CFE9DF80030DB0602D4002002B010
:1002700010BD06236A4600212068FFF7FFF9002819
:10028000F4D09DF801209DF8001012029DF8023074
:10029000DFED4A6A02EB01429DF8041014024FEAB6
:1002A00001219DF8034013449DF8052001EB044112
:1002B00048BF03F17F430A44090207EE903A404BDE
:1002C00048BF02F17F42F8EEE77A93ED1B6A07EE32
:1002D000102AB3F97020F8EEC65AB3F97610B8EECA
:1002E000C77A04EE901AB3F97A10C7EE263A87EE71
:1002F000A67A06EE902A334AD3ED1A7A92F82C4168
:10030000B3F97220F8EEE66A112C06EE102AB3F962
:100310007420F8EEE77A05EE102AB3F97820B8EEEB
:10032000C66A04EE102AB8EEC55AF8EEE44AB3F9EC
:100330007C20B8EEC44A66EEA36A27EE232A23D0B7
:10034000A7EE045AA7EE246AE5EE075AE5EE877A8F
:1003500077EEA67AE6EE027AB3F96620F6EE006A48
:10036000C3ED207A07EE902AB3F96410F8EEE77A2D
:1003700007EE101AB8EEC77A67EEA37AE7EE267A90
:10038000C3ED217A02B010BD03EE102AF8EEC32AA5
:1003900003EE101AB8EEC33AA7EE224AE7EE034A7C
:1003A000A4EE075AA4EE876AE5EE075AE5EE877ACF
:1003B00077EEA67AE6EE027ACEE700BF0000784834
:1003C00000650024D8B90024F0B5044683B00D467A
:1003D0001746061D20680379012B19D0022B02D085
:1003E000002003B0F0BD83683246FF21DB075CBF0D
:1003F0003246FF21FFF716FD0028F1D015B1237911
:10040000DB07E7D4002FECD023793B7003B0F0BDBD
:100410008268417C02F0010C90F91000FF22CDE9C6
:10042000006CF3F7BBFBE7E770B50446051D82B02F
:1004300020680379012B16D0022B02D0002002B0D5
:1004400070BD83682A46FF21DE075CBF2A46FF2174
:10045000FFF7E8FC0028F1D02379DB07EFD520680F
:100460000379012BE8D18668FF22417C06F0010662
:1004700090F91000CDE90056F3F790FBEAE700BFD2
:10048000024630B5044652F8040B83B00379012BC1
:100490000ED0022B01D0002008E0FF21FFF7C2FCA4
:1004A0000028F8D02079C04300F0010003B030BD2F
:1004B0008568417C05F0010590F910000092FF224B
:1004C0000195F3F76BFBEBE770B5B42282B00446FD
:1004D000FF210068FEF724FB10B9002002B070BDB8
:1004E0002068251D0379012B13D0022BF5D18368D9
:1004F0002A46FF21DE075CBF2A46FF21FFF792FC58
:100500000028EAD02379DB07E8D520680379012B9E
:10051000EBD18668FF22417C06F0010690F91000BD
:10052000CDE90056F3F73AFBEAE700BF70B50A469B
:1005300082B00446A5210068FEF7F2FA10B9002047
:1005400002B070BD2068251D0379012B13D0022B4A
:10055000F5D183682A46FF21DE075CBF2A46FF21CA
:10056000FFF760FC0028EAD02379DB07E8D5206894
:100570000379012BEBD18668FF22417C06F001064E
:1005800090F91000CDE90056F3F708FBEAE700BF49
:1005900070B582B00446CDE90023FFF795FF10B98E
:1005A000002002B070BD5522A5212068FEF7B8FAE0
:1005B0000028F5D0251D2A46FF212068FFF78EFC74
:1005C0000028EDD02379DB07F5D40DF1FF350DF1CF
:1005D000070615F8011F2046FFF7A8FF0028DFD007
:1005E000B542F6D1DDE700BF002A34D0F0B50446AD
:1005F00083B00E46051D8F1816F8012BA521206823
:10060000FEF78EFA90B9002003B0F0BD8268417CFD
:1006100002F0010C90F91000FF22CDE9005CF3F725
:10062000BDFA0028EFD02379DB070FD520680379C6
:10063000012BEBD0022BE6D183682A46FF21DB0792
:100640005CBF2A46FF21FFF7EDFBEAE7B742D3D1B3
:10065000012003B0F0BD0120704700BFF0B5962225
:1006600083B00E460446FF210068FEF759FA10B920
:10067000002003B0F0BD251D20680379012B1DD09B
:10068000022BF5D183682A46FF21DF075CBF2A468B
:10069000FF21FFF7C7FB0028EAD02379DB07EBD463
:1006A000E12220681146FEF73BFA0028E0D03246EE
:1006B000FF21206803B0BDE8F0400FE48768FF2207
:1006C000417C07F0010790F91000CDE90057F3F7DE
:1006D00065FAE0E7002A42D0F0B5044683B00E4642
:1006E000051D8F189622FF212068FEF719FA90B990
:1006F000002003B0F0BD8268417C02F0010C90F94B
:100700001000FF22CDE9005CF3F748FA0028EFD093
:100710002379DB070FD520680379012BEBD0022B5F
:10072000E6D183682A46FF21DB075CBF2A46FF210A
:10073000FFF778FBEAE7E12220681146FEF7F0F9BF
:100740000028D5D03246FF212068FFF7C7FB0028DC
:10075000CED00136B742C5D1012003B0F0BD012093
:10076000704700BFF0B50B4605461646044683B0F9
:1007700087211A4655F8040BFEF7D2F92068037951
:10078000012B19D0022B02D0002003B0F0BD8368EA
:100790002A46FF21DF075CBF2A46FF21FFF742FB05
:1007A0000028F1D02379DA07E8D4002EEDD0C3F386
:1007B0004013337003B0F0BD8768FF22417C07F01F
:1007C000010790F91000CDE90057F3F7E7F9E7E7E3
:1007D000F0B5782183B01646044600220068FEF783
:1007E0009FF910B9002003B0F0BD251D20680379E2
:1007F000012B13D0022BF5D183682A46FF21DF0796
:100800005CBF2A46FF21FFF70DFB0028EAD02379C1
:10081000DA07EBD45B09337003B0F0BD8768FF22C1
:10082000417C07F0010790F91000CDE90057F3F77C
:10083000B5F9EAE770B5CC2282B00446A52100687C
:10084000FEF76EF910B9002002B070BD2068251DBA
:100850000379012B13D0022BF5D183682A46FF219F
:10086000DE075CBF2A46FF21FFF7DCFA0028EAD04A
:100870002379DB07E8D520680379012BEBD1866863
:10088000FF22417C06F0010690F91000CDE90056E8
:10089000F3F784F9EAE700BF70B5B42282B00446EA
:1008A000FF210068FEF73CF910B9002002B070BDCE
:1008B000251D20680379012B21D0022BF5D18368F7
:1008C0002A46FF21DE075CBF2A46FF21FFF7AAFA6E
:1008D0000028EAD02379DA07EBD4CC212046FFF7B1
:1008E00025FE0028E1D002E02379DB07DED52A4689
:1008F000FF212068FFF7F2FA0028F5D1D5E78668D6
:10090000FF22417C06F0010690F91000CDE9005667
:10091000F3F744F9DCE700BF2DE9F04F82468DB0D4
:10092000002090460AF10407089106900A93079068
:10093000069B5046DC0008EBC3030593FFF7C4FD9C
:1009400028B941E09AF8043013F0010208D03A4681
:10095000FF21DAF80000FFF7C1FA0028F2D133E0F6
:1009600003929A070B9040F1CC80F0215046FFF79C
:10097000DDFD48B3083CDDF80C9008EB04030124CE
:1009800009932546089B003B18BF01230493049B51
:10099000082D8CBF002303F001039B46002B5DD084
:1009A0006E1E089B43FA06F606F00106F201782156
:1009B000DAF80000FEF7B4F830B1DAF80000037995
:1009C000012B3FD0022B07D000220A9B104606992C
:1009D00019700DB0BDE8F08F83683A46FF21DB0740
:1009E0005CBF3A46FF21FFF71DFA0028ECD09AF8C9
:1009F000043013F00102E0D199094FEA531E4FEA87
:100A0000D31C01EA5313DB074BD4664502D0BBF17C
:100A1000000F73D1BCF1000F2DD0059911F80930EA
:100A2000234301F809306400013514F0FF04EDB2EE
:100A3000ADD109F101095FFA89F9B9F1080F30D098
:100A40000124A4E78268417C02F0010C90F91000B7
:100A5000FF22CDE9007CF3F7A1F8C6E7069BD3B1EE
:100A6000079BAB4217D9099B13F809301C4214BFEE
:100A7000012600269AE74EEA0101039B11F0010FBF
:100A8000059908BF2B46039311F8093023EA0403A4
:100A900001F80930C7E7079B5E1BB6FA86F67609B0
:100AA00084E7402D07D80A9B069A1B7893423FF6AD
:100AB0003FAF024689E7059BDD795C1E9E1D14F859
:100AC00001CF082182EA0C0301394FEA5C0C43F3A1
:100AD000000311F0FF0123F0730383EA5202D2B244
:100AE000F0D1A642EBD19542DDD1069B0133DBB2BA
:100AF0000693039B002BDCD00793D4E70B9E324672
:100B000063E70646324660E710B50446006882B0E7
:100B100003796A46022B4FF006030CBF43210321E1
:100B2000FEF7ACFD68B1BDF80010BDF80220BDF8BD
:100B3000043049BA52BA5BBAE1866287238702B0B1
:100B400010BDC4F83600608702B010BD30B5002378
:100B500085B004460221C0F836300DF10702438704
:100B60000068FFF7BBF918B19DF80730DB0703D425
:100B70000025284605B030BD062302AA03212068BF
:100B8000FEF77CFD0DF1070209212068FFF7A6F9A9
:100B900005460028ECD09DF8073013F00C0FE7D184
:100BA000BDF80820BDF80C30BDF80A10C2EB823247
:100BB000C3EB8333206889009B0092002187638701
:100BC0000A21E2860122FDF7ABFF284605B030BDC1
:100BD00010B50446002221210068FDF7A1FFFC2288
:100BE00020212068FDF79CFF402224212068FDF78A
:100BF00097FF0C2223212068FDF792FF002222217B
:100C00002068FDF78DFF012010BD00BF10B5044620
:100C100094220B210068FDF783FF712201212068D7
:100C2000FDF77EFF002204212068FDF779FFC8222E
:100C300005212068FDF774FF002206212068FDF7DA
:100C40006FFFC82207212068FDF76AFF00220821F4
:100C50002068FDF765FFC82209212068FDF760FFC5
:100C6000012010BD01207047044B0022002101200B
:100C70001A605A609A60D960704700BF80D800241B
:100C8000104B11491A680346C868121AFA2A16D876
:100C9000D1ED006A012091ED017AFDEEE66AD1ED19
:100CA000027ABDEEC77AFDEEE77A16EE902ADA8672
:100CB00017EE102A1A8717EE902A5A8770470020DD
:100CC000704700BF742F002480D800240E4B70B5ED
:100CD0001B7C82B00191ABB90C4B1D6895B12B68A0
:100CE0001A687AB19B686BB104462846984748B1A8
:100CF000019922462E6828460B46316802B0BDE8AD
:100D00007040084702B070BD80D80024E8A90024D4
:100D10000B4B70B51E688EB133681A6872B19B6850
:100D200063B1054630460C46984738B131682A46CB
:100D3000234630460968BDE87040084770BD00BFD3
:100D400000AA0024014B5B695B68184780D8002427
:100D5000024B08305B699B68184700BF80D80024AD
:100D60000120704701207047012070470120704723
:100D70000120704731B10B4BD3ED067AF8EEE77ADC
:100D8000C1ED007A6AB10749074BC969DFED076A0F
:100D90000B4407EE903AF8EEE77A87EEA67A82EDFA
:100DA000007A704780D800244D95FFFF0000C842AC
:100DB00001207047012070477A4A0146002394467B
:100DC000104610B490F904400C30012C4DD0013382
:100DD000082BF7D1734C002394F904000C3402283B
:100DE00058D00133082BF7D16E4C002394F904003E
:100DF0000C3403286BD00133082BF7D1694C002346
:100E000094F904000C34052877D00133082BF7D16E
:100E1000644C002394F904000C34062800F083800D
:100E20000133082BF6D1002392F904000C32072875
:100E300000F093800133082BF6D15B4B1B68DC0379
:100E400040F1A180594B086803F58C7403E014331A
:100E5000A34200F098801A689042F8D1DA68D20173
:100E6000F5D501205DF8044B704703EB43035CF8B4
:100E7000233023B34E480B7990F8D14090F8D0003E
:100E8000984218BF9C420CBF01200020A2D15DF8FF
:100E9000044B704703EB43035CF823308BB14548A8
:100EA0000B7990F8D04090F8D100984218BF9C423E
:100EB0000CBF0120002097D15DF8044B7047394CDE
:100EC0008AE7384C94F904000C34032893D103EBDF
:100ED00043035CF82330002B3BD037480B7990F864
:100EE000D04090F8D100984218BF9C420CBF01201E
:100EF000002083D15DF8044B704703EB43035CF89B
:100F0000233043B32D480B7990F8D04090F8D100AE
:100F1000984218BF9C420CBF012000207FF478AF9C
:100F20005DF8044B704703EB43035CF82330002B60
:100F30003FF47AAF22480B7990F8D04090F8D10076
:100F4000984218BF9C420CBF012000208AD0034663
:100F50006AE7144C54E7134C5CE703EB43035CF87B
:100F60002330002B3FF469AF164A0B7992F8D10079
:100F700092F8D0209A4218BF98420CBF012000205E
:100F80007FF45BAF6EE70B79312B04D82F2B94BF26
:100F90000020012066E7343B012B8CBF002001209C
:100FA00060E700BF78890024A46F0024141B00248C
:100FB000340600240C090024E40B0024BC0E002499
:100FC000941100246C1400240B4B8446002010B5AF
:100FD00003F58C7E02E014339E450BD01A686245FF
:100FE000F9D1DA68441C8A42F5D0D9601433E0B2F2
:100FF0009E45F3D110BD00BF141B0024704700BFF5
:1010000040F2FF72034B914203EBC003A8BF1146AD
:101010009984704780D80024112807D8044B03EB2B
:101020008003D3F880300BB19B68196028F080BA38
:1010300080D80024112807D8044B03EB8003D3F891
:1010400080300BB19B681960704700BF80D80024C6
:10105000F0B5484D83B095F8C8303BB195F8C960FC
:101060000446012E38D0022E54D00EB103B0F0BD8C
:10107000012280210068FDF753FD0122FF21206835
:10108000FDF74EFD324631462068FDF749FD95F8E3
:10109000CA2091212068FDF743FD314601222068D6
:1010A000FDF73EFD3246FF212068FDF739FD32464F
:1010B00080212068FDF734FD314601222068FDF7CC
:1010C0002FFD2D4B2D4901221B68087085F8C92082
:1010D000C5F8CC3003B0F0BD01AA00210068FEF7CE
:1010E000FDFE9DF80430254FDA07387039D5D5F864
:1010F000D030002BBAD0204AD5F8CC10126892B26A
:10110000521A9342B2D24FF0FF3200237A6085F830
:10111000C930ABE701AA13210068FEF7DFFE9DF896
:101120000430164F5B073870E1D0334601AA1E2108
:101130002068FEF7A3FABDF80430206801225CBAEB
:101140000B21FDF7EDFC0E4BA4B201223870A3FB7E
:101150000434002385F8D420E40885F8C9307C6085
:1011600084E7054B02221B6885F8C920C5F8CC30FE
:101170007CE700BF80D80024742F00241C270024A3
:10118000CDCCCCCC0C4A13787BB10C4B93F8C81067
:1011900059B193F8D41059B150680022FA2883F855
:1011A000D420A8BF4FF0FF3070476FF001007047A8
:1011B0006FF00200704700BF1C27002480D8002475
:1011C0002DE9F041104C00251746022304F1D80800
:1011D00084F8D910FF210646424684F8D850FEF71D
:1011E000C9F968B1424630460223FF21FEF746FAAC
:1011F00030B1B4F8D83028465BBA3B80BDE8F08106
:101200006FF00C00FAE700BF80D800240B4B93F876
:10121000D82182B193F8D92152B1094900228868B6
:1012200083F8D921B0F5967FA8BF4FF0FF30704703
:101230006FF0020070476FF00100704780D8002403
:101240001C270024024BD3F8DC315B68184700BF31
:1012500080D80024024BD3F8DC319B68184700BFCC
:1012600080D80024024BD3F8DC31DB68184700BF7C
:1012700080D80024014BD868704700BF1C27002489
:10128000044B93F8E03113B1034B186970476FF0CA
:101290000100704780D800241C27002438B52D4D4C
:1012A00004460323002105F118020068FEF7E6F961
:1012B00048B96FF00103002220686B611146BDE858
:1012C0003840FDF72DBC95F81AC008212B7E58B286
:1012D0005B0042000028DBB282F00702B8BFD3B245
:1012E0000139F4D16A7E5340082258B25B004100B4
:1012F0000028DBB281F00701B8BFCBB2013AF4D1CC
:101300009C45206815D12B8B4FF6FD7C5BBA9BB2B8
:10131000591E89B2614514D807EE903AF2EE046A7C
:10132000F8EEE77A87EEA67AFDEEC77A17EE903AE6
:10133000C1E76FF0020311466B61BDE83840FDF76D
:10134000EFBB4FF0FF3311466B61BDE83840FDF74E
:10135000E7BB00BF1C270024014B5869704700BF42
:101360001C270024437A5A1C0344D2B24272997259
:10137000037A934200D802B97047036800F10A016A
:1013800010B50446406898470023637210BD00BF43
:10139000026830B5137985B00446012B61D0022B69
:1013A00003D00025284605B030BD916802AD104637
:1013B000C9072A464CBF19468221FEF733FD002893
:1013C000EFD09DF80830DA07EBD52A460723032132
:1013D0002068FEF753F905460028E2D011220A21C1
:1013E0002068FDF79DFB9DF80E301B07D9D42A49D4
:1013F000BDF80830B1F8E42113FB02F3274A934209
:101400003EDBB3F5000F39DA002BB8BFFF331B12F8
:101410005B421BB2BDF80A20E386B1F8E63112FB4D
:1014200003F31E4A93422FDBB3F5000F30DA002B93
:10143000B8BFFF3343F30F22BDF80C30B1F8E81109
:10144000228713FB01F3154A93421BDBB3F5000F10
:101450001CDA002BB8BFFF331B125B421BB2638741
:10146000A0E7517C02AD92F910009268009502F05D
:10147000010201920222F2F791FBA0E7084BC9E7B3
:10148000084BC7E7074BEAE7064AD5E7044BE6E710
:1014900047F6FF72D0E700BF80D8002401FF7FFF2E
:1014A0000180FFFF0080FFFF10B5002386B00446D7
:1014B00000688DF80F300379012B31D0022B02D058
:1014C000002006B010BD83680DF10F02D9074CBF94
:1014D0002721A721FEF7A6FC0028F1D09DF80F30A8
:1014E0001B07EDD5062304AA28212068FEF7C6F8BD
:1014F00028B3BDF91030002BB8BF03339A10BDF9E3
:101500001230002BE286B8BF03339A10BDF91430B5
:10151000002B2287B8BF03339B10638706B010BD32
:101520008268417C02F0010290F910C001920DF135
:101530000F02604600922722F2F730FBCCE7C4F896
:10154000360060870020BCE730B54FF0000C044641
:10155000006887B0C4F836C0A4F83AC00379012BFC
:101560002AD0022B02D0002007B030BD83680DF1D5
:101570000F02D9074CBF61468021FEF753FC0028BB
:10158000F1D09DF80F301B07EDD5062304AA0121E9
:101590002068FEF773F80028E5D0BDF81430BDF8D8
:1015A0001010BDF812205BBA49BA52BA5B42E1860C
:1015B0002287638707B030BD85686246417C05F0AD
:1015C000010590F9100001950DF10F050095F2F756
:1015D000E5FAD4E710B500230446006886B0C4F8E5
:1015E000363063870379012B23D0022B02D00020F1
:1015F00006B010BD83680DF10F02D9074CBF06215C
:101600008621FEF70FFC0028F1D09DF80F30DB0794
:10161000EDD5062304AA00212068FEF72FF8002844
:10162000E5D0049ABDF81430C4F83620638706B0BC
:1016300010BD8268417C02F0010290F910C0019255
:101640000DF10F02604600920622F2F7A7FADAE7E0
:1016500010B500230446006886B0C4F836306387AE
:101660000379012B29D0022B02D0002006B010BD37
:1016700083680DF10F02D9074CBF09218921FEF7BC
:10168000D1FB0028F1D09DF80F30DB07EDD5062304
:1016900004AA01212068FDF7F1FF0028E5D0BDF87C
:1016A0001210BDF81020BDF81430494252425B427E
:1016B000E1862287638706B010BD8268417C02F014
:1016C000010290F910C001920DF10F0260460092E4
:1016D0000922F2F763FAD4E710B500230446006844
:1016E00086B0C4F8363063870379012B12D0022B01
:1016F0000DD183680DF10B02DB074CBF3421B421FF
:10170000FEF790FB18B19DF90B30002B11DB002088
:1017100006B010BD8268417C02F0010290F910C051
:1017200001920DF10B02604600923422F2F736FA74
:10173000E8E7092303AA24212068FDF79FFF00287A
:10174000E5D09DF810209DF80F109DF8133012047D
:101750001B0442EA01629DF8121043EA01639DF8FE
:101760000C10C2F30F42C3F30F43228763879DF827
